:020000040000FA
:107800005469616E59696E673130300000000000C4
:1078100054593230302E3038303030306200000071
:10782000424154333247313339474B3634464200B4
:1078300043414E5F5354440000000000000000002C
:1078400043414E5F43485F300000000000000000ED
:1078500043414E5F3530304B6270730000000000D2
:10786000E8070000E0070000DF070000000000005C
:020000040000FA
:1080000040300020DD800000E5800000E7800000B7
:108010000000000000000000000000000000000060
:10802000000000000000000000000000EF800000E1
:108030000000000000000000F3800000D5A1010056
:10804000ED0D0100310E0100610E0100910E0100E5
:10805000C10E0100F10E0100210F0100510F0100BE
:10806000810F0100B10F0100E50F0100F90F0100C0
:10807000091001003D1001004D1001005D100100CC
:1080800091100100D51001001D11010065110100C2
:10809000AD110100F51101000512010039120100B6
:1080A0006D1201009D120100D112010005130100A3
:1080B0001513010025130100591301008D13010050
:1080C000EF3FE8FF0448854600F02CFA00480047DF
:1080D000D9E50100C046C046403000201648804720
:1080E00016480047FEE7FEE7FEE7FEE7FEE7FEE78D
:1080F000FEE7FEE7FEE7FEE7FEE7FEE7FEE7FEE758
:10810000FEE7FEE7FEE7FEE7FEE7FEE7FEE7FEE747
:10811000FEE7FEE7FEE7FEE7FEE7FEE7FEE7FEE737
:10812000FEE7FEE7FEE7FEE7FEE7FEE7FEE7FEE727
:10813000FEE7FEE7FEE70000DDA70100C5800000C6
:1081400030B50B46014600202022012409E00D46EF
:10815000D5409D4205D31D469540491B2546954077
:1081600040191546521E002DF1DC30BD70B50024BB
:108170002546002801DA01244042002901DA0125C0
:108180004942FFF7DDFFAC4200D04042002C00D056
:10819000494270BDF0B51FB40646002082B00546C6
:1081A0004024019100901BE0019922460F46304681
:1081B00000F066F9049A059B801A994110D3104685
:1081C0001946224600F04CF9361A8F410197224693
:1081D00001200021009F00F043F938184D41009024
:1081E0002046641E0028DFDC019B009829463246A9
:1081F00007B0F0BDF0B51FB486B00020009001902C
:1082000002900698069980B204900798090C02041F
:108210000014114307900027089D099806913E46D7
:108220003C4603900398A9B20204000C0390049802
:108230002D0C154348430021224600F011F9C719BF
:10824000714110340E46402CECDB3846029A00F0A7
:1082500007F9009A019B80180090594102980191FA
:10826000103002904028CCDB00980BB0F0BD0346E4
:108270000B439B0703D009E008C9121F08C0042A5A
:10828000FAD203E00B780370401C491C521EF9D24D
:108290007047D2B201E00270401C491EFBD2704709
:1082A0000022F6E710B513460A4604461946FFF7C2
:1082B000F0FF204610BD30B504460020034600E024
:1082C0005B1C934203D2E05CCD5C401BF8D030BD18
:1082D0000321001D401E037812021A43491EF9D5DE
:1082E00010467047034603220870000A491C521EBC
:1082F000FAD518467047024670B54A40D30FDB07DF
:1083000040002DD04A002AD0010E140E00021202A5
:108310000919400A520A8418E50104465443000A28
:10832000120A2E045043A4194219200CC543AA185E
:10833000120C0125AD03521C521912047F3924047A
:1083400000D0521C104301D44000491EC2B20C069A
:10835000C0092018401C4008802A02D003E00020F9
:1083600070BD40084000002900DA0020184370BDAD
:1083700070B502464A40D50F40004A00ED0740085C
:108380005208002814D0002A12D0C40DD30D410287
:108390000120C0055202490A520AE41A09181218AB
:1083A0007D34914201D3641C00E04900002C01DAC5
:1083B000002070BD0023914201D3891A0343400875
:1083C00049000028F7D100290AD0914202D10121A9
:1083D000C90705E0914201D2012101E00121C94311
:1083E000E005C018401900F05CF870BD10B500221F
:1083F0009623114600F05DF810BDC20FD207400071
:1084000040080BD0C10D0723DB01C9184002090544
:10841000400A1143C208400711437047002001463B
:108420007047000010B5002904DB0124E407404236
:108430008C412146002B04DB1C460123DB07524202
:10844000A341994200D1904210BD00000122D20701
:10845000002800DB101A002900DB511A88427047FF
:1084600010B5202A04DB0146203A9140002010BDBF
:10847000914020239C1A0346E3401943904010BDCD
:1084800010B5202A04DB0846203AD040002110BD58
:108490000B46D340D0402024A21A914008431946ED
:1084A00010BD002904DA401C490001D140084000F9
:1084B000704770B40024050C05D11024000402D1CB
:1084C000002921D01124050E01D100020834050F26
:1084D00001D10001241D850F01D18000A41C0028BA
:1084E00001DB4000641C002908D020252E1B0D460E
:1084F000F540A14000D001212943084301061B1B80
:10850000000ADB1D02D5002070BC7047DB0518187F
:1085100080180029F8DA401C4900F5D170BC4008E9
:1085200040007047064C0125064E05E0E36807CC85
:108530002B430C3C98471034B442F7D3FFF7C6FDE9
:10854000C8F90100E8F9010070B58C180578401CE5
:108550006B075B0F01D10378401C2A1106D102780A
:10856000401C03E006780E70401C491C5B1EF9D1CC
:108570002B0705D40023521E0DD40B70491CFAE7BB
:108580000378401CCB1A921C03E01D780D70491C27
:108590005B1C521EF9D5A142D8D3002070BD70B526
:1085A00007F010F80524204615F0D0FF00252846D6
:1085B00006F0FCFF204615F0C9FF0126304606F004
:1085C000D1FF204615F0C2FF284606F0CBFF20461B
:1085D00015F0BCFF304606F0E9FF204615F0B6FF67
:1085E00070BDB0B506F0EEFF0524204615F0AEFFD5
:1085F0000125284606F0DAFF204615F0A7FF284699
:1086000006F0B0FF204615F0A1FF002006F0AAFFFB
:10861000204615F09BFFB0BDF0B581B006F0BEFF5F
:10862000052015F093FF08270026012006F09AFF89
:108630000524204615F08AFF204615F087FF06F036
:10864000A3FF0546204615F081FF002006F08AFFB3
:10865000204615F07BFF76002E437F1E3806E4D1BE
:10866000F0B201B0F0BD70B50446002006F07AFF0C
:1086700006F0A8FF052015F069FF0826E0B2C00942
:1086800006F094FF0525284615F060FF012006F04E
:1086900069FF284615F05AFF002006F063FF2846C0
:1086A00015F054FF284615F051FF6400761E300681
:1086B000E4D1052015F04AFF012070BDF0B583B06C
:1086C000019314460E4607460120384302900325C5
:1086D00004E000F08EF86D1E280631D000F067F837
:1086E0003846FFF7C0FF00F0A7F80028F1D1304668
:1086F000FFF7B9FF00F0A0F80028EAD100F057F822
:108700000298FFF7B0FF00F097F80028E1D1019838
:1087100002280BD3451E0026FFF77EFF2070FFF7CF
:108720003EFF641C761CF0B28542F5DCFFF774FF57
:108730002070FFF756FF00F05CF8202003B0F0BD7A
:10874000102003B0F0BDF0B583B01C46009201913B
:108750000290032504E000F04CF86D1E280623D09B
:1087600000F025F80298FFF77EFF00F065F800287A
:10877000F1D10198FFF777FF00F05EF80028EAD109
:10878000002C0CD00026009F3878FFF76CFF00F01B
:1087900053F80028DFD1761C7F1CA642F4D300F0EA
:1087A00028F8082003B0F0BD102003B0F0BDB0B52C
:1087B00006F008FF0524204615F0C8FE01252846CE
:1087C00006F0D0FE204615F0C1FE284606F0EEFE6B
:1087D000204615F0BBFE0025284606F0E7FE2046A1
:1087E00015F0B4FE284606F0BDFE642015F0AEFE7E
:1087F000B0BDB0B506F0E6FE0524204615F0A6FE95
:108800000025284606F0AEFE204615F09FFE2846BD
:1088100006F0CCFE204615F099FE0125284606F00C
:10882000A1FE204615F092FE284606F0BFFE642009
:1088300015F08CFEB0BD0000B0B506F0AFFE05240B
:10884000204615F083FE012006F08CFE204615F030
:108850007DFE0B4D06F098FE044606F07DFE002CD2
:1088600002D06D1E2804F5D10525284615F06EFEB0
:10887000002006F077FE284615F068FE2046B0BDC1
:1088800033210000034801780B2901D8491C0170ED
:108890007047C0462F2C002070B584B0002503958A
:1088A00002950195009506F057FE0F20C6430E4C29
:1088B0001036F1B2A0206A461023FFF744FF20468D
:1088C00015F044FE204615F041FE912EF0D3A02075
:1088D000B0216A461023FFF736FF204615F036FE1A
:1088E0000248058004B070BD581B0000222C0020F7
:1088F00070B5022902D2EB24E0B270BD891EEB25CF
:108900000022134605E0401C5B1CDDB2A94225464F
:108910000EDB04786C40154604E034466E1C072DCF
:108920003546F0D26608E407F7D09A246640F4E7AB
:10893000E0B270BDF0B591B00C91417810AA117001
:1089400083781B025918C37804792402E3181B04A6
:1089500059180B0ED3700C0C94700D0A55700B91B6
:1089600008956918099409190A93C9180278D2431D
:108970008918427983791B029A18C379047A2402F0
:10898000E3181B049A188918130A0693C918130CC4
:108990000593C9180792120E04928918827AC37A35
:1089A0001B029A18037B0F90447B2402E3181B04DC
:1089B00098180918020A02928918020C0192891863
:1089C0000D910390000E0E9000200346014606E034
:1089D00032409A40D2B211435B1C082B0ED00126C4
:1089E00035469D400746024602E07F1C042FEFD02B
:1089F00010ACE45D2542F8D0521CF6E70E9C0D98B1
:108A00000019C3B20F98827B934205D0427A9142FB
:108A100002D1002011B0F0BD1021FFF769FF0C99C1
:108A2000CC72019A8A72029A4A72039A0A72049A62
:108A3000CA71059A8A71069A4A71079A0A710A9A46
:108A4000CA70099A8A70089A4A700B9A0A7011B013
:108A5000F0BDF0B58DB055220270002747720B783B
:108A60004370CA79059202728A790492C2714A7976
:108A7000039282710A7902924271CA7A0892427311
:108A80008A7A019202734E7AC6720C7A84720CAAA8
:108A900013704D782D02EB188D78C97809024919A9
:108AA0000904CB18190E01711D0CC57009931B0A1E
:108AB0000B90837038460A91D17007959570069394
:108AC000537031020919089A1202019BD21812043C
:108AD0005118089103990902029A8918059A1202FD
:108AE000049BD2181204511805913D463A4605E000
:108AF0002640AE4032436D1C082D0ED00124214685
:108B0000A9400346064602E05B1C042BF0D00CAFE4
:108B1000FF5C3942F8D0761CF6E70B9B5A72099835
:108B200006994018079940180A994018059A801824
:108B3000110A4018110C4018110E4018089A80189C
:108B4000110A4018110C4018110E4018563898732D
:108B500010211846FFF7CCFE0DB0F0BDF0B58FB078
:108B60000446FF20E070A07060700F20C0430290A8
:108B70000F302070704815F0E9FC704908686328D0
:108B800001D8642008606E4F002038806D4E01903F
:108B9000308008E00B99814222D338881030388029
:108BA00080B2A1286DD206F0D7FC3978A02003AAA4
:108BB0001023FFF783FD30802028EED103AD0BA9F1
:108BC0002846FFF7B7FEE97B8842E6D1287855288A
:108BD000E3D15D48017800290298DBD10846D9E746
:108BE0003888A0284DD8C0B20021019105E006F0D8
:108BF000B3FC3988C8B2A12943D2C1B2A02003AACC
:108C00001023FFF75BFD3080398810313980202830
:108C100037D103AD07A92846FFF78CFEE97B8842D0
:108C2000E5D128785528E2D14748007800280299F4
:108C300000D1014607988842D9D240490A68962156
:108C400051430B9A824208D90818904219D30BA9B4
:108C50000E222046FFF70BFBC9E78918814210D38B
:108C600007A90E222046FFF702FB0BA80A99818173
:108C700007980B9008980C9009980D9038880190EF
:108C8000B5E72078617809020818A178E278120225
:108C9000511809040818401C24D100200190388084
:108CA000A020B02103AA1023FFF708FD3080202860
:108CB00018D103AD0BA92846FFF73CFEE97B88429B
:108CC00010D1287855280DD11F480078002800D1F0
:108CD00002900B980299884204D20BA90E222046DA
:108CE000FFF7C5FA2078617809020818A178E278C0
:108CF0001202511809040818401C0CD10020E0721F
:108D0000A07260722072E071A07160712071E070D9
:108D1000A070607020700198388020786178090216
:108D20000818A178E27812025118090408180749B6
:108D3000086030880FB0F0BD701101001C2C0020BD
:108D4000222C0020182C00201B2C0020282C002076
:108D5000F0B581B000910646214800250570002A33
:108D60002ED01446C036631B71190F200840102204
:108D7000101A834200D303461A480278102A01D001
:108D8000042A1AD1C809FE2707405F2F13D80127EC
:108D9000B8436038C0B29E3282420CD3009A521956
:108DA000C9B2DFB23B46FFF789FC0F490880ED19D5
:108DB000A542D8D304E0082000E004200A49088036
:108DC000094801880020042902D0082900D0012088
:108DD00003490870411E8841400001B0F0BDC04603
:108DE0002E2C00201A2C00202C2C00200A4A0123B3
:108DF00013700A4A10700A4A11600A4A0021116071
:108E0000042801D105218901102801D11D208101EB
:108E1000054801807047C0461B2C00201A2C0020FA
:108E20001C2C0020282C0020202C0020F0B587B01E
:108E3000994D00262E80994B1B688B4224D1994C6A
:108E40002188202925D1029000920196964C002776
:108E50002760964D964E2878062809D806F07CFBA8
:108E60002068401C2060B042F5D38D480421018069
:108E70002F70904C20880107029B31D08848202118
:108E80000180854D019E0BE001204002844908804D
:108E900006E003A8FFF762FE208081488021018060
:108EA0007F4800883F2807DD874988420BDC40283F
:108EB00012D0802810D010E004280DD008280AD045
:108EC000202809D009E001214A02904204D0C902B9
:108ED000884201D001E002262E80288807B0F0BD2C
:108EE000A128019E00D32780009A012A6A4D1ED135
:108EF000187B012856D1DF719F715F711F711F733D
:108F0000587B012804D1DF729F725F721F725F73FA
:108F100003AF38461946FFF79CFDF87320880028F8
:108F200046D01038C1B2A02003AA102344E0002A82
:108F3000B6D1614801780029B2D00270187859780A
:108F4000090208189978DA781202511809040818E9
:108F50005A490978002901D00F21C943884233D2E8
:108F6000274603AC20461946FFF773FDE0733978B6
:108F7000A02010232246FFF7E6FB029A484908800A
:108F800008288DD13888103038801078517809023F
:108F900008189178D2781202511809040818484923
:108FA00008607DE7597B012911D10128A3D0A7E7EB
:108FB000A02003AA10230146FFF7C5FB384908800B
:108FC0003D48009901706BE70120C0025EE73D4813
:108FD0000078012812D103AC20461946FFF739FD6D
:108FE000E073A020B02110232246FFF7ACFB2C49F0
:108FF00008800828E4D133480770E1E718785978E9
:10900000090208189978DA78120251180904081828
:109010002B490968214A12685118884203D2204816
:1090200040210180CCE725490978002901D00F2192
:10903000C94388422DD203AF384619461C46FFF774
:1090400008FDF8731B480178A02010233A46FFF76B
:109050007AFB134908800828B2D1164908881030D5
:1090600008802078617809020818A178E278120255
:109070005118090408181249086008490A6815219E
:109080005143FFF75DF800299AD101200D4908707E
:1090900096E70120C00291E7342C00201C2C002010
:1090A000322C0020182C0020382C00202F2C0020DF
:1090B000818D5B00222C0020242C00201B2C002002
:1090C000282C0020302C0020FF010000F0B585B0D6
:1090D0000646434C0027278004921018414A128804
:1090E000904241D201910397404F00200290386096
:1090F0003F4C404D2078052809D806F02DFA3868F5
:10910000401C3860A842F5D33748042101800298FA
:1091100020703948018839480278102A01D0042A81
:1091200032D188190346C033049C651A0F240440C9
:109130001020001B854200DB0546DC09603C01264F
:109140003002E7B27F09052F12D3B443E6B29E3254
:10915000B242234C039F0DD301984218D9B2EBB20F
:109160003046FFF7F0FA05E01F482021018011E0AA
:109170001B4C039F1C49088008280BD1E8B21E4AEB
:1091800011880818108005E0012080021649088027
:10919000134C039F144800881F2809DD202813D092
:1091A00001210A0290420FD0890288420CD00CE0C3
:1091B000042809D0082808D10F480088049988425B
:1091C00001D3022700E001272780208802210143E4
:1091D000022902D1084900220A8005B0F0BDC0462C
:1091E000342C0020202C0020322C0020382C002091
:1091F0002F2C0020818D5B003C2C00201A2C00209D
:10920000F0B585B0044600200190042C6FD20BF01D
:109210009BFC002801D10BF017FD0020009000BF3F
:109220000098401C00900BF08FFC039003980028DE
:1092300003D0484900988842F2D30398002856D1B9
:10924000042145480BF062FC44484549088021014F
:10925000444A515C4900404A505A41490A88012118
:10926000090300F055F902900120049020013D49C6
:1092700040184078002801D100264BE020013949F0
:1092800040184078012802D13548068842E0200184
:1092900034494018407802282AD120014018057925
:1092A0002901304A515C49002B4A505A2C490A88FE
:1092B0000121090300F02CF9064628012A49431828
:1092C0002801284940180289280140180021C76850
:1092D0003046B84706462801224BC018C2882801EC
:1092E000C0188178304600F087F8064612E02DE07D
:1092F00020011C4940184078032804D02001401860
:109300004078132804D1200116494018868801E0CE
:10931000002004900498002818D020011249431816
:109320002001104940180289200140183146C768C1
:109330000298B847019020010A4BC018C28820014A
:10934000C0188178019800F057F80190019805B095
:10935000F0BD000050C3000002010020881300008F
:10936000FC00002068F00100A8F00100F8B50546F7
:109370000E4614460020009001211C4801751C482F
:10938000007888431A490870084680780821084305
:109390001749887000208871084600780121084329
:1093A0001349087008460572002717E01048007836
:1093B000802108430E49087000BF0E48007D002838
:1093C000FBD000200B4908750948C0892080A41CE7
:1093D0000748C1890098081800907F1CB742E5D360
:1093E00031460098FEF7ACFE80B2F8BD4061004007
:1093F000005004404060004010B50346012908D1E8
:10940000094CA41A9C4202D99C18A0B20BE0064851
:1094100009E0022906D1934202DD9C1AA0B202E0C3
:10942000002000E0184610BDFFFF000010B5044604
:109430000121202001F0F2FF0020324908700121B3
:1094400031480175002031490875152014F066FD7A
:109450002C488078E17808432A498870084680784B
:1094600021780843274988702078802806D108464B
:109470000079E17949000843224908712148807840
:10948000E17A08431F498870A078002803D1084674
:10949000007908710FE0A078012806D119480079F9
:1094A000602108431749087105E0164800798021BA
:1094B00008431449087113488079217908431149F8
:1094C000887108468079617908430E498871207A4D
:1094D000C872607A88720846007838218843094942
:1094E0000870084600786178C9000843054908708B
:1094F000A07A0873084600780121084301490870E2
:1095000010BD000000500440406100404060004039
:10951000F8B504460E461746002E01D100250FE08F
:10952000A64201DC3D460BE00094009C20467843B7
:10953000009031460098FEF703FE0090009885B237
:109540002846F8BD0146042904D28A00024BD218ED
:10955000508800E00020704748250020014604297B
:1095600003D28A00024B985C00E0002070470000A4
:1095700048250020FFB587B004460898844203DAE6
:109580000A988068002802D12448019042E0089897
:10959000001B82B20292002625460A9880680021AC
:1095A0002F463A463346049605910690FEF722FE72
:1095B00005460E46002328463146029AFEF7EAFD8C
:1095C00005460E46304600210A46494050400143B8
:1095D00002D0124801901DE003950A98C068039DCF
:1095E000A84202D30020019014E00A98C1680398B1
:1095F000401A039009990398FEF7A2FD039003987F
:10960000000C0004002802D00448019002E00398F6
:1096100080B2019001980BB0F0BD0000FFFF000088
:1096200010B5084800788021884306490870012158
:1096300005480175002005490875152014F06EFCD9
:1096400010BD0000005004404061004040600040F8
:10965000F8B505460E4614461F4621462846FEF735
:1096600085FD80B2F8BD0000FFB587B006460A98B8
:109670004068002801D1029035E00A9801684068EE
:1096800008180390002534460021274603980695C4
:109690000491059038462946049B059AFEF7AAFDD9
:1096A00004460D460A984068024600230190204671
:1096B0002946FEF76FFD04460D4600232046294645
:1096C000099AFEF767FD04460D46284607492140E2
:1096D000002359405840014303D00448C04302903E
:1096E00001E0A0B2029002980BB0F0BD0000FFFFB5
:1096F00010B5FE4800688079030014F0F5FB0705FB
:109700009ED8F5F4F3F2F100F848006840790300C0
:1097100014F0EAFB0805138A2A8A468A638A10F045
:1097200091FC0020F1490968C873F048006840794D
:10973000401CEE49096848717DE0ED494969EB4AF2
:109740001268D27A885C10F0F5FCE848006840792D
:10975000401CE64909684871E44800684079401CAB
:10976000E2490968487166E009F050FD002810D10F
:1097700010F0E0FCDD4800684079401CDB490968D6
:109780004871DA4800684079401CD8490968487136
:1097900005E010F081FC0020D449096848714AE0D6
:1097A00009F034FD002811D1112010F0C3FCCF487E
:1097B00000684079401CCD4909684871CB48006871
:1097C0004079401CC9490968487105E010F064FC03
:1097D0000020C649096848712DE009F017FD0028EE
:1097E0001BD1C2480068C07A401CC0490968C872D1
:1097F000BE480068C07ABE49097888420DDB002067
:10980000BA490968C872B94909684862B748006826
:109810008079401CB5490968887110F03DFC002032
:10982000B2490968487106E010F036FC0020AF49E3
:109830000968487100BF00BF32E3AC480068407C53
:10984000002817D0AA48C068002803D0A848C168DB
:10985000192088470020A54909684862A348006884
:109860008079401CA1490968887100209F490968D6
:1098700048711BE09D480068406A282807D29B4831
:109880000068406A401C9949096848620EE000205F
:10989000964909684862954800688079401C934958
:1098A000096888710020914909684871F8E28F4879
:1098B00000684079030014F017FB080518A42FA4D2
:1098C0004CA480A410F0BEFB002088490968C8732E
:1098D000864800684079401C84490968487197E0CF
:1098E000D4E2C7E230E25DE194E0814949697F4A10
:1098F0001268D27A885C10F01DFC7C4800684079C0
:10990000401C7A4909684871784800684079401CD1
:109910007649096848717BE009F078FC002811D18C
:10992000012010F007FC714800684079401C6F4925
:10993000096848716D4800684079401C6B490968A6
:10994000487105E010F0A8FB0020684909684871DB
:109950005EE009F05BFC002828D164490968C97AF7
:1099600024225143634A12688918604A1268D27BE4
:10997000885C10F0DFFB5D480068C07B401C5B49E1
:109980000968C87359480068C07B242814D3574815
:1099900000684079401C554909684871534800687F
:1099A0004079401C51490968487105E010F074FB8A
:1099B00000204E49096848712AE009F027FC002878
:1099C00018D14A480068C07A401C48490968C872E2
:1099D00046480068C07A4649097888420ADB002078
:1099E00042490968C872414800688079401C3F4973
:1099F0000968887110F050FB00203C4909684871E3
:109A000006E010F049FB002038490968487100BFA2
:109A100000BF45E2354800684079030014F064FA5D
:109A20000A0614B92BB948B978B995B910F00AFBF0
:109A300000202E490968C8732C4800684079401CF2
:109A40002A4909684871ABE029494969274A1268DF
:109A5000D27A885C10F06EFB244800684079401C84
:109A6000224909684871214800684079401C1F4913
:109A70000968487194E009F0C9FB002811D14A2017
:109A800010F058FB194800684079401C17490968D4
:109A90004871164800684079401C144909684871AB
:109AA00005E010F0F9FA002010490968487177E0E4
:109AB00009F0ACFB002824D1FF2010F03BFB0B4841
:109AC0000068C07B401C09490968C87307480068E2
:109AD000C07B24281BD3054800684079401C0349FB
:109AE0000968487101480068407905E0C80700200E
:109AF000002C0020C4070020401CEA490968487176
:109B000005E010F0C9FA0020E6490968487147E00D
:109B100009F07CFB002811D1FF2010F00BFBE1487D
:109B200000684079401CDF4909684871DD480068D9
:109B30004079401CDB490968487105E010F0ACFA37
:109B40000020D849096848712AE009F05FFB002825
:109B500018D1D4480068C07A401CD2490968C8723C
:109B6000D0480068C07AD049097888420ADB0020D2
:109B7000CC490968C872CB4800688079401CC94943
:109B80000968887110F088FA0020C6490968487190
:109B900006E010F081FA0020C2490968487100BF50
:109BA00000BF7DE1BF4800684079030014F09CF9D4
:109BB0000C0715C32CC349C366C382C39FC310F0EF
:109BC00041FA0020B7490968C873B648006840796F
:109BD000401CB44909684871B4E0B3494969B14AC5
:109BE0001268D27A885C10F0A5FAAE480068407915
:109BF000401CAC4909684871AA4800684079401C7B
:109C0000A849096848719DE009F000FB002811D1BE
:109C1000772010F08FFAA34800684079401CA149D2
:109C2000096848719F4800684079401C9D4909684F
:109C3000487105E010F030FA00209A49096848712F
:109C400080E009F0E3FA002811D10C2010F072FA3C
:109C5000944800684079401C9249096848719148CD
:109C600000684079401C8F490968487105E010F090
:109C700013FA00208B490968487163E009F0C6FABD
:109C8000002810D110F056FA864800684079401C30
:109C9000844909684871834800684079401C8149BB
:109CA0000968487105E010F0F7F900207D4909685E
:109CB000487147E009F0AAFA002811D1132010F0EA
:109CC00039FA784800684079401C7649096848713B
:109CD000744800684079401C72490968487105E081
:109CE00010F0DAF900206F49096848712AE009F09C
:109CF0008DFA002818D16B480068C07A401C694969
:109D00000968C87267480068C07A6749097888425C
:109D10000ADB002063490968C872624800688079DC
:109D2000401C60490968887110F0B6F900205D494F
:109D30000968487106E010F0AFF900205949096838
:109D4000487100BF00BFABE056480068407903008F
:109D500014F0CAF8080513872A874787638710F02D
:109D600071F900204F490968C8734E48006840796E
:109D7000401C4C49096848717AE04B494969494A95
:109D80001268D27A885C10F0D5F9464800684079AC
:109D9000401C444909684871424800684079401CA9
:109DA00040490968487163E009F030FA002811D190
:109DB000492010F0BFF93B4800684079401C394900
:109DC00009684871374800684079401C354909687E
:109DD000487105E010F060F90020324909684871C7
:109DE00046E009F013FA002810D110F0A3F92D482D
:109DF00000684079401C2B4909684871294800686F
:109E00004079401C27490968487105E010F044F981
:109E100000202449096848712AE009F0F7F9002870
:109E200018D120480068C07A401C1E490968C872D1
:109E30001C480068C07A1C49097888420ADB002067
:109E400018490968C872174800688079401C15498C
:109E50000968887110F020F90020124909684871DA
:109E600006E010F019F900200E490968487100BF9A
:109E700000BF15E000200B4909688871094909688D
:109E80004871062007490968C87009E010F004F914
:109E9000002004490968487102490968887100BFB7
:109EA00000BF10BDC8070020002C002010B56A4874
:109EB00000684079030014F017F8090610C627C699
:109EC00044C6608EC60010F0BDF863480068407953
:109ED000401C614909684871BCE0604949695E4AB3
:109EE0001268D27A885C10F025F95B4800684079E6
:109EF000401C594909684871574800684079401C1E
:109F0000554909684871A5E009F080F9002811D188
:109F10007F2010F00FF9504800684079401C4E49EE
:109F2000096848714C4800684079401C4A490968F2
:109F3000487105E010F0B0F8002047490968487101
:109F400088E009F063F9002810D110F0F3F84248D6
:109F500000684079401C4049096848713E480068E3
:109F60004079401C3C490968487105E010F094F8BC
:109F700000203949096848716CE009F047F9002868
:109F800022D135480068C07A401C33490968C8723C
:109F900031480068C07A3149097888420FDB0020D7
:109FA0002D490968C8722C4800684079401C2A492C
:109FB00009684871002028490968486208E00020C3
:109FC00025490968487103E0002023490968487160
:109FD00010F062F83EE020480068407C002816D06F
:109FE0001E48C068002803D01C48C1681920884753
:109FF00000201949096848621749096848711649DB
:10A0000009688871052014490968C8701AE0124867
:10A010000068406A282807D20F480068406A401C40
:10A020000D49096848620DE000200B490968486243
:10A030000949096848710849096888710520064975
:10A040000968C87006E010F027F800200249096886
:10A05000487100BF00BF10BDC8070020002C0020C1
:10A0600010B50024F7480068807A01287ED1F548B1
:10A070000068C07900287AD0F2480068807900280A
:10A0800004D0012874D0022873D191E1ED48006812
:10A09000007B24286ED2EB480068C07901287AD171
:10A0A000002475E0E7480068C07A24214843E64967
:10A0B00009684018E3490968097B415CE148006888
:10A0C000C07A24225043E14A12688018DD4A12689F
:10A0D000127B805C814229D0DA480068C07A242152
:10A0E0004843DA4909684018D6490968097B415C48
:10A0F000D4480068C07A24225043D34A126880189A
:10A10000D04A1268127B8154CE480068407B2428D4
:10A1100005D3CC480068007BCA4909684873C94820
:10A120000068007BC7490968887308E0C548006873
:10A13000407B242803D20120C24909688871C148A4
:10A140000068007B401CBF4909680873BD4800686F
:10A15000007B242808D3BB480068407B242803D216
:10A160000120B84909688871B64805E0D3E1CDE11E
:10A1700069E0BAE138E00EE00068007B242804D2F0
:10A18000B04800688079012800D103E0601CC4B2A7
:10A19000242C87D356E0002413E0AA480068C07A34
:10A1A00024214843A94909684018015DA548006871
:10A1B000C07A24225043A44A126880180155601CBA
:10A1C000C4B2242CE9D300209E4909684873232097
:10A1D0009C490968887301209A490968887124207C
:10A1E0009849096808732DE00020964909680873AA
:10A1F00094480068C07A401C92490968C872914826
:10A200000068C07A92490978884217DB8D48006857
:10A21000007C012804D102208A490968887106E07F
:10A22000002088490968887186490968C87100203A
:10A2300084490968C8728349096808740020814903
:10A240000968487161E17F4800684079030013F0B4
:10A250004BFE080513A62AA651A68EA60120794911
:10A26000096808740FF0EEFE764800684079401CDB
:10A2700074490968487199E075494969714A1268D9
:10A28000D27A885C0FF056FF6E4800684079401C17
:10A290006C49096848716B4800684079401C6949FD
:10A2A0000968487182E008F0B1FF00281BD16549B8
:10A2B0000968497B491CC8B20FF03CFF614800683F
:10A2C000407B60490968C8735E4800684079401C5B
:10A2D0005C49096848715B4800684079401C5949ED
:10A2E0000968487105E00FF0D7FE0020554909685C
:10A2F00048715BE008F08AFF00282BD151490968BA
:10A30000C97A24225143504A126889184D4A12686A
:10A31000D27B885C0FF00EFF4A480068C07B401C6F
:10A3200048490968C87347480068C07B45490968BF
:10A33000897B88421ADD434800684079401C4149C6
:10A34000096848713F4800684079401C3D490968E8
:10A3500048710BE00FF0A0FE3A480068407B394995
:10A360000968C87300203749096848711EE008F081
:10A370004DFF00280CD133490968887124203149E8
:10A380000968C8732F49096848732E49096888739A
:10A390000FF082FE00202B490968487106E00FF09B
:10A3A0007BFE002027490968487100BF00BFACE070
:10A3B000244800684079030013F096FD08050F8ECD
:10A3C000268E4C8E688E0FF03DFE1E480068407948
:10A3D000401C1C490968487185E01D494969194AB2
:10A3E0001268D27A885C0FF0A5FE164800684079A2
:10A3F000401C144909684871124800684079401CA3
:10A400001049096848716EE008F000FF002811D17A
:10A4100049200FF08FFE0B4800684079401C094925
:10A4200009684871074800684079401C0549096877
:10A43000487105E00FF030FE0020024909684871BC
:10A4400051E00000C8070020C4070020C00700201A
:10A45000002C002008F0DAFE002810D10FF06AFE70
:10A460009C4800684079401C9A490968487199489D
:10A4700000684079401C97490968487105E00FF071
:10A480000BFE00209349096848712CE008F0BEFEDD
:10A4900000281AD18F480068C07A401C8D4909688D
:10A4A000C8728C480068C07A8B49097888420CDBF6
:10A4B000002088490968C8728649096888718549F9
:10A4C0000968487183490968C8710FF0E5FD0020EB
:10A4D00080490968487106E00FF0DEFD00207D49E3
:10A4E0000968487100BF00BF0FE00FF0D5FD0020E4
:10A4F0007849096848717749096888717549096818
:10A50000087374490968C87200BFE2E0002071490D
:10A5100009688872DDE06F480068807A0228F4D10B
:10A520006C480068007A002879D06A480068407951
:10A53000030013F0D9FC0B0711BB25BB41545EBBD4
:10A540007590BB000FF07EFD624800684079401CAA
:10A55000604909684871B7E05F49496908780FF0B8
:10A56000E9FD5C4800684079401C5A490968487117
:10A57000584800684079401C564909684871A3E072
:10A5800008F044FE002810D10FF0D4FD51480068B7
:10A590004079401C4F49096848714E48006840792D
:10A5A000401C4C490968487105E00FF075FD00201A
:10A5B00048490968487187E008F028FE002807D15B
:10A5C000444800684079401C42490968487103E0EA
:10A5D00000204049096848710FF05EFD74E00FF0FB
:10A5E00031FD3C4800684079401C3A49096848718F
:10A5F0006AE0394949690978491CC8B20FF09AFDE7
:10A60000344800684079401C324909684871314833
:10A6100000684079401C2F490968487154E054E0B3
:10A6200008F0F4FD00280FD10FF0DEFC294909687D
:10A63000887001200FF052FD264800684079401CC8
:10A6400024490968487105E00FF026FD00202149E2
:10A650000968487138E01F480068807811280CD1DB
:10A6600000201C4909680872AA201A4909688870E4
:10A67000002018490968487011E0164800684078C1
:10A68000401C144909684870124800684078032843
:10A6900005D308F05BFE00200E49096848700FF0F2
:10A6A000FBFC00200B49096848710DE00FF0F4FC39
:10A6B0000020084909684871064909684870AA20BD
:10A6C00004490968887000BF03E000200149096857
:10A6D000887210BDC8070020002C002010B502466B
:10A6E0009000074BC018405C002802D00320C043F4
:10A6F00010BD01209300024C1B1958540020F7E7AD
:10A700008427002070B5002508E06D1C1B48854299
:10A7100002D20AF0C5FA01E0002503E00AF014FABB
:10A720000028F2D100BF022100200AF01BFA032109
:10A7300000200AF017FA052100200AF013FA072179
:10A7400000200AF00FFA002408E00020A1000C4AC3
:10A750005054A10089184880601CC4B2042CF4D362
:10A7600001200849087000204870052088700020EA
:10A77000C87005480549088070BD000050C300003E
:10A7800048250020FE00002088130000FC00002067
:10A79000F8B58D480078030013F0A6FB06040516F3
:10A7A0003D5EFDFC0EE10AF04FFA00208649C870BC
:10A7B000487008468078002802D10320087002E023
:10A7C000022081490870FDE07F488078002804D08D
:10A7D0007D488078401E7C4988700AF0B5F90028D1
:10A7E0000BD10AF031FA00207749C870084680780A
:10A7F00000280FD1032008700CE07348C078401C7B
:10A800007149C8700846C078052803D30520087030
:10A810000AF046FAD6E00AF097F900280ED1042192
:10A820006A480AF073F900206749C87048706848A0
:10A83000684908800420644908700CE06248C078C8
:10A84000401C6149C8700846C078052803D305201C
:10A8500008700AF025FAB5E05B49497809015E4ABB
:10A86000515C4900594A505A5A490A880121090342
:10A87000FEF74EFE009001255348407800015649EE
:10A8800040184078002801D100243CE04E48407830
:10A890000001514940184078012802D14D480488F0
:10A8A00031E04948407800014B494018407802287F
:10A8B00012D1454949780901474A89180879FEF7B4
:10A8C00041FE0446404949780901434A89180879FC
:10A8D000FEF744FE054616E03B48407800013E493D
:10A8E00040184078032806D03748407800014018C7
:10A8F0004078132806D13448407800013649401882
:10A90000848800E00025002D2FD02F4840780001DA
:10A91000324943182C48407800012F4940180289D9
:10A9200029484078000140182146C7680098B84778
:10A930000646254840780001274BC018C2882248A7
:10A9400040780001C01881783046FEF755FD064674
:10A950001D484078800022494018468001201A494D
:10A96000497889001E4A50540AE000201649497867
:10A9700089001B4A89184880134949788900505436
:10A9800011484078401C1049487008464078042817
:10A9900009D301E013E007E00AF056F900200A4964
:10A9A0004870032008700DE00AF0CEF8002803D1AB
:10A9B00001200549087001E00AF072F902E0FFF792
:10A9C000A1FE00BF00BFF8BDFE0000200201002074
:10A9D00088130000FC00002068F00100A8F00100CE
:10A9E0004825002010B50AF079F8002405E0002081
:10A9F000A100074A5054601CC4B2042CF7D30020B5
:10AA0000044908700520887003480449088010BD77
:10AA100048250020FE00002088130000FC000020D4
:10AA200070B50446002000F0AFF8002000F0DAF81E
:10AA3000002000F09BF8002000F0C4F8002000F097
:10AA400087F8002000F0AEF800BF012000F08EF87B
:10AA5000012000F0B7F8002521E0002000F086F882
:10AA6000002000F0AFF880202040002806D0012010
:10AA700000F08AF8012000F0B5F805E0002000F0B1
:10AA800083F8002000F0AEF800BF012000F06EF85F
:10AA9000012000F097F86006040E681CC5B2082D6E
:10AAA000DBDB012000F054F8012000F07BF870BDE2
:10AAB00070B504460D46012000F066F8012000F054
:10AAC00091F8002000F052F8002000F07BF8002000
:10AAD00000F03EF8002000F065F800BF012000F013
:10AAE00045F8012000F06EF8002628E0002000F074
:10AAF0003DF8002000F066F880202040002803D0B8
:10AB0000012000F041F802E0002000F03DF8802034
:10AB10002840002803D0012000F064F802E0002063
:10AB200000F060F800BF012000F020F8012000F0E4
:10AB300049F86006040E6806050E701CC6B2082EA1
:10AB4000D4DB012000F004F8012000F02BF870BDE8
:10AB500010B50446002C04D0812103200AF02EF900
:10AB600003E0802103200AF029F910BD10B5044646
:10AB7000002C04D0812104200AF020F903E0802178
:10AB800004200AF01BF910BD10B50446002C04D0B7
:10AB9000812102200AF012F903E0802102200AF04C
:10ABA0000DF910BD10B50446002C04D081210448D5
:10ABB0000AF004F903E0802101480AF0FFF810BD13
:10ABC0000107000010B50446002C05D081210720A4
:10ABD00000020AF0F3F804E08021072000020AF0E6
:10ABE000EDF810BD10B50446002C04D081210448B6
:10ABF0000AF0E4F803E0802101480AF0DFF810BD14
:10AC00000207000010B5F920FFF70AFF8820FFF7C0
:10AC100007FF9020FFF704FF9820FFF701FF0821AE
:10AC20000846FFF745FFE820FFF7FAFE1221084625
:10AC3000FFF73EFFA020FFF7F3FE70210846FFF765
:10AC400037FFA820FFF7ECFE70210846FFF730FF22
:10AC5000B020FFF7E5FE70210846FFF729FFB82076
:10AC6000FFF7DEFE00210846FFF722FFC020FFF7B6
:10AC7000D7FE00210846FFF71BFFC820FFF7D0FED4
:10AC800000210846FFF714FFD020FFF7C9FE2F214F
:10AC90000846FFF70DFFD820FFF7C2FE2F21084618
:10ACA000FFF706FFE020FFF7BBFE2F210846FFF766
:10ACB000FFFE4020FFF7B4FE00210846FFF7F8FE34
:10ACC0000A20FFF7ADFE002405E000210846FFF74B
:10ACD000EFFE601CC4B25A2CF7DB00240AE000200F
:10ACE0000B4908550B4908550B4908550B490855A0
:10ACF000601CC4B25A2CF2DB8120FFF791FE0020C9
:10AD0000074908708870C8700871487010BD00004D
:10AD10006C220020C6220020202300207A2300205D
:10AD2000CC00002010B58020FFF77AFE10BD000097
:10AD30000020044908700120034908700020487071
:10AD400070470000D1000020CC00002010B548481A
:10AD5000007800287AD046488078030013F0C4F8C1
:10AD60000604434A535A687E414800794149085CC9
:10AD70003F490979404A515C884209D13C480079F1
:10AD80003E49085C3A4909793D4A515C88421BD0EA
:10AD9000374800793749085C35490979364A5054B3
:10ADA000334800793549085C31490979344A5054AF
:10ADB0002F48C078002803D004202D49887011E066
:10ADC00001202B4988700DE000202949C8700846F1
:10ADD0000079401C0871084600795A2802DB0020DF
:10ADE0000871087041E04020FFF71AFE0220204958
:10ADF00088703AE01E4A11791079FFF759FE032056
:10AE00001B49887031E00A20FFF70AFE0420184928
:10AE100088702AE0164A1279194B995C144A127903
:10AE2000154B985CFFF744FE0520114988701CE023
:10AE30000F480079401C0E490871084600795A28CD
:10AE400005DB002008710870C87003E00EE00120E7
:10AE50000749C87000200649887006E000200449B0
:10AE600008708870C870087100BF00BF10BD000076
:10AE7000CC0000206C220020C622002020230020CD
:10AE80007A23002010B50FF017FD012837D10720D5
:10AE900008F038FF002810D01C480078052805DA93
:10AEA0001A480078401C1949087016E00520174917
:10AEB00008700020164908700FE015480078052832
:10AEC00005DA13480078401C1149087005E0052098
:10AED0000F49087000200D4908700C4800780528BB
:10AEE00006D1FF22A5320021012011F0D3F90BE099
:10AEF0004B22D2000021012011F0CCF904E0002205
:10AF00001146012011F0C6F910BD00001D000020FF
:10AF10001C000020002003490872487088704860B7
:10AF200070470000500D002058221152704710B594
:10AF300004460121022000F071FA0021022000F0F5
:10AF40006DFA10BD014600205322525C10231A40B6
:10AF5000002A08D05322525C0C231A409210032A74
:10AF600018D1032016E05422525A0123DB031A4061
:10AF7000002A0ED05322525C0C231A409210032A4E
:10AF800005D05322525C9207920F032A01D102206E
:10AF900000E0012070470246002058239B5A0B40D6
:10AFA000002B01D0012000E0002070470146002264
:10AFB0006020405AFF231B0218400005020F1001B9
:10AFC000014BC018704700000055044010B5002A1E
:10AFD0000AD056231B5A0C022343562423525623CD
:10AFE0001B5A8B43235209E056231B5A0C02A343DE
:10AFF0005624235256231B5A0B43235210BD0000E4
:10B00000F8B504460D46012700263448844203D192
:10B010000121022000F002FA2878401EA07020884A
:10B02000FF21013108432080208840084000208013
:10B03000A878401EC1B25A20015568790007000C5B
:10B04000E97909020843A97908435C210853288952
:10B0500081B240200153A868C000C10C42200153B6
:10B06000A88981B244200153E868C000C10C462081
:10B070000153288A81B2482001532869C000C10CBD
:10B080004A200153A88A81B24C2001536869C0004C
:10B09000C10C4E2001535020005B2979090208435E
:10B0A000502108535020005B2979884350210853D0
:10B0B00000E0761C5020005B4007400F2979884251
:10B0C00002D007488642F4D15020005B4007400F71
:10B0D0002979884200D000273846F8BD0054044042
:10B0E000FFFF000030B5034600201C898C4209DDBB
:10B0F000082A05D218244C431D682C19A05C02E0D4
:10B10000002000E0002030BD10B5024613898B42BC
:10B1100005DD18234B431468E318987C00E00020F9
:10B1200010BD0146FF22C889C007C00F00280AD001
:10B130000120C88100E0521EC889C007C00F002846
:10B1400001D0002AF7D1C889C007C00F00280FD14D
:10B150000220C8810420C881487A40084000487213
:10B16000487A38239843487200204872012070477B
:10B170000020FCE70246507A012318435072507AAF
:10B180000B78DB0018435072087A012808D18888B0
:10B1900050814868000C0123DB031843908108E0CC
:10B1A000087A002805D15081486880001A4B184061
:10B1B0009081487A012804D1507A40231843507274
:10B1C00006E0487A002803D1507A40239843507211
:10B1D0000878002811D1C87A1072087B1070487B5B
:10B1E0005070887B9070CB7BD370087C10714B7C47
:10B1F0005371887C9071CB7CD371887A002803D0FE
:10B200000120C002D08101E00820D081FF20013060
:10B21000D081012070470000FC1F0000002904D0ED
:10B22000427A80231A43427203E0427A80239A438F
:10B230004272704730B5024600200F4B5024A45A8A
:10B240000D022C435025AC525024A45A8C43AC52CE
:10B2500000E05B1E5024A45A6407640F8C4201D0A6
:10B26000002BF6D15024A45A6407640F002C01D09F
:10B27000002000E0012030BDFFFF0000827A802323
:10B280001A40802A00D081727047000070B50446D1
:10B2900000250023002D02D0012660200653042043
:10B2A000C88188890126F6033040002808D0012093
:10B2B00010728889C004C0084E893043506006E08F
:10B2C0000020107288890F4E304080105060087A3C
:10B2D000D072002304E0CE5C10460C30C6545B1CD8
:10B2E000D07A9842F7DCC88904263040002804D17F
:10B2F000C889F6023040002801D0002070BDD07A05
:10B30000FCE70000FC1F0000027C80231A40802A1A
:10B3100000D00174704710B50246FF23D089C007E2
:10B32000C00F00280AD00120D08100E05B1ED08928
:10B33000C007C00F002801D0002BF7D1D089C0076B
:10B34000C00F002801D0002010BD507A01242043F6
:10B350005072507A3824A0435072C87A1072487ADA
:10B3600000280FD1087B1070487B5070887B90704C
:10B37000CC7BD470087C10714C7C5471887C9071AB
:10B38000CC7CD471FF200130D0814000D081107A74
:10B39000DAE70000F8B504460D460020002C00D185
:10B3A00000BF002A00D100BF012C01D1412630434B
:10B3B000012A01D112263043022C01D1C02630438C
:10B3C000022A01D130263043134E30707678802720
:10B3D000BE43114F7E70012C08D1FF2100BF0E4EDD
:10B3E000B3781E460E4033468B42F8D10A4E76782B
:10B3F0004027BE43084F7E70012A0BD100260096DD
:10B4000003E000BF009E761C0096FF276937009E70
:10B41000BE42F6D9F8BD000000040240002905D064
:10B42000054A12780243044B1A7004E0024A12786B
:10B430008243014B1A70704720040240002905D056
:10B44000054A927E0243044B9A7604E0024A927EB9
:10B450008243014B9A76704700080240012006495A
:10B46000087000BF04480078802108400028F9D007
:10B470000120024908707047000C02409C01002026
:10B4800070B5034614460020002B01D1C0B202E083
:10B4900005468035E8B2012902D1051DE8B206E073
:10B4A000022903D105460835E8B200E0C0B2012CFC
:10B4B00002D1851CE8B200E0C0B2084DA870AD789A
:10B4C00001263543054EB570002201E000BF521C35
:10B4D0007D252D01AA42F9D970BD0000000C024063
:10B4E00070B500242448007920210840002801D0AC
:10B4F000224D3FE000F046F80546214800788021C3
:10B500000840002836D01E4880780840002801D026
:10B510001A4D02E000F036F8054619488078000719
:10B52000840F022C01DBAD0804E0012C01D16D0871
:10B5300000E000BF124880788007C00F002801D0CB
:10B540002D0101E00C2045430D4800784007840F91
:10B55000002C02D1601CC4B207E0032C03D1601C94
:10B560004006040E01E06006040E21462846FCF762
:10B57000E7FD0546284670BD0004024000127A002F
:10B58000000C024000B5C0229178F82211401C4AFC
:10B5900012781143EA2923D00ADC0A46E03A130064
:10B5A00012F0A2FC0A181C20242A2A2A2A161A2A77
:10B5B000ED291FD004DCEB2916D0EC291CD117E0B3
:10B5C000F02903D0F82917D10E4817E00E4815E0EE
:10B5D0000E4813E00E4811E00E480FE00E480DE053
:10B5E0000E480BE00E4809E00E4807E00E4805E063
:10B5F0000E4803E00E4801E00D4800BF00BF00BD4B
:10B60000201C02400090D003006CDC020048E801DE
:10B6100000366E010024F400001BB70000127A000F
:10B62000808D5B0000093D00C0C62D0080841E0097
:10B6300040420F0010B50446204600F083FD002074
:10B6400010BD000010B590211348FCF729FE1248E8
:10B65000124908601248486006200881002088725C
:10B6600006220F490D4800F04BFA00210B48FFF766
:10B6700005FE80210B48FCF713FE0A480A49486082
:10B680000A4B04220A49084800F0CBFB5521064822
:10B69000FFF73AFE10BD00004008002020080020FF
:10B6A000CCEC0100D00800202C08002035B60000AA
:10B6B0005CEC01000C4A127812060B4B5B781B0401
:10B6C0001A43094B9B781B021A43074BDB781A433A
:10B6D000104642084240D20083085A401146034AAD
:10B6E0005140034A11607047130700200102000017
:10B6F00018070020F8B504460F46A07A4006400E11
:10B70000002874D10025ACE018206843216808188F
:10B71000407C01283CD10121182068432268101880
:10B72000017400260CE018206843216808180830CE
:10B73000815D18206843226810188155701CC6B2BC
:10B74000082EF0D3002118206843226810180174D5
:10B750001820684322681018417418206843226832
:10B7600010184161182068432268101881742C2039
:10B77000684361680818406A002809D018236B43A1
:10B780002268D0182C236B436268D218516A88470C
:10B7900018206843216808184069FF21C94388427E
:10B7A0005DD818206843216808184069C11918201D
:10B7B00068432268101841611820684321680818FE
:10B7C00041692C206843626810188069814246D321
:10B7D0001820684321680818807C55283FD05521DF
:10B7E00018206843226810188174002624E03CE089
:10B7F0001820684321680818805D2C21694362681D
:10B8000051181031895D0840182169432268511888
:10B8100088551820684321680818805D2C216943E9
:10B82000626851180831895D08431821694322680C
:10B8300051188855701CC6B2082ED9D32C206843E5
:10B8400061680818806A002809D018236B432268B1
:10B85000D0182C236B436268D218916A8847681C01
:10B8600085B22089A84200DD4EE7F8BD10B5044638
:10B87000002012F09DFE022841D1214800780028C6
:10B8800002D101201E4908701D48007801281FD1EF
:10B890001B484078401C1A49487021465A20FCF742
:10B8A0004FFC17494978884229D80020144948702C
:10B8B00008468078401C8870084680780A2803D3A0
:10B8C0000020887002200870002012F0A1FE16E00F
:10B8D0000B480078022812D109484078401C0849DA
:10B8E000487021467D20C000FCF72AFC04494978B5
:10B8F000884204D800200249487012F089FE10BD29
:10B900007400002000B587B0002168460171042151
:10B9100041710C480290411003910B49049105912B
:10B920000A480690FFF78EFE01A812F0D5FE00F03F
:10B930002FFB00F00FF80021054809F0ABFA07B023
:10B9400000BD0000FFFF1F00FFFFFF1F89BB0000BD
:10B950000205000010B5FF20023065494860002054
:10B960000872012008700020487201208872614826
:10B97000FFF7D7FB5E495F48FFF7FCFB01215D48FD
:10B98000FFF74CFC5C485A494860002008720120CF
:10B990000870002048720120887256481030FFF766
:10B9A000C0FB534953481030FFF7E4FB01215148D5
:10B9B0001030FFF733FC5048401E4D4948600020CE
:10B9C00008720120087000204872012088724948DE
:10B9D0005030FFF7A6FB464946485030FFF7CAFBF8
:10B9E000012144485030FFF719FC4348C138404911
:10B9F0004860002008720120087000204872012071
:10BA000088723C484030FFF78CFB39493948403058
:10BA1000FFF7B0FB012137484030FFF7FFFBFF2065
:10BA2000123033494860002008720120087000205D
:10BA30004872012088722F486030FFF772FB2C4952
:10BA40002C486030FFF796FB01212A486030FFF751
:10BA5000E5FBFF20213026494860002008720120C4
:10BA6000087000204872012088722248A030FFF739
:10BA700058FB1F491F48A030FFF77CFB01211D48E0
:10BA8000A030FFF7CBFB3F20400119494860002060
:10BA90000872012008700020487201208872154841
:10BAA0002030FFF73EFB124912482030FFF762FBBF
:10BAB000012110482030FFF7B1FB10480C494860C5
:10BAC000002008720120087000204872012088724E
:10BAD00008483030FFF725FB054906483030FFF7AE
:10BAE00049FB012103483030FFF798FB10BD0000EF
:10BAF000802600201055044002040000DF070000EB
:10BB0000F0B50B46144643600481002136E0002264
:10BB100016E02C254D4346687519AD5C18274F4338
:10BB20000668F619B5542C254D4346687519AD5C69
:10BB300018274F430668F6190836B554551CEAB263
:10BB4000082AE6D3002518274F430668F6193574EE
:10BB500018274F430668F619757418274F4306686F
:10BB6000F619B57418274F430668F619F5741827A7
:10BB70004F430668F61975614D1CA9B205898D42BF
:10BB8000C5DC00258572F0BD70B50446606800F024
:10BB900031FE0546E27A23460C332946094800F077
:10BBA000F1FD09496068884203D0491C60688842F9
:10BBB00006D1E17AA28890B222460C3202F0DEFE73
:10BBC00070BD000020080020DF070000F8B5054622
:10BBD00000262C46002C07D000BF03E0FF20A05514
:10BBE000701CC6B2082EF9D304F0FCFDC000082179
:10BBF000084007462068884338432060F8BDF8B500
:10BC0000054600262C46002C07D000BF03E0FF208D
:10BC1000A055701CC6B2082EF9D304F033FE0712EB
:10BC20002088000A00023843208004F02BFE000226
:10BC3000FF210902084007462088884338432080B6
:10BC400004F0F4FE07126088000A000238436080A6
:10BC500004F0ECFE0002FF2109020840074660885C
:10BC6000884338436080F8BDFEB5054600260020B5
:10BC7000019001F031FD0A210090FCF761FA0746BE
:10BC800004F0E4FD0A210090FCF770FA80B2019004
:10BC90002C46002C07D000BF03E0FF20A055701CED
:10BCA000C6B2082EF9D307210906206888430199F6
:10BCB0000912090607221206114008432060606835
:10BCC000000A00020199C9B208436060FF2109021D
:10BCD00060688843390C0902FF22120211400843B0
:10BCE0006060110260688843390A09041202114039
:10BCF0000843606060680002000A3906090E090600
:10BD00000843606004F062FDC007C00FC0070090E8
:10BD100020684000400800990843206004F00CF8B7
:10BD20000007000F009020680009000100990843F7
:10BD3000206003F0FBFF022806D1012109072068DB
:10BD400088434018206004E00121090720688843E7
:10BD5000206004F001FD0001F021084000902068FF
:10BD6000884300990843206004F0A2FDFF2806DD07
:10BD7000FF21090420688843401820600BE004F08C
:10BD800097FD0004FF2109040840009020688843C3
:10BD9000009908432060FEBDFEB505460026002040
:10BDA0000190002704F068FB64210090FCF7DEF9A5
:10BDB00080B20190002001F0B1FC87B22C46002C2B
:10BDC00007D000BF03E0FF20A055701CC6B2082EAC
:10BDD000F9D32068000A00020199C9B20843206023
:10BDE000FF2109042068884339120904FF22120444
:10BDF00011400843206020680002000A3906090E3D
:10BE000009060843206003F09DFF28300002FF214F
:10BE10000902084000902068884300990843206088
:10BE2000FEBDFFB581B004460F4600250026002068
:10BE300000902760039820810498E060002020741F
:10BE400000BF9DE01C206843216808586A016168B2
:10BE500088501C2068432168081880686A0161685E
:10BE6000891848601C2068432168081840686A01E6
:10BE70006168891888601C20684321680818C068B8
:10BE80006A0161688918C8601C2068432168081825
:10BE9000007C6A016168891808741C206843216865
:10BEA0000818407C6A016168891848741C2068433E
:10BEB00021680818807C6A016168891888831C20C1
:10BEC000684321680818C07C6A0161688918887411
:10BED00000206A0161688918C8741C2068432168C1
:10BEE00008184068002813D01C20684321680818EF
:10BEF000C07C002805D1401E6A0161688918C8838A
:10BF00001AE00020C0436A0161688918C88313E001
:10BF10001C20684321680818C07C002805D0002038
:10BF20006A0161688918C88306E000206A016168B7
:10BF30008918C88301200090002607E000216A01CB
:10BF40006068801814308155701CC6B26901606841
:10BF50004018808BB042F1DC1C206843216808182F
:10BF6000406900280AD06B016268D218104614306C
:10BF70001C236B432268D21851698847681CC5B2DC
:10BF80002089A84200DD5DE7009805B0F0BD000003
:10BF900000B58BB068480790002108A8017068467A
:10BFA000017608A84170002064498872082108A819
:10BFB000C170002004E0002209A90A54411CC8B243
:10BFC00008A9C9788142F6DC5D48FFF7AAF806A9FE
:10BFD0005B48FFF7CFF85848401C0790002108A89D
:10BFE00001706846017608A84170002053498872A4
:10BFF000082108A8C170002004E0002209A90A5401
:10C00000411CC8B208A9C9788142F6DC4C484030CE
:10C01000FFF787F806A94A484030FFF7ABF84520FC
:10C0200000010790002108A801706846017608A861
:10C030004170002041498872082108A8C170002081
:10C0400004E0002209A90A54411CC8B208A9C97811
:10C050008142F6DC3A485030FFF763F806A93848C9
:10C060005030FFF787F8112040010790002108A801
:10C0700001706846017608A8417000202F49887237
:10C08000082108A8C170002004E0002209A90A5470
:10C09000411CC8B208A9C9788142F6DC2848203082
:10C0A000FFF73FF806A926482030FFF763F80B207A
:10C0B000C0010790002108A801706846017608A811
:10C0C000417000201D498872082108A8C170002015
:10C0D00004E0002209A90A54411CC8B208A9C97881
:10C0E0008142F6DC16486030FFF71BF806A91448B9
:10C0F0006030FFF73FF8FD20C00002900021684645
:10C1000001730171417381730821C173002004E040
:10C11000002204A90A54411CC8B26946C97B814265
:10C12000F6DC07481030FEF7FCFF01A90448103088
:10C13000FFF720F80BB000BDEE06000080260020BF
:10C140008055044030B585B0044600252068019034
:10C15000A1796846C1726179417200210172017052
:10C1600000BF05E020460830415D03A841556D1C25
:10C170006846C07AA842F5D80B22D2010199881AE4
:10C18000914226D007DC1848081A1CD02321090147
:10C19000401A24D111E0FF386F38002802D001285E
:10C1A0001DD104E069461148FFF7B5F818E069466B
:10C1B0000E484030FFF7AFF812E069460B485030A8
:10C1C000FFF7A9F80CE0694608482030FFF7A3F80C
:10C1D00006E0694605486030FFF79DF800E000BFC3
:10C1E00000BF05B030BD00002002000080550440B3
:10C1F000F0B585B004460F4600250026207C400699
:10C20000400E55287ED100BF76E169016068401874
:10C21000807C002877D169016068401840686A0115
:10C22000616889188968884209D269016068401884
:10C230004068C0196A016168891848605AE169015B
:10C2400060684018C068AF49884208D869016068D2
:10C250004018C068401C6A0161688918C86069019B
:10C2600060684018C07C002821D1002607E000212A
:10C270006A016068801814308155701CC6B269016B
:10C2800060684018808BB042F1DC1C206843216854
:10C290000818406900280AD06B016268D21810465D
:10C2A00014301C236B432268D218516988476901F6
:10C2B000606840580090690160684018017C6846D9
:10C2C000017100214171690160684018017F684671
:10C2D0008171690160684018417C6846C17100261F
:10C2E00008E06901606840181430815D02A881553A
:10C2F000701CC6B2690160684018808BB042F0DCE7
:10C30000E06801E0FCE01DE0002806D06846E16836
:10C3100088476A0161688918C874690160684018B3
:10C32000C07C002804D16A01616889184860E1E096
:10C330006901606840184068C01B6A01616889181B
:10C340004860D7E069016068401880680028EED036
:10C35000690160684018C08B0028E8D069016068F6
:10C360004018C08B6A0161688918C968884207D182
:10C37000690160684018C08B6249C94388427DD119
:10C3800069016068401840686A01616889188968B5
:10C39000884209D26901606840184068C0196A0182
:10C3A000616889184860A5E000206A016168891801
:10C3B0004860690160684018C0685249884208D8DE
:10C3C000690160684018C068401C6A01616889188A
:10C3D000C860002607E000216A01606880181430F8
:10C3E0008155701CC6B2690160684018808BB042EC
:10C3F000F1DC1C20684321680818406900280AD035
:10C400006B016268D218104614301C236B432268FB
:10C41000D2185169884769016068405800906901E5
:10C4200060684018017C6846017100214171690112
:10C4300060684018017F6846817169016068401832
:10C44000417C6846C171002608E0690160684018B7
:10C450001430815D02A88155701CC6B26901606804
:10C460004018808BB042F0DCE068002808D06846B5
:10C47000E16888476A016168891800E015E0C874BE
:10C48000690160684018C07C002804D16A016168B5
:10C49000891848602EE06901606840184068C01B38
:10C4A0006A0161688918486024E01C20684321689B
:10C4B0000818406800280FD00020C0436A01616856
:10C4C0008918C8831C2068432168081840686A01DD
:10C4D00061688918886008E000206A01616889182D
:10C4E000C8836A0161688918886000206A016168F0
:10C4F0008918C860681CC5B22089A84200DD84E69E
:10C5000005B0F0BD0000FFFF38B500BF1921254878
:10C510000078FBF715FE044623486043234A811840
:10C52000002201200BF082FE20460A225043643094
:10C53000001981B2002201200CF07CFF01200A22A8
:10C5400062431219D1B20A22624312190090D0B28A
:10C5500001231A4608F0B2FFBA220721002006F094
:10C56000EDFC6F20604381B201200DF009FA104804
:10C5700060430246032101200AF05AFD002505E030
:10C58000012128460AF08EFC681CC5B20F2DF7DB8E
:10C5900021460B2251436431C8B20DF055FC0DF019
:10C5A0003DFC38BD6F000020672B0000A086010015
:10C5B000FCB10100002005490870054908700549D3
:10C5C0000870054908700549087070477000002020
:10C5D000710000206F0000206E0000206D00002020
:10C5E000F0B589B000BF00BF00BF00BF00200690BB
:10C5F00000BF00BF00BF00BF00BF03215348007849
:10C60000FBF7B4FD52494843029003210120029AEE
:10C610000AF00EFD05214D480078FBF791FD044618
:10C62000E1B201200AF0CCFA032148480078FBF778
:10C630009DFD0B214843643080B20790E1B2012395
:10C640001846079A09F014FA404909788A008818B0
:10C650000621FBF78BFDFF21F531484380B208909E
:10C660000898FBF783FDC7B23946012009F0E4FEC4
:10C67000032136480078FBF779FD0B2148436430ED
:10C6800085B20022294601200CF0D4FE03212F4858
:10C690000078FBF76BFD2F4948432F494018039062
:10C6A0000022012003990BF0C1FD032127480078E7
:10C6B000FBF75CFD0B21484380B204900321234823
:10C6C0000078FBF753FD0B21484386B20120F1B2FD
:10C6D0000090049AD0B201231A4608F0EFFEBA2265
:10C6E0000721002006F02AFC032118480078FBF7F8
:10C6F0003DFD6F21484380B20590012005990DF062
:10C700003FF9164800783C2805DA14480078401CA8
:10C710001249087002E03C20104908700F48007868
:10C720001D2805DC09480078401C084908700BE00A
:10C7300006480078002802D10449087004E0034844
:10C740000078401E0149087009B0F0BD700000205B
:10C75000FCB10100672B0000A086010071000020E1
:10C76000002000BF06E00021044A1154044A11547D
:10C77000411CC8B25A28F6DB704700006C2200202A
:10C7800020230020FFB581B004460F463D46208996
:10C79000A8422DDD1820684321680818007C002875
:10C7A00026D1002609E00498815D1820684322689C
:10C7B000101808308155701CC6B2082EF3D3012121
:10C7C000182068432268101841742C20684361685F
:10C7D0000818006A00280BD018236B432268D2186F
:10C7E000104608302C236B436268D218116A8847C0
:10C7F00005B0F0BD01460620104BCA1A99420FD071
:10C8000008DCCA1FFA3A002A12D0102A0AD01F2ABE
:10C8100010D10BE0C02A07D0C12A0BD100200BE0B9
:10C82000012009E0022007E0032005E0042003E0E6
:10C83000052001E0062000BF00BF70474103000053
:10C8400010B504467D21C90061430846322103F03A
:10C85000B5FD10BD01480068704700004C00002085
:10C8600001480068704700004800002010B50549E5
:10C8700009886522514308466421FBF777FC80B2A2
:10C8800010BD0000560000200148007870470000ED
:10C890005B00002001480078704700005400002031
:10C8A00010B50EF009F801282CD100F063F8012032
:10C8B00000F066F803F0E6FD044600F043F803F0EC
:10C8C000A3FF044600F04AF804F0E2F8012805D17D
:10C8D00000F03EF8012000F047F805E0002000F0ED
:10C8E00037F8002000F040F8002013490860134892
:10C8F0000068134988421ED210480068801C0F4906
:10C90000086018E000200D4908600B4800680C49D9
:10C91000884204D208480068801C0749086000204B
:10C9200000F028F8012000F02BF8002000F00AF8B1
:10C93000002000F013F810BD4C000020480000203B
:10C94000FFFFFF7F0149088070470000560000206C
:10C9500001490870704700005B0000200149088011
:10C96000704700005800002001490870704700001F
:10C970005C0000200149087070470000540000204E
:10C9800001490870704700005A0000200021014A48
:10C990001171704700600040002201494A757047DC
:10C9A00000600040002201494A7670470060004064
:10C9B0000021014A11727047006000400021014AC5
:10C9C00011737047006000400021014A11747047E4
:10C9D000006000400021014A11757047006000406E
:10C9E0000021014A11767047006000400022014991
:10C9F0004A73704700600040002201494A74704742
:10CA00000060004010B51C4C1C49206888421ED1B3
:10CA100006221B49201DFBF74EFC002817D10D22D2
:10CA2000184920460A30FBF746FC00280FD10622A1
:10CA3000154920461730FBF73EFC002807D1062297
:10CA4000124920461D30FBF736FC00280DD000F0BF
:10CA500089FE0A480E490860074811F00AFF0C4A8F
:10CA60002421054811F030FF04E024222146084823
:10CA7000FBF7FDFB10BD0000000250007AA7A55A8D
:10CA8000290700202F070020230700201D07002072
:10CA9000542B002000200849087008490870012024
:10CAA00007490870002007490870074807490860CF
:10CAB00000200749087070470B0700200A07002074
:10CAC0000D07002012070020250600003C0700206B
:10CAD0001C07002070B5054600BF9120684304463E
:10CAE0000A212046FBF72CFB0446641D204670BD3E
:10CAF00070B5A8B0054600240026A0216846FBF7C3
:10CB0000CFFB00F09FFC1E490A6814216943505076
:10CB100000211B480268142068431018416018481F
:10CB20000268142068431018816015484068002886
:10CB300024D000BF17E06006060E282E00D316E0B2
:10CB40000F480168142060430858B1006A465050ED
:10CB50000B4801681420604308184168701C80006D
:10CB60001150601CC4B20648007AA042E3DC00BF4A
:10CB700062000348694643680220984728B070BDA8
:10CB8000C82B002030B5A9B000240025A02101A8A1
:10CB9000FBF786FB00BF25E06006050E00F052FCA7
:10CBA0001F490A6814216143505000211C48026843
:10CBB0001420604310184160194802681420604333
:10CBC00010188160282D0BD215480168142060438D
:10CBD0000858A90001AA50500021681C800011507B
:10CBE000601CC4B20E48007AA042D5DC0C484068F4
:10CBF000002813D00A48007A4000282806D30848A5
:10CC0000282201A943680220984707E00448007AD7
:10CC10004200034801A943680220984729B030BD6B
:10CC2000C82B002010B50DF047FE01287ED1FFF77C
:10CC300017FE5549884216D20F2054494871887111
:10CC400008468078002801D1052048704F48807838
:10CC5000052802D100204D49487000204B49087238
:10CC60004872087035E0FA2048494871887148498F
:10CC7000088803F0F3FC4648807800280CD143492B
:10CC8000087008464079C87008468079087100200D
:10CC90008870487048721CE001203C4908700846C2
:10CCA000407A022805D1012048720020C87008711E
:10CCB0000FE03648407A00280BD1022033494872F1
:10CCC00008464078887008464079C87008468079E0
:10CCD00008712E4880782D494978884213DD00205C
:10CCE0002A49C87008460079401C08710846007936
:10CCF0008979884222DB002024490871084680781F
:10CD0000401E88701AE0214880782049497888427E
:10CD100014DA00201D4908710846C078401CC8700C
:10CD20000846C0784979884208DB00E01EE0002010
:10CD30001649C87008468078401C8870144880786E
:10CD4000002803D10120114908721BE01048008817
:10CD5000732803DB02200D49087213E00C48008899
:10CD600070280FDC0020094908720BE000200749F9
:10CD7000087008464079C87008468079087100201C
:10CD80000872487210BD0000B80B00005009002066
:10CD9000780000200020044988704870C87008712D
:10CDA00008724872704700005009002000200649B0
:10CDB00008808870054988704870FA20C87008712A
:10CDC0000020087248727047780000205009002047
:10CDD00070B503F087FB044603F096FB05460DF0A3
:10CDE0006BFD01282ED105211A48FEF78DF9552833
:10CDF00004D1002018498870088027E0012D04D153
:10CE0000002015498870088020E0012012498870B0
:10CE10001248844202DB201A84B200E000240A2176
:10CE20002046FBF7A3F9052901DB601D84B20C48FD
:10CE3000844200DD04460A212046FBF797F90649A3
:10CE4000088003E00020044988700880FFF7EAFEAC
:10CE500070BD00002008002078000020AA0A000011
:10CE6000C60700001CB500200090019000F0EAFA0F
:10CE70000B49086000200B49096808600A480068EF
:10CE800000280CD00749096808680A21FBF758F9FF
:10CE90000090012269460520034B1B6898471CBD82
:10CEA000D8070020CC070020D40700200020084924
:10CEB00048800849088008490880084908700849DE
:10CEC0008872084908804880012008717047000076
:10CED000300000202000002022000020240000203C
:10CEE0000408002028000020F8B503F0DDFA07460A
:10CEF00003F0ECFA0090FFF7CDFC012860D105218A
:10CF0000C548FEF701F9552802D00098012807D13D
:10CF10000020C2490870C2490880C249887256E0A0
:10CF2000BE480078002810D10120BC4908703D4659
:10CF30002846E917890F091889030D0CBA4885425C
:10CF400000DD0546B648058041E0B648807A4000DD
:10CF5000B4490F520846867A0EE07000B1490D5A66
:10CF6000701E4000085A7100AE4A5052701E4000B8
:10CF700011460D52701EC6B2002E08DD7000A94980
:10CF8000095A701E4000A74A105A8142E5DBA548A5
:10CF9000807A401CA34988720846807A052816DBEF
:10CFA000002088720846C5882846E917890F0918A5
:10CFB0008D109D48854200DD05469948058006E0B4
:10CFC00000209649087096490880964988729448CE
:10CFD000058896480088A84257DA94480088281A9D
:10CFE00084B292480079012827D190484088A04215
:10CFF0000BDA8E4840880A308C49488008464088C1
:10D00000A04204DD0846448001E088484480874807
:10D0100044882046E117890F09188C100A2C00DA81
:10D020000A24824800880019804908800846008840
:10D03000A84201DD08460580CDE07C4840881428E0
:10D0400005DD7A48408814387849488002E000209D
:10D0500076494880754844882046E117890F0918A9
:10D060008C100A2C03DA012070490871B3E06F4874
:10D070000088A04205DD6D480088001B6B490880D0
:10D08000A9E0002069490880A5E068480088A84216
:10D0900059DD66480088401B84B264480079012845
:10D0A00027D162484088142805DD6048408814383C
:10D0B0005E49488002E000205C4948805B48448823
:10D0C0002046E117890F09188C100A2C03DA022078
:10D0D000564908717FE05548008800195349088077
:10D0E000084600885049884275DD08464F49088047
:10D0F00071E04E484088A0420BDA4C4840880A3024
:10D100004A49488008464088A04204DD08464480D9
:10D1100001E046484480454844882046E117890F8D
:10D1200009188C100A2C00DA0A24404800882919B2
:10D13000884202DA3D4805804DE03C480088001BEB
:10D140003A49088047E0394844882046E117890F6A
:10D1500009188C100A2C3EDD34484088142805DD5F
:10D160003248408814383149488002E000202F4975
:10D1700048802E4844882046E117890F09188C10F2
:10D180002A480079012813D10A2C03DA0220274902
:10D19000087120E0254800880019244908800846C5
:10D1A00000882149884216DD08462049088012E09F
:10D1B0000A2C03DA01201D4908710CE01B48008885
:10D1C000A04205DD19480088001B1849088002E0CC
:10D1D00000201649088016480088502804DC1348AF
:10D1E00000881349088016E0104800881049098813
:10D1F000884204DD0D4800880D4908800BE00B488B
:10D2000000880B490988081A84B2502C03DB0748B0
:10D21000008807490880F8BD20080020240000206D
:10D220002000002004080020E02E0000280000203C
:10D230002200002010B5044664204443A12120466A
:10D24000FAF77EFF0446204610BD00007CB500249E
:10D2500000200190009000F03FFA05460A21FAF7FD
:10D260006FFF044601226946042000F027FD009864
:10D27000401C002814D17D20C000201811490860EE
:10D28000084600680190012201A9032000F062FD18
:10D290000120009001226946042000F05BFD0FE0B0
:10D2A000009801280CD17D20000120180549086054
:10D2B000084600680190012201A9032000F04AFD00
:10D2C0007CBD00002001002010B501200F4908702E
:10D2D00000200F49096808600D49096848600C4939
:10D2E0000968886000F07EF9FFF7BCFDFFF74AFC93
:10D2F00008480068002807D0012205480168083165
:10D300000020044B1B68984710BD0000A5070020B3
:10D31000A00700209C07002010B518480068184995
:10D32000884229D117480068002804D015480068B1
:10D3300080471549087015480068002804D0134834
:10D34000006880471249087012480068002804D01D
:10D35000104800688047104908801048006800287D
:10D3600005D00E48006880470D49088002E00D484E
:10D370000B49088000F078F810BD0000B0070020CD
:10D38000785634128C070020A40700209007002054
:10D39000A607002094070020A80700209807002077
:10D3A000AA0700201027000010B50023174C2360A7
:10D3B000174C2370174C2370174C2370174C238085
:10D3C000174C2380174C2370174C13682360174C9D
:10D3D00053682360164C93682360164CD36823600F
:10D3E000154C1369236000280CD0144B1860134CA3
:10D3F0000B682468A3600023104C246823600F4C42
:10D40000246863600E4B014C236010BDB007002000
:10D41000AC070020A4070020A6070020A8070020D2
:10D42000AA070020A50700208C07002090070020F5
:10D4300094070020980700209C070020A0070020E8
:10D4400078563412054800680549884203D10548DA
:10D450000068806870470020C043FBE7B0070020E9
:10D4600078563412A007002070B50024002500264D
:10D470003048007801285CD12F480078002858D126
:10D480002E480078012854D12D4805882D49098857
:10D49000694308462C49FAF753FE85B2E1200001A2
:10D4A000854207D81921694308460921FAF748FE41
:10D4B000044600E0244C2548006800680019234910
:10D4C00009680860214800680068204909684968BF
:10D4D000884207D31D48006800681C4909684968EC
:10D4E000461A0AE01948006840680021C943081A32
:10D4F0001649096809684018461C1548864218D321
:10D50000344601462046FAF71BFE04460F480068E1
:10D5100041680F48604308180C49096848600120B9
:10D520000C490870094800688068001907490968B3
:10D53000886070BDA4070020A5070020A607002072
:10D54000A8070020AA07002010270000A00700203D
:10D55000A0860100AC07002000220C4B1A600C4B87
:10D560000A681A600B4B4A681A600B4B8A681A608B
:10D570000A4BCA681A600A4B0A691A60002801D06F
:10D58000084A1060084A014B1A607047B007002033
:10D590008C070020900700209407002098070020A7
:10D5A0009C070020A00700207856341210B50A48C6
:10D5B000006800280ED00948007801280AD1002010
:10D5C0000649087001220648016808310020024B14
:10D5D0001B68984710BD00009C070020AC07002086
:10D5E000A00700201CB50020009001900024FFF748
:10D5F00029FF04460E480068046000200C490968B1
:10D6000048600B49096888600A48006800280DD006
:10D61000074800680068009005480068406801906D
:10D62000022269460120034B1B6898471CBD00007D
:10D63000B4070020B8070020F8B505460C4616468A
:10D640000027002D17D00E480560FFF7FBFE0746A8
:10D650002068B84203D90A480068076003E0084917
:10D6600020680968086006496068096848600449DC
:10D67000A0680968C8600348066000F005F8F8BDB6
:10D68000B4070020B807002070B500240025FFF77C
:10D69000D9FE04460F4800680068A04200D903E0A4
:10D6A0000C4800680068251A0A480068406840195C
:10D6B0000849096888600748006880680549096862
:10D6C000C968884205D903480068C06801490968EB
:10D6D000886070BDB407002001480068806870470A
:10D6E000B4070020002801D0024A1060024A1160ED
:10D6F00070470000B4070020B8070020054900204B
:10D7000005E00A1D135C044A1354421CD0B22028C1
:10D71000F7DB7047000650007C2B002001461048C4
:10D72000026814204843101882680D4803681420CA
:10D7300048431818C06882420BD90948026814206F
:10D7400048431018C2680648036814204843181854
:10D7500082600348026814204843101880687047AC
:10D76000C82B0020002005E019490A5C19490A5419
:10D77000411CC8B20628F7DB002006E016490A5C07
:10D780001449891D0A54411CC8B20D28F6DB00203B
:10D7900006E012490A5C0F4913310A54411CC8B211
:10D7A0000628F6DB002006E00D490A5C094919311C
:10D7B0000A54411CC8B20628F6DB002005E000220E
:10D7C00004491F310A54411CC8B20128F7DB7047D5
:10D7D00029070020582B00202F07002023070020B6
:10D7E0001D07002038B50446002000900094012257
:10D7F0006946052000F0AEFA38BD00001CB50020D7
:10D800000090019002226946062000F057FA06496E
:10D810000098C860019808610846C0680349C8605C
:10D820000148006908611CBD5C2400205C090020DF
:10D830001CB500200090019002226946062000F0ED
:10D840003DFA0B490098C860019808610020094919
:10D850000860486008724872887202F0C9FF054982
:10D86000C8720348C068C8600148006908611CBDEF
:10D870005C2400205C0900207CB5002400250020E9
:10D880000090019002F084FE9A49C86002F094FE74
:10D89000984908610846C0689749C968884205D117
:10D8A0009448006994490969884211D09148C06838
:10D8B000009090480069019002226946062000F01D
:10D8C00049FA8C48C0688C49C8608A480069086178
:10D8D00002F08EFF8749C87202F064FE044602F02F
:10D8E00077FE0546FEF7D6FF012874D10121834853
:10D8F000FDF70AFC552807D100207E4908724872BE
:10D90000086048608872A7E0FF2C01D0FF2D63D12A
:10D91000FF2C2AD1FF2D28D0002076490872022042
:10D92000487277480860FF201430684348604868B0
:10D930006621FAF705FC6F4948600846406870495F
:10D94000884202D908466B4948606A484068AA285C
:10D9500003D368484068FA2803D9012065498872D2
:10D960007AE000206349887276E0FF2C2AD0FF2DF0
:10D9700028D102205F490872002048726048486040
:10D98000FF2014306043086008686621FAF7D8FB6E
:10D9900058490860084600685949884202D9084633
:10D9A0005449086053480068AA2803D351480068C6
:10D9B000E62803D901204F4988724DE000204D49E7
:10D9C000887249E04E484B490860486000208872E0
:10D9D0000872487240E085E00220464908724872A9
:10D9E000FF2014306043086008686621FAF7A8FB3E
:10D9F00040490860084600684149884202D9084603
:10DA00003C490860FF20143068433A494860486840
:10DA10006621FAF795FB374948600846406838495F
:10DA2000884202D908463349486032480068AA282B
:10DA30000BD330480068E62807D82E484068AA284B
:10DA400003D32C484068FA2803D901202949887259
:10DA500002E00020274988722748C068002802D1C8
:10DA60002449087215E02448C068012802D12149E0
:10DA700008720EE02048C068022804D11D490872CF
:10DA80001F48486005E01C48C068032801D11949B7
:10DA9000087219480069002802D11649487215E039
:10DAA00015480069012802D1124948720EE0124857
:10DAB0000069022804D10F4948721148086005E046
:10DAC0000D480069032801D10A4948720A480069D3
:10DAD00002280ED00848C06802280AD00020054954
:10DAE000887206E0002003490872487208604860A6
:10DAF00088727CBD5C0900205C2400202008002086
:10DB0000DE030000FFB583B006460D46174600242D
:10DB10000020029000BF1420784380190190002E4D
:10DB200057D00198002854D02B4806602A490698FF
:10DB300048600846077200BF45E0FFF783FC02908B
:10DB4000200129580298814204D820012858401CFD
:10DB5000002806D1204902980A68142161435050D8
:10DB600006E0200129581C48026814206043115027
:10DB7000200140194068401C002807D100211648A8
:10DB80000268142060431018416008E02001401929
:10DB90004168114802681420604310184160200158
:10DBA000401981680C480268142060431018C16055
:10DBB00020014019017B08480268142060431018B6
:10DBC0000161601CC4B20448007AA042B5DC00F0D8
:10DBD00005F807B0F0BD0000C82B002070B5002488
:10DBE00000250026FFF72EFC054600BF4EE02A4820
:10DBF0000168142060430858A84239D826480168B3
:10DC00001420604308582E1A2348016814206043EA
:10DC100008184068811920480268142060431018D1
:10DC200081601D48016814206043081881681A4803
:10DC30000268142060431018C068814224D9164835
:10DC400001681420604308180069002803D02046AA
:10DC5000FEF74EFF18E010480168142060430818D2
:10DC6000C1680D48026814206043101881600BE001
:10DC700009480168142060430818406806490A688A
:10DC80001421614351188860601CC4B20248007AB4
:10DC9000A042ACDC70BD0000C82B002010B500BF56
:10DCA00014244C432318002805D0002B03D0024C29
:10DCB00020606260217210BDC82B0020F8B50546B7
:10DCC0000E4614462B0010F00FF90705131A2128F1
:10DCD0002F363D001D48FAF741FF1D4908701B48CB
:10DCE000FAF7F6FA07466421FAF72AFA30602AE0D2
:10DCF000A004020C31461020FBF72AF823E0A00410
:10DD0000020C31463020FBF723F81CE0A004020C83
:10DD100031465020FBF71CF815E0A004020C3146F8
:10DD20007020FBF715F80EE0A004020C31468020AD
:10DD3000FBF70EF807E0A004020C31469020FBF739
:10DD400007F800E000BF00BF0020F8BD4E2400200F
:10DD5000D500002070B505460E4614462B0010F085
:10DD6000C3F807051D242B323940470030680028CE
:10DD700002D1FAF791FD10E0642231685143084660
:10DD80001D49FAF7AFFA00201C49087001226421EE
:10DD90001948FBF74BF8194908702AE0A004020C57
:10DDA00031461020FBF792F923E0A004020C314623
:10DDB0003020FBF78BF91CE0A004020C3146502008
:10DDC000FBF784F915E0A004020C31467020FBF744
:10DDD0007DF90EE0A004020C31468020FBF776F9B5
:10DDE00007E0A004020C31469020FBF76FF900E039
:10DDF00000BF00BF70BD000040240020D400002000
:10DE000000B5B1B050211DA8FAF74AFA00201C90C5
:10DE1000142117A8FAF744FA0020149015901690D0
:10DE20001390402103A8FAF73BFA002001900290DA
:10DE30005249086001221DA9FFF740FF1D98401CB0
:10DE4000002801D11C9001E01D981C904C481790AF
:10DE50004C4818904C48199000201A904B481B9041
:10DE600017AA1CA94A48FFF79FFA02221EA90120FF
:10DE7000FFF724FF1E98401C002801D1149001E0F8
:10DE80001E9814901E98401C002801D1159001E0A6
:10DE90001F9815903F48169014A93F481B9AFFF70A
:10DEA000CBFB082220A90220FFF708FF2098401C86
:10DEB000002801D1039001E020980390219804905C
:10DEC00036480590012069460876801E079034493F
:10DED0000991012103A80177881E0B9030490D910B
:10DEE00001210BA80173881E0F902D49119101216A
:10DEF0000FA80173042203A92A481B9BFFF702FE07
:10DF000001221DA90320FFF7D9FE27491D980860AB
:10DF10001D98401C002806D1FF20F5300860012222
:10DF20000320FFF717FF01221DA90520FFF7C6FEFA
:10DF30001D98401C002807D101201C49886001223F
:10DF400008310520FFF706FF02221DA90620FFF772
:10DF5000B5FE1D98401C00280AD11448C0680190E5
:10DF6000124800690290022201A90620FFF7F2FE82
:10DF70000F480249086031B000BD0000D800002001
:10DF800095C8000089C800006DC8000055DD00007C
:10DF9000D423002076841E00E02300200F270000F9
:10DFA0009F860100F0230020200100205C24002037
:10DFB000A33AA55A00B585B014216846FAF770F95E
:10DFC00000200F4908600F4800900F4801900F484B
:10DFD0000290002003900E48049069460D48FFF718
:10DFE000BBFA0D480499FFF77DFB04210B48049A06
:10DFF000FFF754FE0A480249086005B000BD000062
:10E00000D800002095C8000089C800006DC8000035
:10E0100055DD0000D4230020E0230020F023002061
:10E02000A33AA55A00200B4908800B4908800B49E8
:10E03000088001200A49087000200A4908730A492B
:10E040000880488001200871002006494880088027
:10E0500070470000380000203A0000203C000020FB
:10E060003E0000201008002040000020FEB502F015
:10E0700055FA009002F05CFA0190FEF70BFC0128C3
:10E080006BD10521D448FDF73FF8552807D1002072
:10E09000D2490870D2490880D249888067E0019847
:10E0A000012807D10020CD490870CD490880CD490D
:10E0B00088805CE0C9480078002808D10120C74961
:10E0C0000870009D0A206843C54908804FE0009809
:10E0D00081B2C448007B4200C248801D8152801F2B
:10E0E000067B11E07100BF48801D455A701E41003B
:10E0F000BC48801D415A72008152701E4100B948CF
:10E10000801D4552701EC6B2002E0ADD7100B54852
:10E11000801D415A701E4200B248801D805A8142C3
:10E12000E0DBB048007B401CAE4908730846007B2A
:10E13000032807DB00200873084605890A20684386
:10E14000A74908800020A74908804880A448008883
:10E1500088800120A149087009E000209F490870CB
:10E160009F4908809F4908804880087388809C48A0
:10E1700005889D480088A84256D29B480088281AE6
:10E1800084B299480079012826D197484088A04256
:10E190000BDA95484088801C93494880084640889F
:10E1A000A04204DD0846448001E08F4844808E4848
:10E1B000448803212046F9F7D9FF84B2022C00DA03
:10E1C0000224894800880019874908800846008889
:10E1D000A84200D90D80CDE083484088062805DD9F
:10E1E00081484088801F8049488002E000207E49A5
:10E1F00048807D48448803212046F9F7B7FF84B260
:10E20000022C03DA012078490871B3E076480088CF
:10E21000A04205DD74480088001B73490880A9E00E
:10E22000002071490880A5E06F480088A84259D9AC
:10E230006D480088401B84B26B480079012827D1C3
:10E2400069484088062805DD67484088801F664980
:10E25000488002E0002064494880634844880321E4
:10E260002046F9F783FF84B2022C03DA02205E49CC
:10E2700008717FE05C48008800195B490880084607
:10E2800000885A49884275DD08465749088071E080
:10E2900055484088A0420BDA53484088801C5249B8
:10E2A000488008464088A04204DD0846448001E0DA
:10E2B0004D4844804C48448803212046F9F756FFD6
:10E2C00084B2022C00DA02244748008829198842C7
:10E2D00002D245490D804DE043480088001B424969
:10E2E000088047E04048448803212046F9F73EFF74
:10E2F00084B2022C3EDD3C484088062805DD3A48C1
:10E300004088801F3849488002E000203649488014
:10E310003548448803212046F9F728FF84B2324863
:10E320000079012813D1022C03DA02202E4908714A
:10E3300020E02D48008800192B49088008460088F5
:10E340002A49884216DD08462749088012E0022C37
:10E3500003DA0120244908710CE023480088A04218
:10E3600005DD21480088001B1F49088002E00020CD
:10E370001D4908801C4800881D490988884203DA25
:10E38000194800880F2804DA1748008818490880BF
:10E390000AE01548008816490988081A0F2803DB87
:10E3A0001148008812490880114807880B480078F6
:10E3B00000280DD06C20474364213846F9F7C0FE91
:10E3C00007460A48874200D907460A490F8002E0FB
:10E3D000002008490880FEBD200800203E000020E3
:10E3E000380000201008002040000020C607000070
:10E3F0003C0000203A00002000200749088007491F
:10E4000008800749088048800120087100200549DC
:10E4100048800880704700003A0000203C0000203F
:10E420004000002010080020002004490870044922
:10E430000870002103480176704700008400002026
:10E4400085000020300D002070B500250024FEF767
:10E4500021FA012863D103213448FCF755FE5528E1
:10E4600008D1002032490870324908700021324832
:10E47000017659E02F480078002807D102F0B2F861
:10E480002B49087001202B4908704DE001202949D3
:10E49000087002F0A7F82849097E8900264A603AE8
:10E4A00050502548047E10E0A000234960390D5CDF
:10E4B000601E80000858A1001F4A603A5050601E3C
:10E4C000800011460D50601EC4B2002C0ADDA00071
:10E4D000194960390958601E8000174A603A10587F
:10E4E0008142E1D31448007E401CC1B2124801763B
:10E4F000007E1E2818DB00210F4801760146603996
:10E50000896B0246603AD26B89180246603A126CF7
:10E5100088180321F9F714FE0549087004E000206B
:10E52000034908700349087070BD000020080020EE
:10E530008400002085000020300D0020F0B5A9B037
:10E5400004460E460025002700202890A02168469A
:10E55000F9F7A6FEFEF776FF26490A681421614303
:10E56000505024480168142060430818C068B04225
:10E570000CD220480168142060430818C1681D4867
:10E580000268142060431018416005E019480168D2
:10E59000142060430818466016484068002826D0BA
:10E5A000002517E06806070E282F00D316E0114853
:10E5B0000168142068430858B9006A4650500D4855
:10E5C00001681420684308184168781C80001150C5
:10E5D000681CC5B20748007AA842E3DC00BF6A00A5
:10E5E00004486946436802209847012028902898EB
:10E5F00029B0F0BDC82B002010B500F0F5FD00F0EB
:10E60000D7F80EF0A7FB00F00DFB00F001F810BDED
:10E6100070B541480078912800D070BD00F0BEF878
:10E62000012876D13D4800883D4908800846807819
:10E63000F021884320303A498870084680780009E4
:10E6400000013549097A0907090F084334498870E0
:10E650003148807A401E3049887208460089401C43
:10E66000088108460089C988884216DA08202C49A2
:10E67000887200240EE0284841882848001D415C2B
:10E680002748C01C015524484088401C2249488026
:10E69000601CC4B2072CEEDB2DE01F4800891E4928
:10E6A000C98888421CD11C4800791B498978401AC6
:10E6B000C5B2681C1A49887200240EE016484188C9
:10E6C0001648001D415C1648C01C01551248408880
:10E6D000401C11494880601CC4B2AC42EEDB0AE029
:10E6E00000F00EFD00200C4908700C490888092133
:10E6F00000F0B8F991E7012000F0C4FC084A917AD3
:10E700001088921C00F070F905490888002100F07B
:10E71000C1F800BF81E7000008290020A4280020DC
:10E72000342800201B49097E002932D01949897EEE
:10E730000C225143174A515A174A118000200CE00D
:10E740001449897E0C225143124A8918891C0A5C9B
:10E750001149891C0A54411CC8B20828F0DB0D4934
:10E76000897E0C2251430B4A8918897A0A4A917290
:10E770000121D1720749097E491E064A11761146C8
:10E78000897E491C91761146897E022901DB002190
:10E790009176704700280020282800200349487BF4
:10E7A000012802D10021014A517370471829002025
:10E7B00010B533484068002861D13148007B030020
:10E7C0000FF092FB07590512212E3D4A59002D48A2
:10E7D0000078002807D000202A4908702A490888B4
:10E7E000012100F03FF947E026480078002809D0D1
:10E7F00000202449087025494A8808880123091DFA
:10E8000000F040F938E01F480078002807D00020C9
:10E810001C4908701C490888022100F023F92BE0EC
:10E8200018480078002809D00020164908701749B8
:10E830004A8808880923091D00F024F91CE01148C2
:10E840000078002807D000200E4908700E4908887B
:10E85000092100F007F90FE00A480078002809D0E4
:10E8600000200849087009494A8808880323091DBF
:10E8700000F008F900E000BF00BF00F041FC10BD4F
:10E880001829002008290020A42800204028002062
:10E890007047000070B504460D4634480088A04219
:10E8A00063D1002D61D13248007822284ED004DC9B
:10E8B00020283DD0212856D141E0902802D091282F
:10E8C00051D115E02A48C08801280AD100202849E2
:10E8D000087000F015FC27490888002100F0C2F8F4
:10E8E00005E0032000F0CEFBA020214908703BE0AA
:10E8F0001F4800891E49C98888420AD100201C4946
:10E90000087000F0FDFB1B490888002100F0AAF800
:10E910000DE01748807A002806D000F0F1FB14497A
:10E92000087B00F091FB02E0032000F0ABFB1BE052
:10E93000062000F0A7FB11200D49087014E0062006
:10E9400000F0A0FB11200A4908700DE000200849E2
:10E95000087000F0D5FB08494A8808880923091D7A
:10E9600000F090F800E000BF00BF70BD1C28002040
:10E9700008290020A42800204028002070B5034664
:10E98000184C247E022C00DB70BD164C647E0C25D6
:10E990006C43144D2B5300200AE0155C114C647E2F
:10E9A0000C2674430F4EA419A41C2554441CE0B239
:10E9B0008842F2D30B4C647E0C267443094EA41992
:10E9C000A1723446247E641C35462C762C46647E27
:10E9D000641C6C762C46647E022C01DB00246C7671
:10E9E00000BFD1E700280020F0B585B007460D46EE
:10E9F00016461A480780002406E031781748801C24
:10EA00000155761C601CC4B2AC42F6DB2C4605E016
:10EA1000AA211248801C0155601CC4B2082CF7DBE7
:10EA20000E480088019008216846C1720021417299
:10EA300001720170002406E00848801C015D03A8F3
:10EA40000155601CC4B2082CF6DB69460448FCF78B
:10EA500062FC01200149887205B0F0BD1C2800202D
:10EA60009055044070B504460D46294620460EF0E8
:10EA700093F870BD70B504460D46294620460EF049
:10EA800099F870BDF8B504460D4616461F463B463C
:10EA90003246294620460EF08EF8F8BDF8B50746F6
:10EAA0000E4615465C480078002804D009213846F7
:10EAB000FFF7D8FFF8BD002D01D0602D04DD09213E
:10EAC0003846FFF7CFFFF5E754480780458000241C
:10EAD00006E031785148001D0155761C601CC4B217
:10EAE000AC42F6DB00204C49487008468580FF2088
:10EAF00088727F2008730846808808282EDA012053
:10EB0000C8800846808848800120088143480088E2
:10EB10004349088008468078F0218843404988703E
:10EB200008468078000900013B4909790907090F67
:10EB300008433B49887038480079401C887200249B
:10EB400007E03648001D015D3548C01C0155601CBA
:10EB5000C4B231488088A042F3DC4AE00721681C37
:10EB6000F9F704FB002907D0072128460830F9F7F8
:10EB7000FDFA2949C88005E00721681CF9F7F6FA73
:10EB80002549C8800620244948800120088123485F
:10EB900000882349088008468078F0218843103097
:10EBA0001F49887008468078000900011A49898841
:10EBB0000905090F08431A49887008464088FF2153
:10EBC00009028843144989880902FF221202114070
:10EBD00008431349488008208872002407E00F4842
:10EBE000001D015D0E48001D0155601CC4B2062CBD
:10EBF000F5DB012000F046FA094A917A1088921C50
:10EC0000FFF7F2FE902004490870054908880021AA
:10EC1000FFF740FE00BF4DE708290020A428002090
:10EC20003428002010B5FFF77DFD1448C07A002875
:10EC300022D0124880780009002806D0012807D089
:10EC400002280AD0032810D10CE000F0A5F90FE04B
:10EC500000F09EF800F062FA0AE000F011F800F00F
:10EC60005DFA05E000F000F902E0FFF711FE00BFD9
:10EC700000BF00200149C87210BD000028280020F4
:10EC800010B540480078112800D010BD3E480088DB
:10EC90003F214901884200D0F7E73B4880780007D0
:10ECA000000F3849097A0907090F88420CD0002063
:10ECB0003449087000F024FA34494A88088804234B
:10ECC000091DFFF7DFFEE0E72E480089401C2D49B3
:10ECD00008810846807A401E887208460089C988E3
:10ECE00088421BDA2848807A082800D0CDE7002423
:10ECF0000EE02548C01C015D224842882348001DC3
:10ED0000815420484088401C1E494880601CC4B281
:10ED1000072CEEDB062000F0B5F930E019488088BA
:10ED200018494988401A1849897A884203DA1648EE
:10ED3000807A082800D0A8E700240EE01248C01C02
:10ED4000015D104842881148001D8154601CC4B206
:10ED50000C484088401C0B4948800A4840880949B3
:10ED600089888842EADB00200649087000F0C8F96B
:10ED700006494A8808880023091DFFF783FE00BF63
:10ED800083E70000082900202828002040280020D0
:10ED900070B53248007880210840802800D170BDCD
:10EDA0002F4800883F214901884200D0F7E72C48CE
:10EDB000807A082800D0F2E72948807805072D0FCF
:10EDC0002D0227484088000A0543082D00DAE6E7AF
:10EDD000002022494870062048800846858001208E
:10EDE0000881082088720020C8728988481C072181
:10EDF000F9F7BCF9002909D0184989880846083074
:10EE00000721F9F7B3F91549C88007E01349898844
:10EE1000481C0721F9F7AAF91049C8801048008852
:10EE20001049088008464580002407E00C48001D72
:10EE3000015D0C48001D0155601CC4B2062CF5DBB9
:10EE4000042000F01FF9102004490870054A518879
:10EE50001088FFF70FFE00BFA1E70000082900207F
:10EE6000282800204028002010B548480078A02815
:10EE700008D046480078912804D044480078A1285A
:10EE800000D010BD424800883F21490188420AD085
:10EE9000404908880921FFF7E5FD00F031F900201D
:10EEA0003A490870EDE73A48807A08280AD039498B
:10EEB00008880921FFF7D6FD00F022F90020334928
:10EEC0000870DEE7324880780007000F002804D081
:10EED00001282DD002284BD136E02C48407800285C
:10EEE00000D050E02A48C078002803D101202749EB
:10EEF000487003E02648C078244988722348007887
:10EF000091280BD022480079002803D101201F4905
:10EF1000087303E01E4800791C49087391201B49BF
:10EF2000087000F0EDF81949087B00F08DF82AE030
:10EF300016484078002800D025E0A1201349087029
:10EF4000032000F09FF81EE010484078002800D011
:10EF500019E00E480078A02809D10E490888082138
:10EF6000FFF780FD00F0CCF80020084908700AE0A7
:10EF7000084908880521FFF775FD00F0C1F8002059
:10EF80000249087000BF00BF00BF7AE708290020CF
:10EF900028280020A428002010B5284800788021C7
:10EFA0000840802800D110BD24480078002806D0F1
:10EFB000234800883F214901884200D0F3E72048D8
:10EFC000807A1F4989780907090F884203DD1C48A8
:10EFD000807A082800D0E6E7194880780007000FFB
:10EFE000002805D0164880780007000F072800DDAC
:10EFF000D9E7134800881349088011488078000732
:10F00000000F4880002407E00D48C01C015D0D483A
:10F01000001D0155601CC4B20A484088A042F3DCC0
:10F0200000200649087000F06BF806494A880888F5
:10F030000023091DFFF726FD00BFB4E708290020C3
:10F0400028280020402800207F2805DC7D21C900D9
:10F0500041430A4A91600DE0F12808DBF92806DCFB
:10F060000107090F64225143044A916002E00449F8
:10F07000024A91600221014A517370471829002009
:10F0800018F0010000B503000EF02EFF0729050B54
:10F0900011171D2329000121144A117314495160CD
:10F0A00022E00221114A1173114951601CE0032131
:10F0B0000E4A11730F49516016E004210B4A117377
:10F0C0000D49516010E00521084A1173002151607B
:10F0D0000AE00621054A11730849516004E0002145
:10F0E000024A1173516000BF00BF00BD1829002003
:10F0F000A8610000F824010028230000F049020064
:10F100000020014908737047182900200249098826
:10F110000918014A118070471829002010B52F489E
:10F120000078102818D12E48408860280ADD2D4824
:10F13000807800090001801C2A4988702220274914
:10F14000087025E02748807800090001254988706B
:10F150002020224908701BE020480078112816D191
:10F160001E48807A002800D010BD1C484078002836
:10F1700000D0F9E70820194988721A4880780009F8
:10F1800000011849887020201449087000E0EBE75E
:10F19000FD20C0001349088008468078F02188438C
:10F1A0003030104988700846C0780020C870084682
:10F1B000007914200871032088720220FFF762FF93
:10F1C000084A917A1088921CFFF70EFC05490888BE
:10F1D0000021FFF75FFB00BFC6E700000829002001
:10F1E0004028002034280020244A118852888A426E
:10F1F00042D0224A52888A4204DA204A52888A1A25
:10F2000090B207E01D4A52880023DB439A1A521C31
:10F21000521890B2194A5180127B002A10D0174A16
:10F220005268002A0CD0154A5268824205D9134A06
:10F230005268121A114B5A6002E000220F4B5A60BA
:10F240000E4A527B022A17D10C4A9268002A0CD02F
:10F250000A4A9268824205D9084A9268121A074BF4
:10F260009A6002E00022054B9A60044A9268002AE4
:10F2700002D10122014B5A73704700001829002067
:10F28000FEB5002700200290019000900025002686
:10F290000024FDF7FFFA012879D10021A748FBF7E8
:10F2A00033FF552808D1A6480178A648F8F7F8FF9B
:10F2B0000020A349087040E101F0A8F9074601F0D9
:10F2C000B9F9029001F0ACF9019001F0BDF900909C
:10F2D00001F092F99C490870F020384000110A288A
:10F2E00005DBF02038400011C01C054303E0F0208E
:10F2F0003840001105432D023807000F0A2804DBAF
:10F300003807000FC01C054302E03807000F054313
:10F310002D02F0210298084000110A2805DB02980E
:10F3200008400011C01C054304E0F0210298084089
:10F33000001105432D0202980007000F0A2805DB83
:10F3400002980007000FC01C054303E00298000765
:10F35000000F0543F0210198084000110A2805DB41
:10F36000019808400011C01C064304E0F0210198F8
:10F37000084000110643360201980007000F0A28D2
:10F3800006DB01980007000FC01C064304E0CCE038
:10F3900001980007000F06433602F021009808404C
:10F3A00000110A2805DB009808400011C01C064324
:10F3B00004E0F0210098084000110643360200984E
:10F3C0000007000F0A2805DB00980007000FC01C8B
:10F3D000064303E000980007000F06435A480078F0
:10F3E000002811D100240AE00020A100554A505005
:10F3F000A100564A5050A100554A5050641C482C58
:10F40000F2D3002053490870524800784E490978D9
:10F41000884218DA002D16D04E4802784B4928460B
:10F4200000F0D8F800280ED14A48007880004749FB
:10F430000D5048480078401C46490870084601783D
:10F44000424800F0D8F8434800783F49097888429C
:10F4500018DA002E16D03F4802783C49304600F0BA
:10F46000B9F800280ED13B480078800037490E508B
:10F4700038480078401C37490870084601783348FE
:10F4800000F0B9F8334800782F49097888420EDD3A
:10F49000002407E00020A1002C4A5050A1002C4A73
:10F4A0005050641C482CF5D300202A490870294884
:10F4B00000782549097888423FD100240FE0A00058
:10F4C00022490858A100224A50500020A1001F4A9A
:10F4D00050501B4801781E4800F08DF8641C1D48F0
:10F4E00000788442EBD31848007815490870002052
:10F4F00018490870002413E0A00012490858A10020
:10F50000134A515888420AD0A00011460858A10059
:10F510000C4A50500A480178104600F06CF8641C00
:10F52000074800788442E7D307E00548017805489A
:10F53000F8F7B6FE002002490870FEBD2008002042
:10F540007E000020B00B00207C000020900A0020EC
:10F55000700900207D00002010B505F075FD10BD7C
:10F5600000BF704710B504468020204301460320A9
:10F57000400205F023FC10BD10B51021032040020D
:10F5800005F01CFC10BD000010B50224024805F077
:10F5900065FC0446204610BD0106000010B50021A0
:10F5A000014805F00BFC10BD0106000010B5044633
:10F5B000802020430146024805F000FC10BD0000F9
:10F5C0000106000010B51021014805F0F7FB10BD41
:10F5D0000106000030B503460C460021002000BFA4
:10F5E00006E08D0065599D4200D101204D1CE9B215
:10F5F0009142F6DB30BDF8B505460E4600240EE01C
:10F60000601CC7B207E0BA005119A200501900F0FF
:10F610000AF8781CC7B2B742F5DB601CC4B2701E92
:10F62000A042EDDCF8BD10B503680C68A34203D915
:10F630000A6803680B60026010BD70B505460024BF
:10F64000FFF71EFE70BD00002E480078401C2D49BB
:10F6500008702D480078401C2B4908702B48007812
:10F66000401C2A4908702A480068401C2849086044
:10F6700008460068FF219131884202D900202449C0
:10F68000086020480078C82802D900201D49087069
:10F690001D480078842802D900201B4908701B48A7
:10F6A0000078502802D900201849087019481849D4
:10F6B0000968405C18490870184812490978405C8C
:10F6C00017490870174810490978405C16490870B6
:10F6D00016480E490978405C1549087015480949D3
:10F6E0000978405C14490870144806490978405C60
:10F6F00013490870134803490978405C124908709F
:10F70000704700004B0700204C0700204D070020E9
:10F7100050070020FFF30100440700208FF501008F
:10F720004507002057F6010046070020A3F7010017
:10F7300048070020DBF6010047070020F3F701002F
:10F7400049070020BBF801004A07002010B58200DD
:10F75000054BD218525C012A04D100228300024CCE
:10F760001B195A5410BD00008427002010B5044610
:10F77000204600F049FA204600F002F810BD0000D3
:10F7800010B50446B248007800287DD1B148008801
:10F79000B149884278DAB148007800284FD0B048A3
:10F7A0000078002803D0AB480088AE490880AE48F6
:10F7B0000078002818D1A7480188AA480088193085
:10F7C000814206D30120A8490870A2480088A549B3
:10F7D0000880A0480088A349098888421CDA9D480F
:10F7E0000088A049088017E09E4801889948008851
:10F7F0001930814206D300209B4908709548008843
:10F80000984908809348008896490988884203DD12
:10F81000904800889349088093480078002857D181
:10F8200092480078042803D08D480078002807D03B
:10F8300088480088822803DA05208C490870A1E0F6
:10F840008A480078032803D085480078002809D02A
:10F8500080480088FF211931884203DA0420834957
:10F8600008708FE081480078022803D07C48007837
:10F8700000280AD077480088FF21AF31884204DA97
:10F8800003207A4908707DE0E0E07848007801289C
:10F8900003D073480078002808D06E480088744967
:10F8A000884203DA0220714908706BE06F480078E3
:10F8B000002803D06A480078002863D06548008893
:10F8C0003721090188425DDA01206849087059E052
:10F8D00065480078012855D164480078012803D094
:10F8E0005F480078002809D05A480088372109016C
:10F8F000884203DB00205D49087043E05B480078E4
:10F90000022803D056480078002808D051480088C3
:10F910005749884203DB01205449087032E05348BC
:10F920000078032803D04E480078002809D04948C1
:10F930000088FF21AF31884203DB02204B49087069
:10F9400020E04A480078042803D045480078002881
:10F9500009D040480088FF211931884203DB032089
:10F96000424908700EE041480078052803D03C4821
:10F970000078002806D037480088822802DB04205F
:10F980003A490870FCF76CFF3349643988425DD30B
:10F990003848006800193749086031480078002865
:10F9A00008D000202E490870324908602F4800789E
:10F9B0003149087000F066FD00281FD12D4800680D
:10F9C0002E49884239D300202A4908602A48007805
:10F9D00026490978884205DA27480078401C2649DC
:10F9E00008702AE02448007820490978884224DDFC
:10F9F00021480078401E204908701EE01D4800681C
:10FA00001F49884219D300201A4908601A48007813
:10FA100016490978884205DA17480078401C1649CB
:10FA200008700AE01448007810490978884204DD1B
:10FA300011480078401E104908700F4800780B49A3
:10FA40000978884202D100200A49086010BD0000F0
:10FA50000B000020020000201C0C000012000020FF
:10FA600008000020040000200A00002006000020FA
:10FA7000760200001800002007000020C05D000092
:10FA8000407E050000200B4908700B4908700120DA
:10FA90000A4908700A49087000200A4908700A4992
:10FAA00008700A4908800A4908800A4908800A49FA
:10FAB00008707047060000200700002008000020A2
:10FAC000090000200A0000200B0000200C0000208C
:10FAD0000E000020100000201200002000200B4922
:10FAE00008700B49087001200A4908700A4908701B
:10FAF00000200A4908700A4908700A4908800A4922
:10FB000008800A4908800A490870704706000020EA
:10FB10000700002008000020090000200A00002043
:10FB20000B0000200C0000200E0000201000002020
:10FB300012000020F1B500272D480078002804D0DD
:10FB40000320F9F7FFFC2B4908802B48008819286F
:10FB500047D300202849088028480078142829D253
:10FB60000320F9F7EFFC0746002407E06000244972
:10FB7000085AB84200DD05E0601CC4B21F48007896
:10FB80008442F3DB00BF1D48057808E0681E400092
:10FB90001B49085A69001A4A5052681EC5B2A5424C
:10FBA000F4DC600016490F5214480078401C1349D9
:10FBB000087016E00026052405E060001049085A88
:10FBC0008619601CC4B20F2CF7D30A213046F8F70F
:10FBD000B7FA08490880002008490870012009493F
:10FBE0000870054801880098081803490880F8BD86
:10FBF0000900002002000020160000200000002064
:10FC0000DC070020120000203A4909881E2928DA62
:10FC10000021394A1180394A118039490988394A05
:10FC2000914207DC38490978002914D03449098801
:10FC3000914210DD0121354A11700021344A1170C2
:10FC4000344A1170304A11700121334A1170002179
:10FC5000324A11704CE02A4909880918284A118053
:10FC600046E024490988274A643291422BDB00216F
:10FC7000234A1180214A11801F490988AF221201AD
:10FC8000914207DC20490978002916D01A490988D1
:10FC9000914212DD02211D4A117000211C4A11708F
:10FCA00005211C4A11700021174A117001211A4ABE
:10FCB00011700021194A11701AE00F4909880918BA
:10FCC0000D4A118014E000210D4A11800A4A11806A
:10FCD0000A4909880B4A914205DD00210B4A11703F
:10FCE000094A117004E0054909880918034A11807E
:10FCF0007047000002000020100000200C000020CF
:10FD00000E000020B80B0000090000200B000020AE
:10FD10000600002007000020080000200A00002044
:10FD20000148007870470000500900200148007A1F
:10FD3000704700005009002001488078704700009B
:10FD4000500900200148008870470000780000201A
:10FD5000F8B50023002500950024002200BF94E0A0
:10FD600001259D40ACB20D8825400095009DA5421F
:10FD70006FD11A468D79012D0DD1464D03263602DD
:10FD8000AD192D5C012696403543424E03273F02B4
:10FD9000F61935540CE03F4D03263602AD192D5CA3
:10FDA00001269640B5433B4E03273F02F6193554D2
:10FDB000CD78002D4ED1374D60352D5CCE78002E9C
:10FDC00001D1012600E000269640B543314E603651
:10FDD00035548D78002D2ED12E4D19267601AD1972
:10FDE0002D5C8E78002E01D1012600E00026964081
:10FDF000B543284E19277F01F61935540D79002D8A
:10FE00000ED1244D50352D5C0E79002E01D10126E6
:10FE100000E000269640B5431E4E5036355423E090
:10FE20001C4D50352D5C0E7996403543EEB2194D80
:10FE300050352E5418E0174D19267601AD192D5C5A
:10FE40008E7896403543134E19277F01F6193554A5
:10FE50000AE018E00F4D60352D5CCE7896403543B2
:10FE6000EEB20C4D60352E544D79012D0AD1094D5D
:10FE700030352D5C012696403543EEB2054D3035C8
:10FE80002E5400E000BF5D1CABB2082B00DA67E720
:10FE9000F8BD000000000440FFB5074615461E46A9
:10FEA00000243846019900F01FF8002802D00120F4
:10FEB00004B0F0BD00240CE00A2060430949085C4E
:10FEC000B04204D12946204600F05EF807E0601CED
:10FED00084B20A2060430349085C0028ECD100BFCB
:10FEE0000020E5E7A80100200246002A03D14029AE
:10FEF00001DD01207047032A03D1022901DD012021
:10FF0000F8E7042A03D1202901DD0120F2E7052AC0
:10FF100003D1202901DD0120ECE70C2A03D11029AF
:10FF200001DD0120E6E70D2A05D1012903DD402985
:10FF300001DA0120DEE70E2A03D1202901D10120B8
:10FF4000D8E70020D6E7000010B5064A03231B02BD
:10FF5000D218125C8A43034B032424021B191A543F
:10FF600010BD00000000044010B5064A03231B0228
:10FF7000D218125C0A43034B032424021B191A549F
:10FF800010BD00000000044070B502460020B1E042
:10FF90000A2353435A4C1B195B1C440004191B19B8
:10FFA0009B788B427DD10A235343554C1B195B1C14
:10FFB000440004191B195B78082B33D10A235343DF
:10FFC0004F4C1B195B1C440004191B574D4C4E4DE4
:10FFD0006419E35C012423430A245443484D641903
:10FFE000641C450045196457464D474EAD192B55C5
:10FFF0000A235343424C1B195B1C440004191B5732
:020000040001F9
:10000000404C35466419E35C022423430A245443DC
:100010003B4D6419641C450045196457394DAD19B1
:100020002B5564E00A235343354C1B195B1C4400D9
:1000300004191B195B78092B34D10A235343304C24
:100040001B195B1C440004191B572E4C2E4D6419C0
:10005000E35C402423430A245443294D6419641C5F
:10006000450045196457274D274EAD192B550A23D6
:100070005343234C1B195B1C440004191B57214C90
:1000800035466419E35C8024A3430A2454431C4D81
:100090006419641C4500451964571A4DAD192B5558
:1000A00025E025E00A235343154C1B195B1C440033
:1000B00004191B57134C144D6419E35C0A24544370
:1000C0000F4D6419641C45004519641965780124B5
:1000D000AC402343DCB20A235343094D5B195B1C3C
:1000E000450045195B57074D074EAD19EC5404E028
:1000F000431CD8B2032800DA4AE700BF70BD0000F5
:10010000A80100200000044075080000F8B5002494
:10011000FCF7C0FB012861D100F02AFB0446BA229B
:100120000721002002F00AFF012C21D100F09EFBE4
:1001300000280ED000F050FB054600F041FB0646BB
:1001400001200346024629460090304605F0B6F9E4
:1001500050E000F041FB054600F032FB064601206E
:100160000023024629460090304605F0A7F941E0F9
:10017000022C21D100F07AFB00280ED000F02CFBDD
:10018000054600F01DFB06460120034602462946AF
:100190000090304605F092F92CE000F01DFB05467A
:1001A00000F00EFB0646002001231A462946009067
:1001B000304605F083F91DE000F058FB054600F0DD
:1001C0000BFB064600F0FCFA0746012003462A46D0
:1001D00031460090384605F071F90BE000200346E7
:1001E00002460146009005F069F9002207211046F9
:1001F00002F0A4FEF8BD0000F8B5002465480078C0
:10020000012824D1FCF746FB012812D1FCF77CF928
:1002100000BF0BE0182C02D1601CC4B204E0BA226B
:100220002146002002F08AFE601CC4B2242CF1DBBF
:10023000AEE0FCF795FA002406E0002221461046C5
:1002400002F07CFE601CC4B2242CF6DBA0E0FCF7BC
:1002500021FB01286DD1FCF703FB4F49884265D390
:100260004E480088032805DA4C480088401C4B495A
:10027000088011E000204949088000F0A7FA0646EE
:1002800000F0C2FA07460A21F7F75AFF0546324640
:100290002946012009F0CEF800F0DEFB064600F00A
:1002A000ABFB07460A21F7F74BFF054600F08EFA35
:1002B00032462946009007F0B9FFFFF727FF00F00C
:1002C0004BFA05462946012006F07AFC00F096FA22
:1002D0000646FF21F531F7F749FFC5B2294601204F
:1002E00006F0AAF8FFF71CFD0546FFF72BFD0646B2
:1002F000FFF722FD07462B4632463946012005F01E
:10030000B7FB00F0C5F805462946012009F038FB87
:1003100000F066FB054600F05DFB064600F066FB5C
:1003200007462A46314606F083FE31E0FCF758F9CD
:100330002EE0FCF715FA00222321104602F0FEFD04
:1003400000222221104602F0F9FD0022072110466A
:1003500002F0F4FD00220821104602F0EFFD002219
:100360000921104602F0EAFD00220A21104602F09F
:10037000E5FD00221321104602F0E0FD00221121CC
:10038000104602F0DBFD00221221104602F0D6FDDD
:10039000F8BD0000F9000020B80B0000720000203A
:1003A0000149086070470000780700200248006893
:1003B000401C01490860704774070020F3B581B004
:1003C000064600200E49086000F01EF8044600F0C2
:1003D0001BF805462F1B3046029903F013FD0090D1
:1003E0000AE000F011F805462F1B064800680028B7
:1003F00002D004480068804700988742F1D3FEBDD0
:10040000740700207807002001480068704700004A
:10041000740700200B490978012901D101200FE060
:1004200008490978022901D1022009E00549097823
:10043000032901D1042003E00121024A11700120A7
:10044000704700000D07002010B5094B1B8899B2BA
:100450000A12C8B2D3433133064C2370C34323334B
:10046000637013465633A37003467133E37010BDB7
:100470003C07002013070020014800887047000057
:10048000200000200148008870470000380000204C
:10049000014800787047000084000020014800787F
:1004A000704700008500002010B500220521064895
:1004B000FAF718FE0402012205210348FAF712FE9A
:1004C000201880B210BD00002008002010B50622C0
:1004D00005210348FAF706FEC006C00F10BD000054
:1004E0002008002010B5042205210648FAF7FAFD7D
:1004F0000402052211460348FAF7F4FD201880B2E1
:1005000010BD00002008002010B506220521024879
:10051000FAF7E8FDC01110BD2008002010B5022236
:1005200005210248FAF7DEFD10BD0000200800207A
:1005300010B5062205210348FAF7D4FD8006C00F46
:1005400010BD00002008002010B50422022103483D
:10055000FAF7C8FDC007C00F10BD0000200800203A
:1005600010B5052202210348FAF7BCFDC007C00FF1
:1005700010BD00002008002010B50022042103480F
:10058000FAF7B0FD4006400F10BD00002008002023
:1005900010B5042201210248FAF7A4FD801110BD14
:1005A0002008002010B5002201210248FAF79AFD28
:1005B00010BD00002008002010B5052201210348CD
:1005C000FAF790FD8007800F10BD00002008002082
:1005D00010B5012211460248FAF784FD10BD000053
:1005E0002008002010B5022203210248FAF77AFD04
:1005F00010BD00002008002010B503220021024891
:10060000FAF770FD10BD00002008002010B5002290
:1006100011460248FAF766FD10BD000020080020D0
:1006200010B5042200210248FAF75CFD10BD00005D
:100630002008002010B5012200210248FAF752FDDF
:1006400010BD00002008002010B50522002102483E
:10065000FAF748FD10BD000020080020322815DA06
:100660003C498978012903DD01213A4A517070E043
:1006700038498978002905DD2F286ADC0021354AB0
:10068000517066E00021334A517062E03E2817DA6B
:10069000322815DB2F498978022903DD02212D4AF2
:1006A000517056E02B498978012905DD3B2850DC43
:1006B0000121284A51704CE00121264A517048E03E
:1006C000502817DA3E2815DB22498978032903DDF3
:1006D0000321204A51703CE01E498978022905DD3A
:1006E0004D2836DC02211B4A517032E00221194AA2
:1006F00051702EE0622817DA502815DB15498978E9
:10070000042903DD0421134A517022E0114989783C
:10071000032905DD5F281CDC03210E4A517018E017
:1007200003210C4A517014E073280FDA62280DDBA4
:1007300008498978042905DD70280ADC0421054A66
:10074000517006E00421034A517002E00521014A7C
:100750005170704750090020014800787047000030
:10076000070000200148007870470000E5000020E5
:100770000148007870470000E4000020F8B500262A
:1007800000240025FCF7A8FF07460A21F7F7D8FC4C
:10079000054609480068854200D303E00648006822
:1007A000461B34467D200001844200D304460348A2
:1007B00004600068F8BD0000200100201C0100203A
:1007C0000148007870470000F100002001480079DE
:1007D000704700005C24002001484078704700000A
:1007E000F10000200148007A704700005C240020DE
:1007F00001484079704700005C24002001480088CF
:10080000704700002200002010B50024FFF7DEFF33
:1008100000280AD10A4800880A49884202DB0846B3
:10082000074908800648048808E005480088FCF766
:1008300001FD84B20448844200DB0446204610BD1A
:100840003A000020C6070000CE0400000020054941
:100850000988054A914202DB1146024A118001498A
:10086000088870473A000020C60700000148007859
:1008700070470000450700200148007870470000DD
:100880004707002070B5002407490868FCF722F9E3
:1008900005460A21F7F754FC84B20448844200DD7F
:1008A0000446204670BD00005C090020DE03000005
:1008B00010B5002400F016F8012801D103240CE043
:1008C00000F010F8022802D1FF24373405E00A2195
:1008D00003480088F7F74AFC84B2204610BD0000A8
:1008E0000200002001480078704700000B00002043
:1008F00010B50024044804F0B1FA002801D0012406
:1009000000E00024204610BD0307000010B50024BD
:10091000054804F0A3FA002802D00120044601E0B3
:100920000020044610BD00000507000010B500249B
:10093000054804F093FA002802D00120044601E0A3
:100940000020044610BD00000707000010B5002479
:10095000062004F083FA002801D0012400E00024DE
:10096000204610BD10B50024052004F077FA0028B9
:1009700001D0012400E00024204610BD10B5002461
:10098000054804F06BFA002802D00120044601E07B
:100990000020044610BD00000607000010B500242A
:1009A000044804F05BFA002801D0012400E0002490
:1009B000204610BD0305000010B50024044804F0D3
:1009C0004DFA002801D0012400E00024204610BD8B
:1009D000040500000148807870470000500D002099
:1009E0000148406870470000500D002001484078E1
:1009F00070470000500D002070B50024FFF7E6FEA0
:100A0000002803D1FCF768FE04460DE0FFF7DEFE88
:100A1000012806D1FCF760FE0546FCF70BFC0446F6
:100A200002E0FCF759FE0446204670BD70B5002474
:100A300007494868FCF74EF805460A21F7F780FB9E
:100A400084B20448844200DD0446204670BD0000A4
:100A50005C090020DE03000070B50024FFF7B6FE3D
:100A6000002803D1FCF75AFE04460FE0FFF7AEFE64
:100A7000012807D10020FCF751FE0546FCF7DAFB00
:100A8000044603E00020FCF749FE0446204670BD02
:100A900001480078704700003E00002070B5054610
:100AA0000024032D00D170BD002D01D0012D1BD1DC
:100AB00081210320800204F081F98021134804F091
:100AC0007DF932211248FFF779FC002409E0A200E9
:100AD000104BD2189178A200985A04F06FF9601C5C
:100AE000C4B23B2CF3DB0FE0022D0DD1002409E052
:100AF000A200094BD2189178A200985A04F05EF92E
:100B0000601CC4B23B2CF3DB00BFCCE70206000044
:100B1000A086010084EA010070EB0100F8B5002115
:100B200000240023002200BF0AE001258D40ABB263
:100B300005881D402C469C4200D10A464D1CA9B296
:100B40001029F2DB0588FF2D1FDC284D6D7E0688FD
:100B5000B543264E757635462D7E0688B543234E21
:100B6000357635466D7E8678F607F60F9640354326
:100B70001E4E757635462D7E867802273E407608D5
:100B800096403543194E357622E0184DED7E0688A5
:100B9000B543164EF5763546AD7E0688B543134E01
:100BA000B5768578ED07ED0F1646083EB5400F4E39
:100BB000F67E35430D4EF5768578022635406D0874
:100BC0001646083EB540094EB67E3543074EB5760B
:100BD0000025009505E000BF6D462D786D1CEEB236
:100BE00000966D462D78012DF5D9F8BD206B044097
:100BF000C107C90F002905D00021394A117100220F
:100C000038490A7102210140002905D00021344AE7
:100C10001172002233490A7204210140002905D0D3
:100C200000212F4A117300222E490A730821014026
:100C3000002905D000212A4A1174002229490A748A
:100C400010210140002905D00021254A11750022FC
:100C500024490A7520210140002905D00021204A9D
:100C6000117600221F490A7640210140002904D054
:100C700000221B494A711B494A7180210140002909
:100C800004D0002216494A7216494A72FF210131E6
:100C90000140002904D0002211494A7311494A73C6
:100CA000012149020140002904D000220C494A7464
:100CB0000C494A74012189020140002904D0002214
:100CC00007494A7507494A750121C90201400029AF
:100CD00004D0002202494A7602494A767047000051
:100CE0000060004000610040C107C90F002905D025
:100CF00001223C490A7100213B4A11710221014045
:100D0000002905D0012237490A720021364A1172A2
:100D100004210140002905D0012232490A73002133
:100D2000314A117308210140002905D001222D49C3
:100D30000A7400212C4A117410210140002905D0A9
:100D4000012228490A750021274A117520210140F6
:100D5000002905D0012223490A760021224A117672
:100D600040210140002905D001221E494A7100227C
:100D70001D494A7180210140002905D001221949ED
:100D80004A72002218494A72FF21013101400029AC
:100D900005D0012213494A73002213494A730121E5
:100DA00049020140002905D001220E494A7400225F
:100DB0000D494A74012189020140002905D0012210
:100DC00008494A75002208494A750121C9020140B3
:100DD000002905D0012203494A76002202494A76B9
:100DE00070470000006100400060004010B50C48F2
:100DF0000078002803D00B4A50689168884708485B
:100E00004078002803D0084A506891688847044811
:100E10008078002803D0054A50689168884710BD43
:100E200000600040F802002078040020F80500204F
:100E300010B508480079002803D0074A10695169A5
:100E4000884704484079002803D0044A50689168D4
:100E5000884710BD00600040F80200208404002094
:100E600010B50848007A002803D0074AD069116AF3
:100E700088470448407A002803D0044A50689168A3
:100E8000884710BD00600040F80200209004002058
:100E900010B50848007B002803D0074A906AD16A41
:100EA00088470448407B002803D0044A5068916872
:100EB000884710BD00600040F80200209C0400201C
:100EC00010B50848007C002803D0074A506B916B8E
:100ED00088470448407C002803D0044A5068916841
:100EE000884710BD00600040F8020020A8040020E0
:100EF00010B50848007D002803D0074A106C516CDB
:100F000088470448407D002803D0044A506891680F
:100F1000884710BD00600040F8020020B4040020A3
:100F200010B50848007E002803D0074AD06C116D28
:100F300088470448407E002803D0044A50689168DE
:100F4000884710BD00600040F8020020C004002067
:100F500010B50848407F002803D0074A50689168C0
:100F600088470448007F002803D0044A906DD16D63
:100F7000884710BD00600040CC040020F80200202B
:100F800010B508484078002803D0074A5068916897
:100F9000884704480078002803D0044A506E916EB8
:100FA000884710BD20600040D8040020F8020020CF
:100FB00010B509480079002803D0084A106F516F16
:100FC00088470548001D4078002803D0044A50682F
:100FD0009168884710BD000020600040F8020020A2
:100FE000E404002010B5034AD06F78329168884736
:100FF00010BD0000F802002010B5024A5068916848
:10100000884710BD7C03002010B50948007C0028EB
:1010100003D0084A506891688847054810304078E6
:10102000002803D0044A50689168884710BD00002A
:1010300020600040880300200805002010B5024A07
:1010400050689168884710BD9403002010B5024A8B
:1010500050689168884710BDA003002010B509486A
:10106000007F002803D0084A5068916888470548E7
:101070001C304078002803D0044A506891688847A3
:1010800010BD000020600040AC0300202C050020B3
:1010900010B50C480078002803D00B4A50689168BE
:1010A000884708484078002803D0084A506891686B
:1010B000884704488078002803D0054A5068916822
:1010C000884710BD40600040B8030020380500206C
:1010D000B806002010B50D480079002803D00C4A4E
:1010E0005068916888470948001D4078002803D05F
:1010F000084A5068916888470448001D8078002895
:1011000003D0054A50689168884710BD4060004090
:10111000C403002044050020C406002010B50D487B
:10112000007A002803D00C4A506891688847094823
:1011300008304078002803D0084A506891688847F2
:10114000044808308078002803D0054A5068916828
:10115000884710BD40600040D003002050050020AB
:10116000D006002010B50D48007B002803D00C4AA3
:1011700050689168884709480C304078002803D0AF
:10118000084A50689168884704480C3080780028E5
:1011900003D0054A50689168884710BD4060004000
:1011A000DC0300205C050020DC06002010B50D48A3
:1011B000007C002803D00C4A506891688847094891
:1011C00010304078002803D0084A5068916888475A
:1011D000044810308078002803D0054A5068916890
:1011E000884710BD40600040E803002068050020EB
:1011F000E806002010B5024A50689168884710BD83
:10120000F403002010B50948007E002803D0084AE6
:10121000506891688847054818304078002803D006
:10122000044A50689168884710BD00004060004043
:10123000000400208005002010B50948007F002828
:1012400003D0084A50689168884705481C304078A8
:10125000002803D0044A50689168884710BD0000F8
:10126000406000400C0400208C05002010B50848A8
:101270000078002803D0074A5068916888470448DE
:101280004078002803D0044A50689168884710BD10
:1012900060600040180400209805002010B509483F
:1012A0000079002803D0084A5068916888470548AB
:1012B000001D4078002803D0044A50689168884790
:1012C00010BD00006060004024040020A405002040
:1012D00010B50948007A002803D0084A5068916880
:1012E0008847054808304078002803D0044A5068F1
:1012F0009168884710BD0000606000403004002005
:10130000B005002010B5024A50689168884710BDAA
:101310003C04002010B5024A50689168884710BD0F
:101320004804002010B50948007D002803D0084A71
:10133000506891688847054814304078002803D0E9
:10134000044A50689168884710BD00006060004002
:1013500054040020D405002010B50948007E002860
:1013600003D0084A5068916888470548183040788B
:10137000002803D0044A50689168884710BD0000D7
:101380006060004060040020E005002010B50948BE
:10139000007F002803D0084A5068916888470548B4
:1013A0001C304078002803D0044A50689168884770
:1013B00010BD0000606000406C040020EC050020BF
:1013C00010B5FE4800688079002806D001286ED04C
:1013D00002286DD003286CD104E2F84800684079F7
:1013E00003000CF081FD0A0614BC2BBC47BC67BC93
:1013F0009BBC08F027FE0020F0490968C873EF483D
:1014000000684079401CED4909684871AEE0EC493C
:101410000969EA4A1268D27A885C08F08BFEE748CC
:1014200000684079401CE54909684871E348006854
:101430004079401CE1490968487197E001F0E6FEF7
:10144000002810D108F076FEDC4800684079401C86
:10145000DA4909684871D94800684079401CD74981
:101460000968487105E008F017FE0020D3490968B3
:1014700048717BE001F0CAFE002811D1012008F07C
:1014800059FECE4800684079401CCC490968487133
:10149000CA4800684079401CC8490968487105E09D
:1014A00008F0FAFD0020C549096848715EE05FE078
:1014B000FEE0A3E101F0AAFE002828D1BF49096897
:1014C000C97A24225143BF4A12688918BB4A12685C
:1014D000D27B885C08F02EFEB8480068C07B401CB8
:1014E000B6490968C873B5480068C07B242814D37E
:1014F000B24800684079401CB04909684871AF485B
:1015000000684079401CAD490968487105E008F061
:10151000C3FD0020A9490968487127E001F076FE63
:10152000002815D1A5480068C07A401CA349096865
:10153000C872A2480068C07AA1490978884207DBCE
:1015400000209E490968C87201209C490968887179
:1015500008F0A2FD002099490968487106E008F0EA
:101560009BFD002095490968487100BF00BF4FE10D
:1015700092480068407903000CF0B6FC080513910E
:101580002A914791709108F05DFD00208B49096810
:10159000C8738A4800684079401C884909684871C6
:1015A00084E087490969854A1268D27A885C08F024
:1015B000C1FD824800684079401C80490968487133
:1015C0007E4800684079401C7C49096848716DE09C
:1015D00001F01CFE002811D1262008F0ABFD774851
:1015E00000684079401C7549096848717348006873
:1015F0004079401C71490968487105E008F04CFDCC
:1016000000206E490968487150E001F0FFFD002894
:101610001DD1012008F08EFD68480068C07B401C89
:1016200066490968C87365480068C07B242814D3DC
:10163000624800684079401C6049096848715F4809
:1016400000684079401C5D490968487105E008F070
:1016500023FD002059490968487127E001F0D6FDB3
:10166000002815D155480068C07A401C53490968C4
:10167000C87252480068C07A51490978884207DB2D
:1016800000204E490968C87202204C4909688871D7
:1016900008F002FD002049490968487106E008F099
:1016A000FBFC002045490968487100BF00BFAFE05E
:1016B00042480068407903000CF016FC0805138BC3
:1016C0002A8B478B638B08F0BDFC00203B490968DF
:1016D000C8733A4800684079401C38490968487125
:1016E0007EE037490969354A1268D27A885C08F089
:1016F00021FD324800684079401C30490968487132
:101700002E4800684079401C2C490968487167E000
:1017100001F07CFD002811D1252008F00BFD2748A1
:1017200000684079401C25490968487123480068D1
:101730004079401C21490968487105E008F0ACFC7B
:1017400000201E49096848714AE001F05FFD002849
:1017500010D108F0EFFC194800684079401C174987
:1017600009684871154800684079401C13490968A8
:10177000487105E008F090FC0020104909684871A4
:101780002EE001F043FD002815D10C480068C07A16
:10179000401C0A490968C87208480068C07A0849AC
:1017A0000978884207DB002004490968C8720320D1
:1017B00002490968887108F06FFC05E0C80700203D
:1017C000002C0020C407002000201249096848713D
:1017D00006E008F061FC00200E490968487100BF6E
:1017E00000BF15E000200B490968887109490968A4
:1017F0004871062007490968C87009E008F04CFCE8
:10180000002004490968487102490968887100BFCD
:1018100000BF10BDC807002010B56A4800684079B5
:1018200003000CF061FB090610C627C644C6608E93
:10183000C60008F007FC634800684079401C614915
:1018400009684871BCE0604909695E4A1268D27A49
:10185000885C08F06FFC5B4800684079401C59497F
:1018600009684871574800684079401C5549096823
:101870004871A5E001F0CAFC002811D14F2008F002
:1018800059FC504800684079401C4E49096848712D
:101890004C4800684079401C4A490968487105E095
:1018A00008F0FAFB002047490968487188E001F018
:1018B000ADFC002810D108F03DFC4248006840799A
:1018C000401C4049096848713E4800684079401C06
:1018D0003C490968487105E008F0DEFB0020394901
:1018E000096848716CE001F091FC002822D135486C
:1018F0000068C07A401C33490968C87231480068E2
:10190000C07A3149097888420FDB00202D490968E7
:10191000C8722C4800684079401C2A4909684871FF
:10192000002028490968486208E000202549096824
:10193000487103E0002023490968487108F0ACFBB6
:101940003EE020480068407C002816D01E48C06851
:10195000002803D01C48C168192088470020194975
:101960000968486217490968487116490968887109
:10197000052014490968C8701AE012480068406AD6
:10198000282807D20F480068406A401C0D490968A2
:1019900048620DE000200B4909684862094909685E
:1019A0004871084909688871052006490968C870A6
:1019B00006E008F071FB002002490968487100BF89
:1019C00000BF10BDC8070020002C002010B5002467
:1019D000F7480068807A01287ED1F5480068C07910
:1019E00000287AD0F24800688079002804D00128C5
:1019F00074D0022873D191E1ED480068007B24285F
:101A00006ED2EB480068C07901287AD1002475E0D5
:101A1000E7480068C07A24214843E649096840182D
:101A2000E3490968097B415CE1480068C07A2422E7
:101A30005043E14A12688018DD4A1268127B805CCC
:101A4000814229D0DA480068C07A24214843DA4923
:101A500009684018D6490968097B415CD448006888
:101A6000C07A24225043D34A12688018D04A1268A0
:101A7000127B8154CE480068407B242805D3CC4893
:101A80000068007BCA4909684873C9480068007B40
:101A9000C7490968887308E0C5480068407B242866
:101AA00003D20120C24909688871C1480068007BDF
:101AB000401CBF4909680873BD480068007B2428A2
:101AC00008D3BB480068407B242803D20120B849D2
:101AD00009688871B64805E0D3E1CDE169E0BAE173
:101AE00038E00EE00068007B242804D2B04800688B
:101AF0008079012800D103E0601CC4B2242C87D374
:101B000056E0002413E0AA480068C07A2421484324
:101B1000A94909684018015DA5480068C07A2422D7
:101B20005043A44A126880180155601CC4B2242C8A
:101B3000E9D300209E490968487323209C4909681D
:101B4000887301209A490968887124209849096896
:101B500008732DE0002096490968087394480068CE
:101B6000C07A401C92490968C87291480068C07ADE
:101B700092490978884217DB8D480068007C01286B
:101B800004D102208A490968887106E0002088494A
:101B90000968887186490968C87100208449096804
:101BA000C87283490968087400208149096848712E
:101BB00061E17F480068407903000CF095F9080561
:101BC00013A62AA651A68EA6012079490968087491
:101BD00008F038FA764800684079401C7449096872
:101BE000487199E075490969714A1268D27A885C2E
:101BF00008F0A0FA6E4800684079401C6C490968FA
:101C000048716B4800684079401C6949096848710F
:101C100082E001F0FBFA00281BD165490968497B85
:101C2000491CC8B208F086FA61480068407B6049E8
:101C30000968C8735E4800684079401C5C490968BF
:101C400048715B4800684079401C594909684871EF
:101C500005E008F021FA00205549096848715BE069
:101C600001F0D4FA00282BD151490968C97A2422FD
:101C70005143504A126889184D4A1268D27B885CD9
:101C800008F058FA4A480068C07B401C4849096877
:101C9000C87347480068C07B45490968897B88420A
:101CA0001ADD434800684079401C41490968487181
:101CB0003F4800684079401C3D49096848710BE085
:101CC00008F0EAF93A480068407B39490968C87366
:101CD00000203749096848711EE001F097FA002892
:101CE0000CD1334909688871242031490968C873C7
:101CF0002F49096848732E490968887308F0CCF9A0
:101D000000202B490968487106E008F0C5F9002059
:101D100027490968487100BF00BFACE0244800684B
:101D2000407903000CF0E0F808050F8E268E4C8EEB
:101D3000688E08F087F91E4800684079401C1C49ED
:101D40000968487185E01D490969194A1268D27A03
:101D5000885C08F0EFF9164800684079401C144987
:101D600009684871124800684079401C10490968A8
:101D700048716EE001F04AFA002811D1252008F0E0
:101D8000D9F90B4800684079401C09490968487135
:101D9000074800684079401C05490968487105E01A
:101DA00008F07AF9002002490968487151E0000002
:101DB000C8070020C4070020C0070020002C002016
:101DC00001F024FA002810D108F0B4F96448006842
:101DD0004079401C6249096848716148006840794F
:101DE000401C5F490968487105E008F055F900207A
:101DF0005B49096848712CE001F008FA00281AD103
:101E000057480068C07A401C55490968C872544850
:101E10000068C07A5349097888420CDB0020504999
:101E20000968C8724E49096888714D490968487146
:101E30004B490968C87108F02FF900204849096822
:101E4000487106E008F028F9002045490968487102
:101E500000BF00BF0FE008F01FF9002040490968EB
:101E600048713F49096888713D49096808733C49D0
:101E70000968C87200BF71E000203949096888729A
:101E80006CE037480068807A022867D134480068DF
:101E9000007A00285ED0324800684079002804D0DB
:101EA00001280CD0032846D11BE008F0CBF82C48C1
:101EB00000684079401C2A490968487149E00020BF
:101EC00008F038F9264800684079401C2449096820
:101ED0004871234800684079401C214909684871CD
:101EE00037E008F079F8002812D11D4800684078E2
:101EF000401C1B490968487019480068407803284D
:101F000012D301F023FA00201549096848700BE04C
:101F10000020134909680872AA20114909688870CD
:101F200000200F490968487008F0B6F800200C49F5
:101F3000096848710DE008F0AFF800200849096809
:101F40004871074909684870AA20054909688870DE
:101F500000BF03E0002002490968887210BD00003C
:101F6000C8070020002C0020F8B504460D460026C6
:101F70000C2060431D49085C002801D00120F8BDF9
:101F80000C2060431949401885600C2060434018BC
:101F90008068002801D10120F1E701210C20604375
:101FA000124A115400222046E317DB0E1B185B1166
:101FB0005B01E31A9B000E4FDB19E717FF0E3F1979
:101FC0007F11DA550BF0C2FF00222046E317DB0E2B
:101FD0001B185B115B01E31A9F00064BFB18E71708
:101FE000FF0E3F197F11DA553046C8E7F80200208E
:101FF000006000400061004000BFFEE70948008823
:10200000401C08490880084600880749884208DDC6
:1020100006480078002804D00846024908800120BC
:1020200088707047E0000020DC050000E40000201C
:1020300010B515488078012824D11448007801286B
:102040000CD113480078012808D10020114988706C
:10205000084602F0D5FC00200D4908700B480078B6
:1020600002280CD10C480078012808D10020094929
:102070008870084602F0C4FC002007490870002060
:102080000249087010BD0000E0000020E4000020BC
:10209000E6000020F1000020E7000020704700006B
:1020A00010B500F03DFE012803D100200149088051
:1020B000887010BDE0000020F0B505460E461746BA
:1020C00000243A463146284600F038FE00BF42E080
:1020D00000202101394A126850522101374A126802
:1020E0008918488000212001344A126880188180B4
:1020F0002001324A12688018C18020012F4A1268DC
:102100008018017220012D4A126880184172200146
:102110002A4A1268801881722001284A12688018A1
:10212000C17200202101254A126889180873002114
:102130002001224A126880184173002021011F4AA1
:10214000126889188873002120011C4A12688018BF
:10215000C173601CC4B21A484078A042B8DC642045
:102160001849096808807D20C00016490968488020
:1021700015481449096888807D20000111490968C3
:10218000C88010490968088110480E4909684881CB
:102190000F480C490968888140000A490968C881CC
:1021A0003220084909680882FF20F530054909688E
:1021B0004882044909688882F0BD00008807002031
:1021C0007C070020840700204C040000102700003A
:1021D0003075000038B5002404E00020134908558C
:1021E000601C84B2282CF8D301216846417001702C
:1021F0006A460F490D48FFF75FFF7D21C900322075
:1022000000F08CF90B490C4800F0A6F9094864303D
:1022100000F038F90748C83000F044F9074800F0EA
:1022200057F9074800F06AF938BD00007024002013
:10223000F4EF010028230000B80B00005424000034
:102240001027000010B51D480078002803D1012098
:102250001A49087030E019480078012810D1184850
:102260000078012808D1002016498870084602F03D
:10227000C7FB0020124908700220104908701BE0BB
:102280000E480078022810D10F480078012808D1A4
:1022900000200C498870084602F0B2FB00200A4971
:1022A000087003200549087006E0044800780328F8
:1022B00002D100200149087010BD0000E400002098
:1022C000E6000020F1000020E7000020F8B500241F
:1022D000002500262D48007800281ED12C480078C3
:1022E000002803D101202A49087016E02848007808
:1022F000012803D10220264908700EE02448007806
:10230000022803D103202249087006E02048007803
:10231000032802D100201E4908701C4800780128BB
:102320000ED10124172500261A48012332462946DA
:102330000090204601F0BAFD01201749087024E002
:102340001248007802280FD101243B2500261148AD
:10235000401C0123324629460090204601F0A6FD8C
:1023600001200E49087010E00848007803280CD1BD
:10237000FEF72CFA002803D101200949087102E078
:102380000020074908710BF081FDF8BDE400002032
:10239000E5000020F1000020E6000020E70000201A
:1023A0005C24002010B5044623000BF09DFD095B62
:1023B000060E16171819595A5E00FAF751FA2C49E9
:1023C000884201D3FFF782FF50E0FAF749FA284923
:1023D000884201D3FFF736FF48E047E046E045E09A
:1023E000FAF73EFA2249884239D301F019FD214813
:1023F0000078032814D120480078002810D1FEF777
:10240000F1F9002806D101201C4988608868FBF793
:10241000E9F905E00020194988608868FBF7E2F9CE
:1024200014480078012805D113480078002801D10C
:10243000FAF7A8FB10480078052803D101201049BD
:1024400008700AE00C480078062803D102200C49E5
:10245000087002E000200A49087009F0F9FA05E066
:1024600004E003E0FFF7CAFD00E000BF00BF10BDBD
:10247000B80B0000E5000020E40000205C240020F0
:10248000E800002001460020054A126852898A426D
:1024900001DC012002E0024A12681181704700004D
:1024A0008407002001460020084A126812898A42E7
:1024B00001DB012009E0054A126892898A4201DCA9
:1024C000012002E0014A1268518170478407002010
:1024D00001460020084A126852898A4201DB012025
:1024E00009E0054A1268D2898A4201DC012002E033
:1024F000014A12689181704784070020014600203C
:10250000054A126892898A4201DB012002E0024AF0
:102510001268D18170470000840700200246002025
:102520000C4B1B681B8A934201DD012010E08A429C
:1025300001DB01200CE0074B1B689B888B4201DC10
:10254000012005E0034B1B681A80024B1B68598071
:102550007047000084070020024600200C4B1B68D7
:102560001B8A934201DD012010E08A4201DB012039
:102570000CE0074B1B685B88934201DB012005E000
:10258000034B1B689A80024B1B68D9807047000080
:102590008407002070B5044600250C206043FE49E6
:1025A000096840184068002807D00C216143FA4AA6
:1025B000126889184868804705460C206043F64930
:1025C0000968085C002873D10C206043F24909684F
:1025D00040188068002874D02001F049096840182C
:1025E000C07A02280AD1032D08D10C206043EA4AA0
:1025F0001268801881680120884762E02001E7495D
:1026000009684018C07A02280AD1042D08D10C208C
:102610006043E14A1268801881680220884750E0D0
:102620002001DE4909684018C07A02280AD1052D28
:1026300008D10C206043D84A1268801881680320B2
:1026400088473EE02001D54909684018C07A022831
:102650000AD1062D08D10C206043CF4A1268801899
:102660008168042088472CE02001CC490968401883
:10267000C07A02280AD1072D08D10C206043C64A2F
:10268000126880188168052088471AE02001C34934
:1026900009684018C07A02280BD1082D09D10C20F6
:1026A0006043BD4A1268801881680620884708E0A8
:1026B0000DE00C206043B84A126880188168002041
:1026C00088472001B54909684018C5720CE30C2001
:1026D0006043B1490968085C012873D10C2060434C
:1026E000AD49096840188068002874D02001AB49C2
:1026F00009684018C07A03280AD1022D08D10C209D
:102700006043A54A1268801881680120884762E00A
:102710002001A24909684018C07A04280AD1022D74
:1027200008D10C2060439C4A1268801881680220FE
:10273000884750E02001994909684018C07A052867
:102740000AD1022D08D10C206043934A12688018E8
:102750008168032088473EE02001904909684018BD
:10276000C07A06280AD1022D08D10C2060438A4A7B
:10277000126880188168042088472CE0200187496E
:1027800009684018C07A07280AD1022D08D10C2008
:102790006043814A126880188168052088471AE0E2
:1027A00020017E4909684018C07A08280BD1022D03
:1027B00009D10C206043784A12688018816806208D
:1027C000884708E00DE00C206043734A12688018C7
:1027D0008168002088472001704909684018C57247
:1027E00082E20C2060436C490968085C0228F7D13A
:1027F000002D7DD1200169490968085A6849096896
:10280000098A884275DA200164490968085A0A3041
:1028100081B22001614A1268115220015F490968A2
:10282000085A5F490968098A884231DB20015B49FF
:102830000968401840885A4909680988884227DB96
:102840002001564909684018408855490968498857
:1028500088421DDC00202101504A126889184880F6
:1028600020014E4909684018807A0028B8D10C2010
:10287000604349490968401880680028B0D00C209E
:102880006043454A126880188168012088472BE21E
:10289000200142490968085A41490968098A884261
:1028A0009EDB20013D490968401840883C49096881
:1028B0008988884294DB200138490968401840889B
:1028C00037490968C98888428ADC00202101334AD7
:1028D0001268891848802001304909684018807AB8
:1028E0000028D4D10C2060432B490968401801E02E
:1028F00063E00BE080680028C9D00C206043264AC2
:1029000012688018816802208847EDE100202101CB
:10291000224A1268891848802101204A12688918C1
:10292000C872002120011D4A12688018C180200150
:102930001A4A1268801841722001184A12688018D9
:102940008172184801782001144A126880180172B7
:1029500000202101114A12688918888021010F4A3C
:1029600012688918087321010C4A12688918487383
:1029700021010A4A12688918887300212001074A38
:1029800012688018C1730C2060430349096840181D
:1029900080680028B9D007E0800700208807002061
:1029A000840700207C0700200C206043CF4A126877
:1029B000801881680020884796E1012DA5D120016B
:1029C000CB4909684018C07AA84225D000212001CF
:1029D000C74A12688018418000202101C44A126849
:1029E0008918C8802001C24909684018C572C148C9
:1029F00000782101BE4A126889184872002021011E
:102A0000BB4A126889188880BA4801782001B84A00
:102A100012688018017267E12001B5490968401801
:102A2000007AB4490978884220D0B2480078210160
:102A3000AF4A1268891808722001AD490968401828
:102A4000407AAC490978884209D02001A849096830
:102A5000401880882101A64A12688918C880002180
:102A60002001A34A12688018818012E02001A04949
:102A7000096840188088A04988420AD220019C49F0
:102A80000968401880880A302101994A126889181B
:102A900088802001964909684018408896498842F4
:102AA0000AD2200192490968401840880A30210161
:102AB0008F4A12688918488020018D49096840189A
:102AC000407A8C490978884205D001202101884A42
:102AD0001268891888722001854909684018408861
:102AE000864909680988884204DB00212001804A60
:102AF0001268115220017E4909684018807A002826
:102B00007ED10C206043794909684018806800280C
:102B100077D02001764909684018408877490968CC
:102B20000989884214DB2001714909684018007B3B
:102B300000280DD10C2060436C4A1268801881680F
:102B40000320884701202101694A12688918087307
:102B5000200167490968401840886849096849891F
:102B6000884214DB2001624909684018407B002834
:102B70000DD10C2060435D4A1268801881680420E2
:102B80008847012021015A4A126889184873200198
:102B90005749096840184088584909688989884216
:102BA00014DB2001524909684018807B00280DD1B0
:102BB0000C2060434D4A12688018816805208847C0
:102BC000012021014A4A1268891888732001484966
:102BD00009684018408849490968C989884210DB5A
:102BE0002001434909684018C07B00287CD10C2093
:102BF00060433E4A1268801881680620884701E0D9
:102C000007E03BE001202101394A12688918C873A6
:102C10006AE02001364909684018407A01282ED11F
:102C20003448007802282AD1200131490968401827
:102C3000C08832490968498A884255DB20012C49FD
:102C40000968401880882D490968898A88424BDBC9
:102C50000C2060432549096840188068002843D04B
:102C60000C206043214A1268801881680720884739
:102C7000002021011E4A12688918487234E02001A0
:102C80001B4909684018407A02282DD1194800785C
:102C9000012829D12001164909684018C088174920
:102CA0000968898A88421FDB200111490968401898
:102CB000808812490968498A884215DB0C206043E4
:102CC0000A4909684018806800280DD00C2060432C
:102CD000064A126880188168082088470020210170
:102CE000034A12688918487270BD000080070020EE
:102CF000880700207C070020F0FF000084070020E8
:102D000010B5002400BF04E02046FFF743FC601C20
:102D1000C4B202484078A042F6DC10BD7C07002017
:102D200010B50024044802F099F8002800D000E013
:102D30000124204610BD00000304000010B5074B1D
:102D400014781C7054785C70054B1960054B186042
:102D500003461833044C236010BD00007C0700209C
:102D600080070020840700208807002010B5044653
:102D7000012C09D1BA220C21002000F0DFF801213A
:102D8000022004F08FF808E000220C21104600F029
:102D9000D5F80021022004F085F810BD10B50024FC
:102DA00004210848F8F7B0F9552801D1012407E0BB
:102DB000042000F0A7FF002801D0002400E0012437
:102DC000204610BD2008002010B50446012C09D172
:102DD000BA221C21002000F0B1F80121062004F0E5
:102DE00061F808E000221C21104600F0A7F800213D
:102DF000062004F057F810BD10B50024062000F09E
:102E000081FF002801D0012400E00024204610BDED
:102E100010B50446012C09D1BA221721002000F078
:102E20008DF80121042004F03DF808E0002217216C
:102E3000104600F083F80021042004F033F810BDA0
:102E400000200449097A002901D0012000E0002077
:102E500070470000500D002010B50446022C1CD114
:102E600000220D21104600F069F8FDF7FFFC002854
:102E700009D0BA220B21002000F060F801210D20BA
:102E800004F010F847E000220B21104600F056F83D
:102E900000210D2004F006F83DE0032C1CD1002297
:102EA0000B21104600F04AF8FDF7E0FC002809D09D
:102EB000BA220D21002000F041F801210D2003F07D
:102EC000F1FF28E000220D21104600F037F8002124
:102ED0000D2003F0E7FF1EE0012C0ED1BA220D21D8
:102EE000002000F02BF800220B21104600F026F8FD
:102EF00001210D2003F0D6FF0DE000220D21104628
:102F000000F01CF800220B21104600F017F80021F9
:102F10000D2003F0C7FF10BD10B50024FCF706FF1D
:102F2000022801D1022406E0FCF700FF012801D1AC
:102F3000032400E00124204610BD000010B5064B1C
:102F40001B78834207DD242905D224234343034C05
:102F500024681B195A5410BD002C0020C007002003
:102F600010B574480068407903000AF0BDFF0B07F4
:102F700011D325D35A6D77D38DA8D30007F062F80B
:102F80006C4800684079401C6A4909684871CFE084
:102F900069494969087807F0CDF8664800684079C2
:102FA000401C644909684871624800684079401CC7
:102FB000604909684871BBE000F028F9002811D188
:102FC0007F2007F0B7F85B4800684079401C5949FA
:102FD00009684871574800684079401C554909689C
:102FE00048711DE0534800684078401C5149096809
:102FF000487050480068407803280BD300204D49A2
:1030000009684870AA204B4909688870032049491B
:103010000968C87007F040F80020464909684871FF
:1030200086E000F0F3F8002807D1424800684079B4
:10303000401C40490968487103E000203D49096887
:10304000487107F029F873E006F0FCFF3948006882
:103050004079401C37490968487169E03649496937
:103060000978491CC8B207F065F832480068407911
:10307000401C3049096848712E4800684079401C5E
:103080002C490968487153E000F0C0F800280FD1BE
:1030900006F0AAFF274909688870012007F01EF88A
:1030A000244800684079401C22490968487105E0BD
:1030B00006F0F2FF00201F490968487138E01D48FA
:1030C0000068807818280CD102201A490968087015
:1030D0000020184909684870042016490968C8701A
:1030E00011E0144800684078401C12490968487093
:1030F000104800684078032805D300F027F9002025
:103100000C490968487006F0C7FF002009490968A2
:1031100048710DE006F0C0FF0020064909684871BB
:10312000044909684870AA2002490968887000BFEC
:1031300000BF10BDC8070020002C002010B531488A
:1031400000684079002804D001280CD0032848D119
:103150001DE006F077FF2B4800684079401C2949A4
:10316000096848714BE028490969087806F0E2FFD0
:10317000244800684079401C224909684871214868
:1031800000684079401C1F490968487137E000F029
:103190003DF800280CD101201A4909680870002068
:1031A000184909684870042016490968C87011E078
:1031B000144800684078401C12490968487011485A
:1031C00000684078032805D300F0C0F800200D49BE
:1031D0000968487006F060FF00200A4909684871D4
:1031E0000DE006F059FF00200649096848710549BD
:1031F00009684870AA2003490968887000BF00BFA9
:1032000010BD0000C8070020002C002010B506F0FB
:10321000E3FE04461F4800680078002838D01D48A7
:103220000068C078042833D3002C09D10021194844
:103230000068C07A8200174800681430815027E087
:1032400014480068C07A8100124800681430405861
:103250001149884211D20F480068C07A81000D4898
:10326000006814304058401C0A490968C97A8A002D
:1032700008490968143188500AE000F067F8002115
:1032800004480068C07A8200024800681430815007
:10329000204610BDC8070020B80B000000B587B05D
:1032A00001206946087108480290084803900848C0
:1032B0000490084805900848069001A9074800F0C6
:1032C0000FF807B000BD00000536010049500100AD
:1032D00075E0010061F0010060F00100D8240020D9
:1032E000F8B506460F46002400253946304600F062
:1032F000EFF900BF14E000250EE000212420604318
:103300000B4A12688018415524206043094A12680C
:1033100080184155681CC5B2242DEED3601CC4B280
:1033200005480078A042E6DC00F010F8F8BD000087
:10333000C0070020C4070020002C00200120024903
:103340000968087170470000C807002010B500F038
:1033500073F9002003490968087002490968C870B8
:1033600010BD0000C807002007480068C078062884
:1033700008D105480068C079002803D1012002491E
:103380000968C87170470000C807002010B555488B
:103390000068C07803000AF0A7FD08671D1A17141B
:1033A000110E056650484068002803D04E48416819
:1033B0000020884793E000F0E5F890E000F0C6F8C0
:1033C0008DE000F0D1F88AE0FFF7B8FE87E0FFF764
:1033D000C7FD84E044484068002803D04248416863
:1033E000012088473F480068407C00281AD03E48AA
:1033F000C068002803D03C48C168C8208847002026
:10340000384909684862374800680078002804D0C5
:10341000042034490968C87024E002203149096851
:10342000C8701FE02F480068406A401C2D49096899
:1034300048622C480068406A7D21C900884211D347
:10344000002028490968486226480068007800285A
:1034500004D0042023490968C87003E002202149F0
:103460000968C8703BE000BF1F484068002803D0CF
:103470001D484168002088471A480068407C0028A1
:1034800013D01948C068002803D01748C168C82065
:103490008847002013490968486212480068C078CC
:1034A000401C10490968C87018E00E480068406A5E
:1034B000401C0C49096848620A480068406A7D213E
:1034C000C90088420AD300200649096848620548B5
:1034D0000068C078401C03490968C87000BF00BF7D
:1034E00010BD0000C8070020002C002010B51548B2
:1034F0000068C078072824D0012012490968487460
:1035000008E011488068002802D00F498868804789
:10351000FFF73CFF0B480068C0780628F1D1094846
:103520000068007A0028ECD106480068C0790028BD
:10353000E7D104480068807A0028E2D1014909688F
:10354000487410BDC8070020002C002010B50548A5
:1035500000680078012802D1FDF732FF01E0F6F79C
:10356000C7F810BDC807002010B5054800680078EE
:10357000012802D1FEF750F901E0F6F797FC10BDE3
:10358000C807002010B51D480068807A002829D19E
:103590001A480068007A002803D0022017490968F9
:1035A000887216480068C079002803D001201349AA
:1035B00009688872114800680079012812D100203A
:1035C0000E49096808710D490968887207200B497E
:1035D0000968C8700A484068002803D00848416854
:1035E00000208847054800680078012802D1FEF7CE
:1035F000EDF901E0F6F734FD10BD0000C80700202A
:10360000002C002010B504462146084801F042FC79
:1036100007480078002805D1002C03D03221054846
:10362000FCF7CCFE0248047010BD0000010300004E
:10363000FA00002050C300000020244909684870A7
:10364000AA20224909688870002020490968486238
:103650001E49096808711D49096848711B490968B4
:1036600088711A490968C8711849096808721749A8
:103670000968887215490968C8721449096808738D
:1036800024201249096848731049096888730F4952
:103690000968C87300200D49096808740B49096856
:1036A00048740A490968887408490968C874074950
:1036B0000968486100210548006881610348006885
:1036C000C16102480068016270470000C80700201D
:1036D00010B50A780D4B1860034628330C4C236054
:1036E00024235343044628341B190A4C23600A4CF4
:1036F0004B6863608B68A360CB68E3604B69636170
:103700000B6923610B78237010BD0000C8070020EF
:10371000C0070020C4070020002C002007480068D4
:10372000C078062808D105480068007A002803D12F
:10373000012002490968087270470000C80700208C
:1037400010B50446012C09D1BA2220210020FFF730
:10375000F5FB0121084603F0A5FB08E0002220212B
:103760001046FFF7EBFB0021012003F09BFB10BD8F
:1037700010B50024032000F0C5FA002801D0012470
:1037800000E00024204610BD10B50446032C0ED1E5
:10379000BA2215210020FFF7D1FB00221421104688
:1037A000FFF7CCFB01210E2003F07CFB39E0022C5B
:1037B0001CD1FDF75BF8002809D0BA2214210020A3
:1037C000FFF7BCFB01210E2003F06CFB08E0002298
:1037D00014211046FFF7B2FB00210E2003F062FB1C
:1037E000002215211046FFF7A9FB1AE0012C0ED18B
:1037F000BA2214210020FFF7A1FB01210E2003F0C3
:1038000051FB002215211046FFF798FB09E000222A
:1038100015211046FFF792FB002214211046FFF7F6
:103820008DFB10BD10B50024F9F71AF8094988423C
:103830000DD3FDF757F8002807D1FCF78DFF0128BD
:1038400001DD032404E0022402E0022400E001245C
:10385000204610BDB80B000010B50446012C09D15C
:10386000BA221D210020FFF769FB0121002003F08F
:1038700019FB08E000221D211046FFF75FFB002125
:10388000084603F00FFB10BD10B50024022000F025
:1038900039FA002801D0012400E00024204610BDA0
:1038A00010B50446012C09D1BA221E210020FFF7D1
:1038B00045FB0121092003F0F5FA08E000221E2152
:1038C0001046FFF73BFB0021092003F0EBFA10BD87
:1038D00070B5002400250026FCF736FE0546FCF7EF
:1038E0003FFE064602210848F7F70EFC552800D196
:1038F00008E0012E01D1002404E0012D01D10124B2
:1039000000E00024204670BD2008002010B50446C9
:10391000012C09D1BA221F210020FFF70FFB012142
:10392000082003F0BFFA08E000221F211046FFF72D
:1039300005FB0021082003F0B5FA10BD70B5002486
:103940000025FCF74FFE054603211A48F7F7DCFB7C
:10395000552806D101201849088000201749088001
:1039600023E016480088012811D114490880FCF78B
:103970008FFD762803DA01200F49088015E0FCF757
:1039800087FD782811DB00200B4908800DE001201D
:103990000A490880FCF77CFD762803DA01200649F5
:1039A000088002E00020044908800348048820467B
:1039B00070BD000020080020180100201A0100201E
:1039C00010B50446012C09D1BA2221210020FFF7AD
:1039D000B5FA0121072003F065FA08E00022212151
:1039E0001046FFF7ABFA0021072003F05BFA10BD89
:1039F00010B50024FCF7C2FE002801D1012400E02C
:103A00000024204610BD10B50446012C09D1BA226D
:103A100016210020FFF792FA0121032003F042FA59
:103A200008E0002216211046FFF788FA0021032043
:103A300003F038FA10BD10B50024052000F062F93B
:103A4000002801D0012400E00024204610BD10B55C
:103A50000446012C09D1BA2219210020FFF76EFA81
:103A60000121052003F01EFA3CE0022C17D1FCF7DF
:103A7000FDFE002809D0BA2219210020FFF75EFAC6
:103A80000121052003F00EFA2CE000221921104636
:103A9000FFF754FA0021052003F004FA22E0032C7A
:103AA00017D1FCF7E9FE002809D0BA22192100201D
:103AB000FFF744FA0121052003F0F4F912E0002297
:103AC00019211046FFF73AFA0021052003F0EAF920
:103AD00008E0002219211046FFF730FA00210520E6
:103AE00003F0E0F910BD000010B50024FCF77AFEE9
:103AF00001282FD104211948F7F706FB552801D1D9
:103B0000012428E0FCF738FD01280BD0FCF734FD38
:103B1000022807D0FCF730FD032803D0FCF72CFD6A
:103B2000052801D1012416E0FCF726FD042801D167
:103B3000022410E0FCF720FD062801D103240AE04E
:103B4000FCF71AFD002803D0FCF716FD072802D168
:103B5000002400E00024204610BD000020080020C2
:103B600010B5F8F797FE0446204610BD10B5034B7C
:103B700008220349034800F013F910BD613B01001E
:103B800000F001009824002070B506465C4880686B
:103B9000002804D05A4988688047054600E000257F
:103BA0000024A6E0564841680C206043081840886D
:103BB000A84207D0524841680C206043081840884A
:103BC00002287DD14E4841680C2060430818806867
:103BD00000280CD04A494A680C2161435118886872
:103BE000804747490968E2008918487009E044485D
:103BF00041680C206043095C41480068E20080187D
:103C000041703F480068E100401840783C4909682D
:103C1000E200895C88420FD039480068E100401812
:103C2000417837480068E20081540020344909682F
:103C3000E200891848605AE031480068E100401805
:103C400041782F4842680C20604310184078814228
:103C50001FD12B480068E10040184168284842689D
:103C60000C2060431018808881420BD824480068DB
:103C7000E10040184068801921490968E20089186C
:103C8000486034E001201E490968E2008918488034
:103C90002DE01B480068E100401841681848426860
:103CA0000C2060431018C08881420DD81448006869
:103CB000E10040184068811911480068E20000E006
:103CC00009E08018416012E000200D490968E20017
:103CD000891848800BE0002009490968E20089182A
:103CE0004880002106480068E20080184160601C9E
:103CF00084B203488089A04200DD53E770BD000014
:103D0000B82B00200146064A92898A4205DD044A02
:103D10001268CB00D218508800E0002070470000E5
:103D2000B82B0020002000BF14E00D494A680C2188
:103D300041435118498801290AD10021084A1268D3
:103D4000C300D2185180064A1268C300D2185160CD
:103D5000411C88B2024989898142E6DC7047000033
:103D6000B82B0020002000BF13E00C494A680C214A
:103D7000414351184988002909D1084A1268C300F3
:103D8000D2185180054A1268C300D2185160411CF4
:103D900088B2024989898142E7DC7047B82B00204C
:103DA000F0B504460020164DAB6069602C60AA8116
:103DB00000BF1FE0124D6E680C254543755D104E27
:103DC0003668C700F61975700D4D6E680C254543B1
:103DD000755D0B4E3668C700F5550025084E3668F0
:103DE000C700F6197580064E3668C700F61975606B
:103DF000451CA8B2024DAD898542DBDCF0BD000058
:103E0000B82B002070B505460E46002E05D0314671
:103E10002846F4F795F9044600E02C46204670BD8C
:103E200010B5FCF7ABFC00280DD10748007801283D
:103E300009D005480078032805D0044800780028F8
:103E400001D1F9F703FA10BDE5000020E4000020DD
:103E500008B500200090012269460520F9F72EFFE1
:103E600005490098886000200449087004490870DA
:103E70000449087008BD00005C240020E400002014
:103E8000E6000020E700002008B500200090012295
:103E900069460520F9F712FF0020034908714871AF
:103EA0000098886008BD00005C24002070B5049C68
:103EB0002578914216DD01280AD18D4206DAFF26C7
:103EC000F61AAE420ED3EE18F5B20BE0154609E035
:103ED000022807D1954204DD9D4203DBEE1AF5B2BC
:103EE00000E00D46257070BD0D4A41685160816942
:103EF0009161C168D160416A5162016A11620168D1
:103F000011604169516181689160C169D161016944
:103F10001161816A91620021024A117070470000AC
:103F2000D42B0020BC07002010B5FFF7FBFEF8F7EC
:103F300041FB00210148F7F7E7F910BD2C080020EC
:103F400010B5F8F737FBFFF70DFF07F0C3FF08F0D8
:103F50005FF8FBF797FDFAF767FAFFF779FFF8F7D5
:103F600019FFF6F7D7FFF9F749FC55210348F7F792
:103F7000CBF9F8F747FDF9F7C1FB10BD2C0800207D
:103F80001CB500203049087006F00CF80020FCF742
:103F900085FD0AF0D1FAF7F7B5FC55212B48F7F764
:103FA000B3F9F8F72FFDF9F7A9FBF6F7ABFBF6F736
:103FB00029FEE120400209F001FF00F063FAF6F764
:103FC000A9FF06F0D1F9F8F7F5FAFAF72BF8F8F7A8
:103FD0006DFFF8F7EBFEFFF7C9FDFEF7FBF8FFF703
:103FE0005DF9FFF783FAF9F70BFFFBF777FDFAF7B7
:103FF0001BFA174AFF219131012008F0D5F8002261
:104000001146012008F014F807F04AFF08F000F804
:10401000FFF73AFFF9F70CFC00200E498871487150
:1040200008710120887048701420087007226846C3
:10403000F4F71DF90199009800F07CFF022101209E
:1040400000F058FE1CBD0000F90000202C080020E4
:104050000090D0030A0100207047000010B504460C
:10406000552C03D105494869804702E00349086897
:10407000804700200249087010BD0000D42B0020AA
:10408000BC07002010B546480078030009F02CFF5B
:104090000A06111B26303B46505173814148406847
:1040A000002802D03F494868804701203C490870F9
:1040B00000BF3C488068002804D03A49886880479F
:1040C0003749087069E03748C068002802D0354990
:1040D000C868804703203249087000BF3148006932
:1040E000002804D02F49086980472D49087054E002
:1040F0002C484069002802D02A494869804700209E
:104100002749087049E027488069002802D02549DE
:104110008869804706202249087000BF2148C0698D
:10412000002804D01F49C86980471D49087034E041
:1041300000BF1B48007807280AD11A48006A0028E7
:1041400002D01849086A804709201549087011E013
:104150001348007808280AD11248406A002802D083
:104160001049486A804709200D49087002E0002084
:104170000B49087000BF0A480078002808D0094899
:10418000806A002804D00749886A8047044908707B
:1041900003E000200249087000BF00BF10BD00000E
:1041A000BC070020D42B00207047000010B5002071
:1041B0000AF07EFA06F09EFF06F0F2FF07F008F81C
:1041C00000F08CFCF6F7AEFD0220FCF767FC002047
:1041D00007490870FFF78AF9FFF7B0F8FFF7D6F83C
:1041E000F6F700FC102008F0F5FB00F077FD10BD9D
:1041F0009401002010B5012406F05EFB012801D1D6
:10420000052407E0F8F726FB0349884201D2012480
:1042100000E00224204610BD204E000010B5062408
:1042200006F04AFB002800D1002406F04BFB0128D1
:1042300003D006F047FB072800D90924204610BD0B
:1042400010B5F6F76FFD00221146012008F022F8A4
:1042500000213A48F7F758F8002400BF00F0F4FEB8
:1042600032217D200001FCF7A9F8002034490870B4
:104270000AE00022324801781046FEF75FFE30481F
:104280000078401C2E4908702D4800782428F0DB67
:1042900000202C49087009E000212A48007807F026
:1042A00007FC28480078401C2649087025480078FB
:1042B0000D28F1DBFFF76AF8F6F76AFA06F04EFA16
:1042C00021480078401C20490870084600780528DD
:1042D00012D300200870FFF747F81C4800780A281E
:1042E00005D3002019490870FFF718FA04E01748B1
:1042F0000078401C1549087006F0E4FA0128ADD991
:1043000006F0E0FA0728A9D200200E49087008E05C
:104310000C48007807F0E6FB0A480078401C094981
:104320000870084800780D28F2DBF6F76BFC552181
:104330000248F6F7E9FF204610BD00002C080020D7
:10434000130100201101002012010020140100209F
:1043500010B5032408E000F077FE012000F07EFD98
:10436000002801D0042400E0F5E700BF204610BD7E
:1043700010B500202749086005F014FE0120FCF765
:104380008DFBF7F7BFFA55212348F6F7BDFFF8F785
:1043900039FBF9F7B3F90AF0CFF8F6F7B3F9F9F703
:1043A00009FEF6F72FFC06F0E9F9F9F73BFEFAF7FC
:1043B00023F8F8F77BFDFFF7D9FBFDF70BFFFFF7BD
:1043C000D1FCFFF745FDFEF769FFFFF78FF800F01E
:1043D00059F8E120400209F0F1FCF6F79BFDFBF7EC
:1043E0007DFBFAF721F80D4AFF219131012007F0FA
:1043F000DBFE00221146012007F01AFE07F050FDF7
:1044000007F006FEF9F7FAF90221012000F072FC2C
:1044100010BD00004C0000202C0800200090D003AC
:1044200070B506460D4614460E4806600E480560F7
:104430000E49206808600E49606808600D49A06850
:1044400008600D49206908600C49E06808600C4963
:104450006069086005480068002802D003480068C9
:10446000804770BDC0000020C8000020A8000020C8
:10447000AC000020B0000020B4000020B8000020F4
:10448000BC00002000B587B00C4801900C48029099
:104490000C4803900020049005900B4806900020E3
:1044A0000A49086048600A490860486001AA012179
:1044B000C9020848FFF7B4FF07B000BDD9440100A6
:1044C00021480100A947010031470100641500207F
:1044D0005C0D00206C1A002001207047F3B5C3B0BA
:1044E0000446449E0020009057E002E0641C761EC3
:1044F00000BF022E05D32078EB28F7D160789028F2
:10450000F4D1072E00D24AE0A778FD1CB54200D9AD
:1045100045E0A81E205C0002691E615C08434290D1
:10452000042D38D9291FA01C0AF020F8429988428E
:1045300026D11D480068002804D0B91EE01C1A4A84
:104540001268904719480068002824D0E17868462E
:104550000171207981116846417120798106890EA7
:1045600068468171381FC1B26846C171C279611D48
:1045700002A8F3F77CFE01A80C49096888470AE005
:104580000020009002E00098401C00900098A84293
:10459000F9D3002000906419761B072EA5D200BF26
:1045A0004498801B45B0F0BDB4000020BC00002042
:1045B000F7B5C0B0154600260027E81DFF210131E0
:1045C000884202DD002043B0F0BDEB216846017057
:1045D00090214170281DC1B2684681700021C170D0
:1045E0004098C1B2684601710524002605E0419853
:1045F000805D69460855641C761CAE42F7DBA11E3F
:1046000000A8023009F0B2FF87B238126946085597
:10461000641C0F55641C06480068002805D021461C
:104620006846034A12689047CDE70020CBE70000B8
:10463000AC00002070B50024002500261B4840680F
:104640001A490968884200D170BD18484068174966
:104650000968884205D91548406814490968451A0F
:1046600007E01248006811494968401A012189028F
:104670000D1AFF2D01D9FF2600E02E4600240DE083
:104680000A4801680830405C094908550748008815
:10469000401C8005800D05490860641CB442EFD3BE
:1046A000B1B2034809F0E6FB00BFCDE76415002076
:1046B0006C19002070B500251A480068002830D019
:1046C000194A1288FF230133991A184A1268164BA7
:1046D0001B88D018134A126890470546002D20D039
:1046E00011480088401910490880084601880F4881
:1046F0000068FFF7F3FE0446002C0DDD0A48008831
:10470000844209DA08480088021B08480068011939
:1047100006480068F3F7ABFD03480088001B024918
:10472000088070BDB0000020C4000020C000002040
:1047300010B50446A07810280CD1207919490870CA
:104740000846007801282BD1002211462020FFF7CF
:104750002FFF25E0A078122803D120791149087293
:104760001EE0A07801281BD12079332803D1012035
:104770000C49487005E02079352802D1002009490C
:104780004870607907498870607A0006217A0904C8
:104790000843E17909020843A179084301494860C7
:1047A00010BD0000500D002070B50346002200240B
:1047B00000251A484068194E3668B04201D10020E1
:1047C00070BD16484068154E3668B04205D913488A
:1047D0004068124E3668841B07E0104800680F4E90
:1047E0007668801B0126F602341AA14201D92546BB
:1047F00000E00D4600220CE0084806680830805DA5
:10480000985406480088401C4005400D034E306017
:10481000521CAA42F0D32846D2E700005C0D0020CB
:1048200070B503460022002415484068144D2D68D9
:10483000A84208D312484068114D2D68401B01253D
:10484000AD022C1A04E00E4800680D4D6D68441B43
:10485000A14201D9012070BD00220CE09D5C0848F6
:1048600046680830855508388088401C8005800DD2
:10487000034D6860521C8A42F0D30020EBE7000031
:104880006415002010B50248FFF72EFB10BD000094
:10489000E8F001000021014A1175704740600040B6
:1048A000014600BFF020084000110A235843024689
:1048B0000807000F8018C0B270470146002204E0CC
:1048C000501CC2B208460A38C1B20A29F8DA1007E9
:1048D000000E08437047000010B5044601218020F7
:1048E000F6F79CFD607A012805D14248C078102176
:1048F00008434049C870607AA22805D13E48007F2D
:10490000802108433C490877607A3B4908770020BA
:104910003A4948770846407F217808433749487725
:10492000E07B002805D00846407F2021084333491A
:1049300048773248407FC008C000A17A08432F4919
:1049400048770846807FF72108402C498877E0782F
:10495000FFF7B3FF29498874A078FFF7AEFF274916
:10496000C8746078FFF7A9FF2449087520780028EB
:1049700005D10846007D2179084320490875E07972
:10498000FFF79BFF1D4988756079FFF796FF1B496C
:104990004875A079FFF791FF1849C875207AFFF78D
:1049A0008CFF164908760846807F4006400E8877BF
:1049B000E07A002806D00846807F402108430F494E
:1049C000887703E00D48807F0C498877A07BFFF74C
:1049D00074FF0A498876607BFFF76FFF0749C87646
:1049E000207B08770846807F102188430349887719
:1049F00010BD00002004024060040440404F044009
:104A000010B504461B48807F012108431949887767
:104A10002078FFF752FF174908756078FFF74DFFC0
:104A20001449C874A078FFF748FF124988742078A9
:104A30000C2806DD0846407F082108430D494877C9
:104A400009E00C48407F0B4948770846007DE17833
:104A50000843084908750748807F40084000054919
:104A6000887700BF0348807F022108400028F9D1E1
:104A700010BD0000404F044010B5002014490876D6
:104A8000162009F057FA0021124801761248407F9B
:104A900080210843104948770846807F0121084358
:104AA0000D49887700BF0C48807F0221084000280C
:104AB000F9D00948807F400840000749887700BF47
:104AC0000548807F022108400028F9D110BD000070
:104AD0004060004040610040404F044010B500205D
:104AE0000749087000212020F6F798FC01210548AD
:104AF0000175002004490875152009F003FA10BD5E
:104B000000500440406100404060004070B50446E1
:104B10000D46002C14D0002D12D0042D10D800F01A
:104B200013F800280CD1002608E00649885D2246CB
:104B30000121F4F71BFCA41C701CC6B2AE42F4DBCE
:104B400070BD00007C01002000200549897DC90757
:104B5000C90F002901D0012000E0002070470000AB
:104B60000050044030B585B005460C460020039047
:104B70000490009001900290072C0BDC0120A040D3
:104B800081B2684681810121C17303A90220FBF72C
:104B9000DFF83EE0082C01D0092C0BD10120A04009
:104BA00081B2684681810121C17303A90120FBF70D
:104BB000CFF82EE00A2C03D00B2C01D00D2C0BD1FA
:104BC0000120A04081B2684681810121C17303A9FF
:104BD0000020FBF7BDF81CE00C2C01D00F2C0BD1F2
:104BE0000120A04081B2684681810121C17303A9DF
:104BF0000E20FBF7ADF80CE00E2C0AD10120A040EE
:104C000081B2684681810121C17303A90C20FBF7A1
:104C10009FF8002168460170C170417001218170C8
:104C200000210171C1720D218172FF2101720021E9
:104C30004172F4F7FBFB03491520FDF795F905B028
:104C400030BD00009548010010B5002010490875DE
:104C5000152009F057F900210E480175152000288C
:104C600009DB00BF00BFC206D20E012191400A4AF3
:104C7000116000BF00BF00BF084880798011032881
:104C800005D006480078802108430449087010BD0B
:104C9000406000404061004000E100E000500440FE
:104CA00010B5F4F7BDFC10BD10B501231A46002164
:104CB0001846F6F76FFB012211461046F6F7E0FBA7
:104CC000F6F7CCFB034809F029FC024802490860CA
:104CD00010BD00000090D0034007002000BF044832
:104CE0000069042108430249086130BF00BF7047D2
:104CF00000ED00E0F3B585B0054600200390049078
:104D0000EEB22804070E0F2F54DA082E52DA0020D4
:104D100009E00C214143284A515AA94201D10446D5
:104D200003E0411CC8B21728F3D300BF0120B040F4
:104D300086B20C20604320494018C3780C206043A1
:104D400040188278F8B231460190FBF7A5F8684622
:104D50008681012181730021C17302214174F8B25F
:104D600003A9FAF7F5FF0C216143134A8918C88893
:104D7000FBF7BAFF0C2060430F494018C188684612
:104D8000018169460698887202A8FBF7C7FE0C22CB
:104D90006243094BD21891680C226243D218042056
:104DA0001056FDF7E1F80C216143034A8918C888C1
:104DB000FBF71EFF07B0F0BD7CF20100FEB5054613
:104DC0000C460020C0430290EFB22804060E0F2EBE
:104DD00042DA082F40DA0120B84069460880802076
:104DE0002040002816D101208870A007800F0228DB
:104DF00001D1487109E0A007800F012802D169465E
:104E0000487102E0002069464871F0B26946FAF73D
:104E10009FFF1FE00020694688700E202040002878
:104E200000D000BF10202040002802D16946087140
:104E300002E0012069460871E007C00F002802D196
:104E40006946887102E0012069468871F0B26946BE
:104E5000FAF77EFF002002900298FEBD30B50146B1
:104E6000CAB20C04230E00200F2B0FDA082A0DDA29
:104E700001249440A2B2064C03252D026419E45C7F
:104E80001440002C01D0012000E0002030BD0000C3
:104E900000000440F8B504460F460020C0430090CF
:104EA000E6B22004050E0F2D11DA082E0FDA0120CC
:104EB000B04086B2002F04D1E8B23146FBF744F887
:104EC00003E0E8B23146FBF74FF80020009000986D
:104ED000F8BD00001649897F01221143144A9177D9
:104EE00000BF1349897F022211400029F9D01049DF
:104EF000897C81700E49C97C41700D49097D017022
:104F00000B498A7D8271497D01710949CA7D4271CF
:104F10000A7EC271897F49084900054A917700BF1E
:104F20000349897F022211400029F9D1704700000E
:104F3000404F044003B585B00020019002900390DB
:104F40000490002168464173817E01A8C1706846C3
:104F5000417E01A881706846017E4171002101A84F
:104F60000171082168460171817D01A8C1716846FF
:104F7000C17D4172417D01A881716846017D01A812
:104F80000172002168468173C17301A881730C21ED
:104F900041734121684601740021C17401A8FFF7E3
:104FA0009BFC1A200449888204491620FCF7DCFF88
:104FB00000F006F807B000BD204F044069E601008C
:104FC00010B5FFF759FD10BD70B504460D46601EC3
:104FD0000D49884200D90124002C00D10124402031
:104FE0000A4908700846007860430949486103216E
:104FF000081F08F0B7FF00200549886107200861F5
:105000000448056070BD0000FFFFFF006C01002038
:1050100000E000E0680100200020C043002809DB18
:10502000C206D20E01219140054A1160BFF34F8F95
:10503000BFF36F8F00BF002002490861886170478D
:1050400080E100E000E000E010B508F031FF10BDA5
:105050001A20084908722B2048723C2088724D2083
:10506000C8727F20044909680860AC200349487071
:105070007047000000040240700100200010024050
:1050800010B51C480078012812D11B48007864280C
:1050900009DB02201949487108710020164908707F
:1050A0001449087004E014480078401C1249087044
:1050B0001348007801281CD112480078012804D137
:1050C000002010490870104908700F4800783228F5
:1050D0000ADBF7F7DFFC00210C48F6F7CFF8552183
:1050E0000B48F6F711F904E007480078401C064920
:1050F000087010BD110700201007002000070020D5
:105100000A0700200C0700200B07002020080020C1
:105110002C080020F8B504460D460027002000901A
:1051200003200003204000130090102C04D0122C08
:1051300002D01148844217D122202840222806D1CB
:1051400027073F0F39460098F5F7C8FA06461220A0
:10515000284012280ED12007000F471C394600981E
:10516000F5F7BCFA064605E02107090F0098F5F7A8
:10517000B5FA06463046F8BD10100000F8B50446F2
:105180000D46002600270120000320400713102CA5
:1051900004D0122C02D00F48844215D1222028407E
:1051A000222805D12607360F31463846FAF7CEFABF
:1051B0001220284012280CD12007000F461C31462F
:1051C0003846FAF7C3FA04E02107090F3846FAF720
:1051D000BDFAF8BD10100000FFB58BB01C460020D2
:1051E0000790069005903848049010210B980840CD
:1051F000002801D0022707E040210B980840002832
:1052000001D0012700E00027002C04D0149804707E
:105210000120089001E010200890002548E0002CB3
:1052200008D025466000294A115A0C98F2F788FFE9
:10523000079006E06800254A115A0C98F2F780FFA3
:1052400007903E4630E0711C0798F2F779FF40085E
:1052500006900D98F3F7CAF803900D9A0699881AEC
:10526000F3F7C4F818490190F3F745F80290039951
:10527000F3F77EF805900598F3F7BFF84900490861
:10528000039102900498F3F7B8F849004908019196
:105290000090039B029AF3F7C5F803D20A9509968A
:1052A00005980490701CC6B27F2ECCDD681CC5B278
:1052B00008988542B3DB14990A98087014990998E4
:1052C000487004980FB0F0BD0000C84290F3010090
:1052D0000246412A2ED010DC212A2AD006DC102AD0
:1052E00045D0122A4BD0202A59D11CE0222A26D0A0
:1052F000232A2AD0402A52D116E081235B01D01AFA
:105300009A4228D008DC422A1AD0432A1ED02548C7
:105310001018002843D13AE0012822D020281BD0C1
:1053200021283CD11EE000BF1F4803890B430381A5
:1053300036E000BF1C4843890B43438130E000BF87
:10534000194883890B4383812AE000BF1648C3892B
:105350000B43C38124E000BF144883880B43838040
:105360001EE000BF1148C3880B43C38018E00E48FD
:1053700043890B43438103890B43038110E00A48AF
:10538000C3890B43C38183890B43838108E00748AA
:10539000C3880B43C38083880B43838000E000BF36
:1053A00000BF7047F0EFFFFF0011044000140440FD
:1053B000F0B505460E46412D30D010DC212D2CD005
:1053C00006DC102D51D0122D56D0202D62D11CE0BC
:1053D000222D2AD0232D30D0402D5BD116E0812103
:1053E0004901681A8D4230D008DC422D1ED0432D71
:1053F00024D02A48281800284CD144E001282CD079
:10540000202823D0212845D128E000BF244F388808
:10541000314600F049F804463DE000BF204F78884F
:10542000314600F041F8044635E000BF1C4FB88813
:10543000314600F039F804462DE000BF184FF888D7
:10544000314600F031F8044625E000BF154F38889A
:10545000314600F029F804461DE000BF114F78885E
:10546000314600F021F8044615E00D4F78883146AA
:1054700000F01AF804460EE0094FF888314600F0B3
:1054800013F8044607E0074F7888314600F00CF81F
:10549000044600E000BF00BF2046F0BDF0EFFFFF74
:1054A00000110440001404400246002013460B4043
:1054B000002B01D0012000E000207047FFB581B033
:1054C0000E461746012F07D1F748407D000900011D
:1054D000C01DF549487505E0F348407D000900010D
:1054E000F1494875049801287ED10A210198F2F704
:1054F00027FE0546ED48445DE007C00F002807D0B1
:10550000E948007C00090001C01DE749087405E076
:10551000E548007C00090001E349087402202040AE
:10552000002807D0E048C07BF02188437030DE4976
:10553000C87305E0DC48C07BF0218843DA49C873B2
:1055400004202040002807D0D748807C00090001B3
:10555000C01DD549887405E0D348807C000900014E
:10556000D149887408202040002807D0CE48407CCC
:10557000F02188437030CC49487405E0CA48407C2B
:10558000F0218843C849487410202040002807D0E3
:10559000C548407C00090001C01DC349487405E0AE
:1055A000C148407C00090001BF49487420202040C8
:1055B000002807D0BC48007CF02188437030BA49ED
:1055C000087405E0B848007CF0218843B6490874A7
:1055D00040202040002808D0B348807CF021884338
:1055E0007030B149887406E08BE0AF48807CF021D0
:1055F0008843AD4988740A210198F2F7A1FD0D4650
:10560000AA48445DE007C00F002807D0A648807B69
:10561000F02188437030A449887305E0A248807B5C
:10562000F0218843A049887302202040002807D039
:105630009D48807B00090001C01D9B49887305E0DF
:105640009948807B00090001974988730420204015
:10565000002807D09448007DF0218843703092499B
:10566000087505E09048007DF02188438E49087553
:1056700008202040002807D08B48007D0009000149
:10568000C01D8949087505E08748007D00090001B3
:105690008549087510202040002807D08248C07C2A
:1056A000F021884370308049C87405E07E48C07C92
:1056B000F02188437C49C87420202040002807D06E
:1056C0007948C07B00090001C01D7749C87305E017
:1056D0007548C07B000900017349C8734020204011
:1056E000002807D07048C07C00090001C01D6E4929
:1056F000C87454E06C48C07C000900016A49C87451
:105700004DE06948007C00090001674908740846BB
:10571000C07BF02188436449C8730846807C000937
:10572000000188740846407CF02188435E49487433
:105730000846407C0009000148740846007CF021BE
:105740008843594908740846807CF02188435649AB
:1057500088740846807BF021884353498873084643
:10576000807B0009000188730846007DF021884392
:105770004D4908750846007D000900010875084676
:10578000C07CF02188434849C8740846C07B0009A2
:105790000001C8730846C07C00090001C8740A985B
:1057A00001287DD10A213046F2F7CAFC05463F4860
:1057B000445DE007C00F002807D03B48407B00094C
:1057C0000001C01D3849487305E03748407B000997
:1057D00000013549487302202040002807D0324894
:1057E000007BF021884370302F49087305E02E4874
:1057F000007BF02188432C490873042020400028B6
:1058000007D02948807DF02188437030264988756B
:1058100005E02548807DF0218843234988750820CC
:105820002040002807D02048807D00090001C01DCD
:105830001D49887505E01C48807D000900011A4952
:10584000887510202040002807D01748407DF0219F
:10585000884370301449487505E01348407DF021B5
:1058600088431149487520202040002807D00E4861
:10587000407BF021884370300B49487305E00A48AB
:10588000407BF0218843084948734020204000288D
:105890000ED00548C07D00090001C01D024900E08E
:1058A00092E0C8750AE000006C220020D4ED0100EF
:1058B0006D48C07D000900016B49C8750A2130465A
:1058C000F2F73EFC0D466948445DE007C00F002832
:1058D00007D06548C07AF021884370306249C872A9
:1058E00005E06148C07AF02188435F49C872022010
:1058F0002040002807D05C48C07A00090001C01D84
:105900005949C87205E05848C07A00090001564953
:10591000C87204202040002807D05348407E000968
:105920000001C01D5049487605E04F48407E0009FF
:1059300000014D49487608202040002807D04A48F9
:10594000007EF021884370304749087605E04648DC
:10595000007EF0218843444908761020204000282A
:1059600007D04148007E00090001C01D3E4908766D
:1059700005E03D48007E000900013B4908762020F3
:105980002040002807D03848007B00090001C01DD6
:105990003549087305E03448007B000900013249AD
:1059A000087340202040002807D02F48C07DF021F8
:1059B000884370302C49C87554E02B48C07DF021D5
:1059C00088432949C8754DE02748407B00090001FC
:1059D000254948730846007BF02188432249087313
:1059E0000846807DF02188431F4988750846807DE0
:1059F0000009000188750846407DF02188431A4956
:105A000048750846407BF02188431749487308468B
:105A1000C07D00090001C8750846C07AF02188439E
:105A20001149C8720846C07A00090001C8720846C8
:105A3000407E0009000148760846007EF021884338
:105A4000094908760846007E0009000108760846E4
:105A5000007B0009000108730846C07DF0218843DF
:105A60000149C87505B0F0BD6C220020D4ED0100DD
:105A7000FFB581B00E461746019801287ED10498E3
:105A8000002828D1FB480078012824D0F6F7E8FE4A
:105A9000F94988421FD3FAF7E9FE00280DD0F748EC
:105AA000807DF02188437030F44988750846C07CB9
:105AB00000090001C01DC8741AE0F048807DF02183
:105AC00088431030ED4988750846C07C0009000104
:105AD000401CC8740CE0E948807DF0218843703098
:105AE000E64988750846C07C00090001C01DC874DD
:105AF000E248C07CF02188437030E049C874084611
:105B0000007EF02188437030DC4908760846807DAD
:105B100000090001401C88750846407DF02188433B
:105B20001030D64948750846407D00090001401CE8
:105B300048750846007DF02188431030CF4908752C
:105B40000846007D00090001401C0875330008F07C
:105B5000CBF9062E261E140C042FC848007D000920
:105B60000001C01DC549087500BFC448007DF02173
:105B700088437030C149087500BF00E0AFE1BF48FD
:105B8000407D00090001C01DBC49487500BFBB48ED
:105B9000407DF02188437030B849487500BFB74850
:105BA000807D00090001C01DB449887500BF00E078
:105BB00000BF00BF049800285ED1AE4800780128DD
:105BC0005AD0F6F74DFEAC49884255D3AB48C07F5A
:105BD000F0218843A949C8770846807F0009000161
:105BE00088770846407FF0218843A44948770846D3
:105BF000007FF0218843A14908770846C07DF02145
:105C000088439E49C8750846C07F00090001C877CF
:105C10000846807FF0218843984988770846407F6E
:105C200000090001C01D48770846807EF0218843A6
:105C3000924988760846807E0009000188760846E9
:105C4000407E0009000148760846007E00090001F8
:105C500008760846007F0009000108770846C07EE4
:105C6000F02188438549C8760846407EF021884364
:105C7000703082494876B8E164213846F2F760FA1C
:105C80000546012D07D17D48C07FF0218843703043
:105C90007A49C87705E07948C07FF0218843774981
:105CA000C8770A213846F2F74BFA0A210090F2F73A
:105CB00047FA0D46642F02D37148445D01E07148F4
:105CC000445DE007C00F002807D06C48807F0009C2
:105CD0000001C01D6949887705E06848807F000998
:105CE00000016649887702202040002807D06348D9
:105CF000407FF021884370306049487705E05F4875
:105D0000407FF02188435D494877042020400028E7
:105D100007D05A48007FF0218843703057490877F0
:105D200005E05648007FF021884354490877082051
:105D30002040002807D05148C07DF02188437030B2
:105D40004E49C87505E04D48C07DF02188434B4958
:105D5000C87510202040002807D04848C07F00099F
:105D60000001C01D4549C87705E04448C07F0009CF
:105D700000014249C87720202040002807D03F4832
:105D8000807FF021884370303C49887705E03B48AC
:105D9000807FF021884339498877402020400028BF
:105DA00007D03648407F00090001C01D33494877BD
:105DB00005E03248407F00090001304948770A2158
:105DC0003846F2F7BDF90D462D48445DE007C00F97
:105DD000002807D02948807EF02188437030274969
:105DE000887605E02548807EF0218843234988761F
:105DF00002202040002807D02048807E00090001B2
:105E0000C01D1E49887605E01C48807E00090001FF
:105E10001A49887604202040002807D01748407E81
:105E200000090001C01D1549487605E01348407E71
:105E3000000900011149487608202040002807D0B9
:105E40000E48007E00090001C01D0C49087605E0DF
:105E50000A48007E00090001084908761020204009
:105E6000002811D00548007F00090001C01D03492A
:105E700008770FE0F9000020B80B00004023002055
:105E8000D4ED0100E7ED01005948007F0009000151
:105E90005749087720202040002807D05448C07E6A
:105EA000F021884370305249C87605E05048C07EE2
:105EB000F02188434E49C87640202040002807D072
:105EC0004B48407EF02188437030494948768CE049
:105ED0004748407EF02188434549487685E044485C
:105EE000807D00090001424988750846407DF02107
:105EF00088433F4948750846407D000900014875C0
:105F00000846007DF0218843394908750846007D20
:105F10000009000108750846C07C00090001C8742A
:105F20000846807DF0218843314988750846C07C49
:105F3000F02188432E49C8740846007EF02188432A
:105F40002B4908760846C07FF02188432849C87746
:105F50000846807F0009000188770846407FF021CD
:105F60008843234948770846007FF0218843204929
:105F700008770846C07DF02188431D49C87508464A
:105F8000C07F00090001C8770846807FF021884360
:105F9000174988770846407F00090001487708467E
:105FA000807EF0218843124988760846807E000969
:105FB000000188760846407E0009000148760846C0
:105FC000007E0009000108760846007F00090001F4
:105FD00008770846C07EF02188430549C876084600
:105FE000407EF02188430249487605B0F0BD0000AC
:105FF0004023002010B50146002200200A0EFE4B6F
:10600000985CC307DB0F002B07D0FC4BDB7FF02431
:10601000A3437033F94CE37705E0F84BDB7FF024C2
:10602000A343F64CE37702230340002B07D0F34B46
:10603000DB7F1B091B01DB1DF04CE37705E0EF4B19
:10604000DB7F1B091B01ED4CE37704230340002B8E
:1060500007D0EA4B9B7F1B091B01DB1DE74CA37795
:1060600005E0E64B9B7F1B091B01E44CA37708234B
:106070000340002B09D0E14B20335B781B091B0147
:10608000DB1DDE4C2034637007E0DC4B20335B7893
:106090001B091B01D94C2034637010230340002BD3
:1060A00009D0D64B20331B78F024A3437033D34C54
:1060B0002034237007E0D14B20331B78F024A34316
:1060C000CE4C2034237020230340002B09D0CB4B2F
:1060D00020331B781B091B01DB1DC84C20342370A7
:1060E00007E0C64B20331B781B091B01C34C20342F
:1060F000237040230340002B07D0C04B9B7FF0242C
:10610000A3437033BD4CA37705E0BC4B9B7FF024C9
:10611000A343BA4CA377FF231B040B401A0CB64BC6
:10612000985CC307DB0F002B07D0B44B1B7F1B0908
:106130001B01DB1DB14C237705E0B04B1B7F1B0916
:106140001B01AE4C237702230340002B07D0AB4B3F
:10615000DB7EF024A3437033A84CE37605E0A74B25
:10616000DB7EF024A343A54CE37604230340002BFD
:1061700007D0A24B9B7EF024A34370339F4CA376A1
:1061800005E09E4B9B7EF024A3439C4CA376082302
:106190000340002B07D0994B5B7FF024A34370335F
:1061A000964C637705E0954B5B7FF024A343934CBB
:1061B000637710230340002B07D0904B5B7F1B09B4
:1061C0001B01DB1D8D4C637705E08C4B5B7F1B094E
:1061D0001B018A4C637720230340002B07D0874B99
:1061E0001B7FF024A3437033844C237705E0834B5B
:1061F0001B7FF024A343814C237740230340002BD3
:1062000007D07E4BDB7E1B091B01DB1D7B4CE3763D
:1062100005E07A4BDB7E1B091B01784CE376FF23FC
:106220001B020B401A0A744B985CC307DB0F002B50
:1062300007D0724B1B7EF024A34370336F4C237640
:1062400005E06E4B1B7EF024A3436C4C23760223A7
:106250000340002B07D0694B1B7E1B091B01DB1D74
:10626000664C237605E0654B1B7E1B091B01634CC6
:10627000237604230340002B07D0604BDB7D1B09F2
:106280001B01DB1D5D4CE37505E05C4BDB7D1B09F1
:106290001B015A4CE37508230340002B07D0574BD2
:1062A0009B7E1B091B01DB1D544CA37605E0534B61
:1062B0009B7E1B091B01514CA37610230340002B2E
:1062C00007D04E4B5B7EF024A34370334B4C637678
:1062D00005E04A4B5B7EF024A343484C63762023C1
:1062E0000340002B07D0454B5B7E1B091B01DB1DC8
:1062F000424C637605E0414B5B7E1B091B013F4C22
:10630000637640230340002B07D03C4BDB7DF02419
:10631000A3437033394CE37505E0384BDB7DF02443
:10632000A343364CE375CAB2334B985CC307DB0F0B
:10633000002B07D0314B1B7DF024A34370332F4C2F
:10634000237505E02D4B1B7DF024A3432B4C2375B7
:1063500002230340002B07D0284B1B7D1B091B0188
:10636000DB1D264C237505E0244B1B7D1B091B01FF
:10637000224C237504230340002B07D01F4BDB7CEA
:106380001B091B01DB1D1D4CE37405E01B4BDB7C73
:106390001B091B01194CE37408230340002B07D091
:1063A000164B9B7CF024A3437033144CA37405E07C
:1063B000124B9B7CF024A343104CA3741023034086
:1063C000002B07D00D4B5B7DF024A34370330B4CA7
:1063D000637505E0094B5B7DF024A343074C6375AF
:1063E00020230340002B0BD0044B5B7D1B091B01BA
:1063F000DB1D024C637509E0D4ED01002023002071
:106400000C4B5B7D1B091B010A4C63754023034049
:10641000002B07D0074BDB7CF024A3437033054CE3
:10642000E37405E0034BDB7CF024A343014CE374ED
:1064300010BD00002023002000B501287ED1FE4AB7
:10644000D278F0239A437032FB4BDA701A461279F5
:1064500012091201D21D1A711A461279F0239A43B9
:106460007032F54B1A711A46527912091201D21D77
:106470005A711A465279F0239A437032EE4B5A7190
:106480001A46D27912091201D21DDA711A46D2794E
:10649000F0239A437032E84BDA711A46527A1209A5
:1064A0001201D21D5A721A46527AF0239A43703260
:1064B000E14B5A721A46927AF0239A437032DE4BBD
:1064C0009A721A469278F0239A437032DA4B9A7095
:1064D0001A46D27A12091201D21DDA721A4652787D
:1064E00012091201D21D5A701A46D27AF0239A4329
:1064F0007032D14BDA721A46203AD27FF0239A4397
:106500007032CD4B203BDA77CB4A127B1209120155
:10651000D21D20331A731A46203A927F12091201B3
:10652000D21D203B9A77C44A127BF0239A437032E3
:10653000C14B1A731A46203A127F00E0F2E1F023B1
:106540009A437032BC4B203B1A77BB4A527B1209EC
:106550001201D21D20335A731A46203AD27E1209F4
:106560001201D21D203BDA76B44AD278F0239A4346
:106570007032B24BDA701A46127B12091201D21D28
:106580001A731A46127912091201D21D1A711A468B
:10659000927AF0239A437032A84B9A721A46127973
:1065A000F0239A437032A54B1A711A465279120998
:1065B0001201D21D5A711A46927912091201D21D86
:1065C0009A711A46127A12091201D21D1A721A46CB
:1065D000127AF0239A437032984B1A721A46527A02
:1065E00012091201D21D5A72934A927912091201AC
:1065F000521C914B9A711A469279F0239A431032A9
:106600008D4B9A711A46127A12091201521C1A7293
:106610001A46127AF0239A431032874B1A721A469E
:10662000927A12091201521C9A721A46D2781209F1
:106630001201521CDA701A46927812091201521C89
:106640009A701A465278F0239A4310327A4B5A7055
:106650001A461278F0239A431032774B1A701A4672
:10666000127812091201521C1A701A46203AD27F6F
:1066700012091201521C203BDA771A46927FF0234E
:106680009A4310326C4B203B9A771A46527FF02384
:106690009A431032684B203B5A771A46527F1209B0
:1066A0001201521C5A771A46127F12091201521C0B
:1066B0001A771A46D27EF0239A4310325E4B203B63
:1066C000DA761A46927EF0239A4310325A4B203BD8
:1066D0009A765A4A127BF0239A431032574B1A7318
:1066E0001A46D27AF0239A431032544BDA721A4681
:1066F000D27A12091201521CDA721A46927A1209DF
:106700001201521C9A721A46527AF0239A4310329E
:106710004A4B5A721A465279F0239A431032474B29
:106720005A711A46D279F0239A431032434BDA71E8
:106730000B0007F0D9FB19F3E9DFD5CBC1B7ADA347
:10674000998F87786E645A50463E362E261E160E56
:10675000F5003A4AD279F0239A437032374BDA7116
:1067600000BF364A5279F0239A437032334B5A7144
:1067700000BF324A527AF0239A4370322F4B5A723A
:1067800000BF2E4A927A12091201D21D2B4B9A7227
:1067900000BF2A4AD27A12091201D21D274BDA729F
:1067A00000BF264AD27AF0239A437032234BDA7222
:1067B00000BF224A127BF0239A4370321F4B1A7398
:1067C00000BF1D4A203A927EF0239A4370321A4B42
:1067D000203B9A7600BF184A203AD27EF0239A4393
:1067E0007032154B203BDA7600BF134A203A127FF5
:1067F00012091201D21D104B203B1A7700BF0E4A1E
:10680000203A527F12091201D21D0B4B203B5A77BE
:1068100000BF094A203A527FF0239A437032064B58
:10682000203B5A7700BF044A203A927FF0239A43D4
:106830007032014B203B03E08C22002060230020BB
:106840009A7700BFDC4AD27F12091201D21DDA4BBF
:10685000DA7700BFD84A2032127812091201D21D0D
:10686000D54B20331A7000BFD34A20321278F02360
:106870009A437032D04B20331A7000BFCE4A203278
:106880005278F0239A437032CB4B20335A7000BFBA
:10689000C94A2032927812091201D21DC64B203308
:1068A0009A7000BFC44A2032D27812091201D21D58
:1068B000C14B2033DA7000BFBF4A2032927A1209EE
:1068C0001201D21DBC4B20339A7200BFBA4A20324B
:1068D000127AF0239A437032B74B20331A7200BFFA
:1068E000B54A2032127A12091201D21DB24B20335E
:1068F0001A7200BFB04A20329279F0239A43703264
:10690000AD4B20339A7100BFAB4A20329279120905
:106910001201D21DA84B20339A7100BF01E0FFE79E
:1069200000BF47E1A44A2032D278F0239A43A24B19
:106930002033DA701A461279120912011A711A46B6
:106940001279F0239A439C4B20331A711A465279DC
:10695000120912015A711A465279F0239A43964B42
:1069600020335A711A46D27912091201DA711A4685
:10697000D279F0239A43904B2033DA711A46527A37
:10698000120912015A721A46527AF0239A438A4B1C
:1069900020335A721A46927AF0239A43864B203358
:1069A0009A721A469278F0239A43834B20339A7056
:1069B0001A46D27A12091201DA721A46527812096C
:1069C00012015A701A46D27AF0239A437A4B203336
:1069D000DA72794AD27FF0239A43774BDA771A46F4
:1069E0002032127B1209120120331A73724A927FED
:1069F00012091201203B9A771A462032127BF023AB
:106A00009A436D4B20331A736B4A127FF0239A43DB
:106A1000694B1A771A462032527B12091201203331
:106A20005A73654AD27E12091201203BDA76634A14
:106A3000D278F0239A43614BDA701A46127B12091E
:106A400012011A731A461279120912011A711A46A2
:106A5000927AF0239A43594B9A721A461279F0238C
:106A60009A43564B1A711A465279120912015A71F9
:106A70001A469279120912019A711A46127A12096B
:106A800012011A721A46127AF0239A434B4B1A7269
:106A90001A46527A120912015A72474A20329279E2
:106AA00012091201444B20339A711A469279F0234D
:106AB0009A43414B20339A711A46127A12091201F5
:106AC0001A721A46127AF0239A433B4B20331A72F9
:106AD0001A46927A120912019A721A46D27812094B
:106AE0001201DA701A469278120912019A701A4647
:106AF0005278F0239A43304B20335A701A4612785A
:106B0000F0239A432C4B20331A701A46127812093C
:106B100012011A70284AD27F12091201203BDA773B
:106B20001A46927FF0239A43234B9A771A46527F54
:106B3000F0239A43204B5A771A46527F12091201CA
:106B40005A771A46127F120912011A771A46D27E14
:106B5000F0239A43184BDA761A46927EF0239A4332
:106B6000154B9A76154A127BF0239A43134B1A73EE
:106B70001A46D27AF0239A43104BDA721A46D27A26
:106B800012091201DA721A46927A120912019A72E5
:106B90001A46527AF0239A43084B5A721A4652798F
:106BA000F0239A43054B5A711A46D279F0239A433F
:106BB000024BDA7100BD00006C220020602300202F
:106BC00070B505460C46012D7ED1B348407D0009C5
:106BD0000001C01DB04948750846007DF02188437A
:106BE0001030AD4908750846007D00090001401CC1
:106BF00008750846C07CF02188431030A649C87447
:106C00000846807CF02188431030A34988740846E8
:106C1000807C00090001401C8874F9F763FE02289B
:106C200003D0F9F75FFE01286ED19C480078012857
:106C30006AD0F5F715FE9A49884265D3F9F716FE32
:106C400000282FD09448007DF0218843703092496D
:106C500008750846007D00090001C01D087508463A
:106C6000C07CF021884370308B49C8740846807C12
:106C7000F02188437030884988740846807C000978
:106C80000001C01D88740846407DF02188437030A3
:106C9000814948750846407CF021884370307E4920
:106CA0004874F8E07C48007DF021884310307A4930
:106CB00008750846007D00090001401C087508465B
:106CC000C07CF021884300E0B8E010307249C874FD
:106CD0000846807CF021884310306F49887408464C
:106CE000807C00090001401C88740846407DF0212A
:106CF00088431030684948750846407CF021884335
:106D0000103065494874C6E0F9F726FD002826D101
:106D1000F5F7A6FD6249884221D3F9F7A7FD0028BF
:106D20000ED05D48407DF021884370305A49487547
:106D30000846407CF02188437030574948741CE075
:106D40005548407DF0218843103053494875084626
:106D5000407CF021884310304F4948740DE04E4884
:106D6000407DF021884370304B4948750846407C8F
:106D7000F0218843703048494874F9F7EDFC012848
:106D80002AD146480078012826D0F5F769FD444904
:106D9000884221D34048407DF021884370303E49ED
:106DA00048750846407CF021884370303A49487461
:106DB000F9F75CFD002807D03748007DF0218843B3
:106DC00070303549087566E03348007DF02188430E
:106DD0001030314908755EE0230007F085F8062C75
:106DE000241C140C042D2C48807C00090001C01DBB
:106DF0002949887400BF2848807CF021884370307E
:106E00002549887400BF2448C07CF0218843703035
:106E10002149C87400BF2048007D00090001C01D41
:106E20001D49087500BF1C48007DF0218843703063
:106E30001949087500BF00E000BF2CE01648407DEE
:106E4000F0218843144948750846007DF0218843A5
:106E5000114908750846007D0009000108750846BB
:106E6000C07CF02188430C49C8740846807CF0211E
:106E70008843094988740846807C000900018874A9
:106E80000846407D0009000148750846407CF02115
:106E900088430149487470BD8C220020F90000200D
:106EA000B80B000030B50246002901D1002000E0F7
:106EB0000720130007F018F80F09141F2B37435051
:106EC0005D67727C88929FA9B500574B5B7EF0246A
:106ED000A3430401F0252C402343534C6376A1E0E7
:106EE000524B9B79F024A3430401F0252C4023430B
:106EF0004E4CA37196E04D4B2033DB791B091B01EF
:106F00000407240F2343494C2034E3718AE0464BA5
:106F10002033DB7C1B091B010407240F2343424C55
:106F20002034E3747EE0404B40331B781B091B0187
:106F30000407240F23433C4C4034237072E03A4B47
:106F40002033DB7FF024A3430401F0252C402343AE
:106F5000354C2034E37765E0334B20335B7BF02402
:106F6000A3430401F0252C4023432F4C20346373AA
:106F700058E02E4B9B791B091B010407240F234368
:106F80002A4CA3714EE0294B9B7CF024A3430401BF
:106F9000F0252C402343254CA37443E0234BDB7E98
:106FA0001B091B010407240F2343204CE37639E01F
:106FB0001D4B2033DB7F1B091B010407240F2343D8
:106FC000194C2034E3772DE0174B9B7E1B091B01E6
:106FD0000407240F2343144CA37623E0134B2033E0
:106FE0009B79F024A3430401F0252C4023430F4C4C
:106FF0002034A37116E00D4BDB7D1B091B01040738
:10700000240F2343094CE3750CE0074B20335B7CD2
:107010001B091B010407240F2343034C2034637412
:1070200000E000BF00BF30BD6C22002040230020E4
:10703000F7B582B00746154600260024FE480078C2
:10704000012804D0F5F70CFCFC49884279D2FC48B1
:10705000407CF02188437030F94948740846807CB0
:1070600000090001C01D88740846007D0009000168
:10707000C01D08750846007DF02188437030F04936
:1070800008750846807CF02188437030EC4988748C
:107090000846C07C00090001C01DC8740846C07CB9
:1070A000F02188437030E649C8740846407C0009E6
:1070B0000001C01D48740846407D00090001C01D44
:1070C00048750846407DF02188437030DC4948759A
:1070D0000846007CF02188437030D949087408467E
:1070E000007C00090001C01D08740846C07BF02127
:1070F00088437030D249C873BA220A210020FBF7B6
:107100001DFFBA2213210020FBF718FFBA2211211C
:107110000020FBF713FFBA2212210020FBF70EFF1D
:10712000BA220E210020FBF709FFBA220F2100200E
:10713000FBF704FFBA2210210020FBF7FFFEFDE35E
:10714000FFE70398801E0F2878D243007B449B887A
:107150005B009F440E007400D9003F01AC01100297
:1071600073007402730073007300DA023D0373004E
:10717000A303B348407CF0218843B14948740846D2
:10718000807C0009000188740846007D0009000128
:10719000C01D08750846007DF02188437030A8495D
:1071A00008750846807CF0218843A5498874084604
:1071B000C07C00090001C01DC8740846C07CF021D5
:1071C00088439F49C8740846407C00090001487400
:1071D0000846407D0009000148750846407DF021C1
:1071E0008843974948750846007CF02188439449B4
:1071F00008740846007C0009000108740846C07B3A
:10720000F02188438E49C873BA220A210020FBF777
:1072100095FEBA2213210020FBF790FE00220E21DA
:107220001046FBF78BFE00220F211046FBF786FE6F
:10723000002210211046FBF781FEF6E393E380481D
:10724000407CF02188437E4948740846807C0009D0
:10725000000188740846007D00090001C01D087502
:107260000846007DF021884370307549087508464E
:10727000807CF0218843724988740846C07C0009EC
:107280000001C8740846C07CF02188436C49C8746A
:107290000846407C0009000148740846407D00090A
:1072A0000001C01D48750846407DF02188436449AF
:1072B00048750846007CF0218843614908740846F7
:1072C000007C0009000108740846C07BF021884357
:1072D0005B49C873BA220A210020FBF72FFEBA22AD
:1072E00013210020FBF72AFE00220E211046FBF797
:1072F00025FE00220F211046FBF720FE0022102160
:107300001046FBF71BFE90E34D48407CF02188437C
:107310004B4948740846807C00090001C01D8874F0
:107320000846007D00090001C01D08750846007D63
:10733000F02188437030424908750846807CF0216E
:10734000884370303E4988740846C07C00090001BB
:10735000C8740846C07CF02188433949C87408467F
:10736000407C0009000148740846407D0009000186
:1073700048750846407DF0218843314948750846E4
:10738000007CF02188432E4908740846007C0009DF
:10739000000108740846C07BF02188432849C8735F
:1073A000BA220A210020FBF7C9FDBA2213210020CE
:1073B000FBF7C4FD00220E211046FBF7BFFD0022A3
:1073C0000F211046FBF7BAFD002210211046FBF7F3
:1073D000B5FD2AE31A48407CF021884318494874D7
:1073E0000846807C00090001C01D88740846007DA5
:1073F00000090001C01D08750846007DF021884382
:1074000070300F4908750846807CF02188430C498C
:1074100088740846C07C00090001C8740846C07C16
:10742000F02188430649C8740846407C00090001E1
:10743000C01D4874084605E0F9000020B80B0000A4
:10744000AC220020407D0009000148750846407DBF
:10745000F0218843FE4948750846007CF0218843A6
:10746000FB4908740846007C0009000108740846BE
:10747000C07BF0218843F649C873BA220A21002054
:10748000FBF75CFDBA2213210020FBF757FD002219
:107490000E211046FBF752FD00220F211046FBF78C
:1074A0004DFD002210211046FBF748FDBDE2E848E3
:1074B000407CF0218843E64948740846807C0009F6
:1074C000000188740846007D00090001087508461F
:1074D000007DF02188437030DD4908750846807CC6
:1074E000F0218843DA4988740846C07C000900010D
:1074F000C8740846C07CF02188437030D449C874F1
:107500000846407C0009000148740846407D000997
:10751000000148750846407DF0218843CC494875F4
:107520000846007CF0218843C94908740846007C5D
:107530000009000108740846C07BF0218843C44953
:10754000C873BA220A210020FBF7F8FCBA221321E3
:107550000020FBF7F3FC00220E211046FBF7EEFCA7
:1075600000220F211046FBF7E9FC002210211046F3
:10757000FBF7E4FC59E2B648407CF0218843B4496B
:1075800048740846807C0009000188740846007D24
:107590000009000108750846007DF021884370301D
:1075A000AB4908750846807CF0218843A849887457
:1075B0000846C07C00090001C8740846C07CF02160
:1075C0008843A349C8740846407C000900014874F8
:1075D0000846407D0009000148750846407DF021BD
:1075E000884370309A4948750846007CF0218843EA
:1075F000974908740846007C000900010874084691
:10760000C07BF02188439249C873BA220A21002026
:10761000FBF794FCBA2213210020FBF78FFC002219
:107620000E211046FBF78AFC00220F211046FBF7C3
:1076300085FC002210211046FBF780FCF5E1844810
:10764000407CF02188437030814948740846807C32
:1076500000090001C01D88740846007D0009000172
:10766000C01D08750846007DF021884370307849B8
:1076700008750846807CF02188437549887408465F
:10768000C07C00090001C8740846C07CF021884312
:107690006F49C8740846407C0009000148740846D8
:1076A000407D0009000148750846407DF02188436F
:1076B000674948750846007CF0218843644908748E
:1076C0000846007C0009000108740846C07BF021D0
:1076D00088435F49C873BA220A210020FBF72EFCB9
:1076E000BA2213210020FBF729FC00220E211046AC
:1076F000FBF724FC00220F211046FBF71FFC0022A1
:1077000010211046FBF71AFC8FE15148407CF02114
:1077100088434F4948740846807C000900018874FA
:107720000846007D0009000108750846007DF0212B
:107730008843474908750846807CF02188434449BE
:1077400088740846C07C00090001C8740846C07CE3
:10775000F02188433E49C8740846407C0009000176
:1077600048740846407D0009000148750846407D80
:10777000F0218843364948750846007CF02188434B
:10778000334908740846007C000900010874084663
:10779000C07BF021884370302D49C87300220A2134
:1077A0001046FBF7CBFB002213211046FBF7C6FB6C
:1077B000BA220E210020FBF7C1FB00220F21104648
:1077C000FBF7BCFB002210211046FBF7B7FB2CE1B6
:1077D0001F48407CF02188431D4948740846807C3E
:1077E0000009000188740846007D00090001087541
:1077F0000846007DF0218843154908750846807CBD
:10780000F0218843124988740846C07C00090001B1
:10781000C8740846C07CF02188430D49C8740846E6
:10782000407C0009000148740846407D00090001C1
:1078300048750846407DF02188430549487508464B
:10784000007CF0218843024908740846007C01E06E
:10785000AC22002000090001C01D08740846C07B4E
:10786000F0218843F949C87300220A211046FBF72A
:1078700065FB002213211046FBF760FB00220E215E
:107880001046FBF75BFBBA220F210020FBF756FBEB
:10789000002210211046FBF751FBC6E0EB48407C6C
:1078A000F0218843E94948740846807C00090001BA
:1078B00088740846007D0009000108750846007DAF
:1078C000F0218843E14908750846807CF02188430F
:1078D000DE4988740846C07C00090001C874084667
:1078E000C07CF0218843D949C8740846407C00090F
:1078F000000148740846407D0009000148750846AB
:10790000407DF0218843D14948750846007CF0212C
:1079100088437030CD4908740846007C0009000196
:1079200008740846C07BF0218843C849C873002208
:107930000A211046FBF702FB002200E076E013214B
:107940001046FBF7FBFA00220E211046FBF7F6FA71
:1079500000220F211046FBF7F1FABA221021002075
:10796000FBF7ECFA61E0B948407CF0218843B74965
:1079700048740846807C0009000188740846007D30
:107980000009000108750846007DF0218843AF49D1
:1079900008750846807CF0218843AC498874084605
:1079A000C07C00090001C8740846C07CF0218843EF
:1079B000A649C8740846407C00090001487408467E
:1079C000407D0009000148750846407DF02188434C
:1079D0009E4948750846007CF02188439B490874FD
:1079E0000846007C0009000108740846C07BF021AD
:1079F00088439649C87300220A211046FBF79EFA75
:107A0000002213211046FBF799FA00220E2110469E
:107A1000FBF794FA00220F211046FBF78FFA0022A1
:107A200010211046FBF78AFA00BF00BF002F76D066
:107A3000BA2211210020FBF781FABA22122100207C
:107A4000FBF77CFA82480078012804D0F4F708FF9D
:107A50008049884216D28048807BF021884370306C
:107A60007D498873084640300078F02188437030A3
:107A70007949403108700846007800090001C01DAE
:107A800008702DE07D20C000854214D27248807BB2
:107A9000F021884370498873084640300078F0210F
:107AA000884370306C4940310870084600780009FE
:107AB0000001087014E06848807BF0218843703032
:107AC00065498873084640300078F0218843624950
:107AD000403108700846007800090001C01D087098
:107AE0007D20C000854205D201462846F0F728FBDC
:107AF000064604E059492846F0F722FB0646584856
:107B0000845DE007C00F00280AD053484030C07899
:107B100000090001C01D50494031C87008E0A6E2CC
:107B20004D484030C078000900014B494031C870D1
:107B300002202040002807D04748C07900090001F2
:107B4000C01D4549C87105E04348C07900090001DE
:107B50004149C87104202040002807D03E48807960
:107B600000090001C01D3C49887105E03A48807950
:107B7000000900013849887108202040002807D0FA
:107B800035484079F021884370303349487105E029
:107B900031484079F02188432F4948711020204016
:107BA000002807D02C48407900090001C01D2A494F
:107BB000487105E0284840790009000126494871CC
:107BC00020202040002807D023480079F021884356
:107BD00070302149087105E01F480079F021884381
:107BE0001D49087140202040002807D01A4880799C
:107BF000F021884370301849887105E01648807973
:107C0000F0218843144988717D20C000854207D245
:107C100064212846F0F794FA06461148845D27E06F
:107C200064212846F0F78CFA7D21C9000090F0F716
:107C300087FA019164210198F0F782FA0646094813
:107C4000854213D30848845D12E00000AC22002076
:107C5000F9000020B80B000020230020A0860100BE
:107C6000E7ED010010270000D4ED0100F948845D24
:107C7000E007C00F002807D0F7488078F02188433C
:107C80007030F549887005E0F3488078F02188432A
:107C9000F149887002202040002809D0EE48403881
:107CA000807A00090001C01DEB494039887207E065
:107CB000E9484038807A00090001E7494039887274
:107CC00004202040002809D0E3484038407A0009C9
:107CD0000001C01DE0494039487207E0DE484038E5
:107CE000407A00090001DC494039487208202040F0
:107CF000002809D0D8484038007AF02188437030F5
:107D0000D5494039087207E0D3484038007AF0215D
:107D10008843D1494039087210202040002809D0FA
:107D2000CD484038007A00090001C01DCA494039D9
:107D3000087207E0C8484038007A00090001C649C7
:107D40004039087220202040002809D0C24840381D
:107D5000C079F02188437030BF494039C87107E0CD
:107D6000BD484038C079F0218843BB494039C871CB
:107D700040202040002809D0B7484038407AF02100
:107D800088437030B4494039487207E0B2484038FF
:107D9000407AF0218843B049403948727D20C000C4
:107DA000854210D20A212846F0F7CAF90A2101902B
:107DB000F0F7C6F90E460A2D02D3A848845D11E0FB
:107DC000A448845D0EE064212846F0F7B9F90A2141
:107DD0000090F0F7B5F90A210190F0F7B1F90E46DD
:107DE0009E498C5DE007C00F002807D09A48807834
:107DF00000090001C01D9849887005E09648807808
:107E0000000900019449887002202040002809D010
:107E100091484038807B00090001C01D8E494039DF
:107E2000887307E08C484038807B000900018A494C
:107E30004039887304202040002809D08648403803
:107E4000407B00090001C01D83494039487307E0A9
:107E500081484038407B000900017F494039487320
:107E600008202040002809D07B484038007BF021C2
:107E70008843703078494039087307E076484038C5
:107E8000007BF0218843744940390873102020405A
:107E9000002809D070484038C07A00090001C01D90
:107EA0006D494039C87207E06B484038C07A000914
:107EB000000169494039C87220202040002809D0BB
:107EC00065484038807AF0218843703062494039F3
:107ED000887207E060484038807AF02188435E4924
:107EE0004039887240202040002809D05A48403844
:107EF000407BF0218843703057494039487307E090
:107F000055484038407BF0218843534940394873F5
:107F10007D20C000854207D20A212846F0F710F9DB
:107F20000E464E48845D0AE064212846F0F708F9C1
:107F30000A210190F0F704F90E4648498C5DE007EC
:107F4000C00F002807D044484078F02188437030A3
:107F50004149487005E040484078F02188433E4957
:107F6000487002202040002807D03B484078000994
:107F70000001C01D3849487005E0374840780009C5
:107F800000013549487004202040002809D03248BB
:107F90004038007CF021884370302F494039087404
:107FA00007E02D484038007CF02188432A494039B9
:107FB000087408202040002809D027484038007C59
:107FC00000090001C01D24494039087407E0224817
:107FD0004038007C000900011F4940390874102016
:107FE0002040002809D01C484038C07BF02188433D
:107FF000703019494039C87307E017484038C07BD2
:10800000F021884314494039C873202020400028BB
:1080100009D011484038C07B00090001C01D0E493D
:108020004039C87307E00C484038C07B00090001A4
:1080300009494039C87340202040002810D0064824
:108040004038407C00090001C01D03494039487494
:10805000E8E00000E7ED010060230020D4ED01001E
:108060007148407C000900016F494874DAE0002241
:108070000A211046FAF762FF002213211046FAF790
:108080005DFF002211211046FAF758FF002212214D
:108090001046FAF753FF00220E211046FAF74EFF62
:1080A00000220F211046FAF749FF00221021104646
:1080B000FAF744FF5C484030C078000900015A4993
:1080C0004031C8705848C079000900014039C87172
:1080D0000846807900090001887108464079F0213E
:1080E00088435149487108464079000900014871A8
:1080F00008460079F02188434B4908710846807989
:10810000F021884348498871084640308078F02142
:1081100088434549403188704348807A000900010E
:10812000403988720846407A0009000148720846C2
:10813000007AF02188433C4908720846007A000919
:10814000000108720846C079F02188433649C87199
:108150000846407AF0218843334948720846403047
:10816000807800090001403188702F48807B000929
:108170000001403988730846407B000900014873BC
:108180000846007BF0218843274908730846C07AD7
:1081900000090001C8720846807AF021884322490C
:1081A00088720846407BF02188431F49487308467F
:1081B00040304078F02188431B49403148700846E0
:1081C00040780009000148701748007CF02188437E
:1081D000154908740846007C000900010874084627
:1081E000C07BF02188431049C8730846C07B000952
:1081F0000001C8730846407C000900014874084625
:10820000807BF02188430849887308464030007815
:10821000F02188430449403108700846007800097D
:108220000001087005B0F0BD20230020F7B582B032
:1082300007460E460121FF200830FCF72BFE0121E6
:10824000FC48FCF727FEFC48007801287ED0F4F7B4
:1082500007FBFA49884279D3F8F78AFA032843D111
:10826000F8F780FA002803D0F8F77CFA01283BD110
:10827000002F1CD1F8F7FAFA00280CD0F048407C07
:10828000F0218843EE4948740846807C00090001CB
:10829000C01D8874EEE0EA48407CF0218843E8493C
:1082A00048740846807C000900018874E2E0F8F711
:1082B000DDFA00280CD0E248407CF0218843703081
:1082C000DF4948740846807C000900018874D1E0C9
:1082D000DB48407CF0218843D94948740846807CBB
:1082E000000900018874C5E0F8F73CFA002803D0C3
:1082F000F8F738FA012865D1002F0CD1D048407C1E
:10830000F0218843CE4948740846807C000900016A
:10831000C01D88740BE0CA48407CF021884370304F
:10832000C74948740846807C000900018874F8F742
:1083300019FA002821D1C2482030C078F0218843A2
:108340007030BF492031C870BD4800E064E0807DD6
:1083500000090001203988750846807DF021884396
:10836000B7498875BA2223210020FAF7E7FD0022D9
:1083700022211046FAF7E2FD7CE0F8F7F3F9012834
:1083800078D1AF482030C078F0218843AC49203103
:10839000C870AB48807D00090001C01D2039887578
:1083A0000846807DF02188437030A54988750022F9
:1083B00023211046FAF7C2FDBA2222210020FAF743
:1083C000BDFD57E09E48407CF02188439C4948749D
:1083D0000846807C00090001887408462030C07877
:1083E000F021884396492031C8709548807D000966
:1083F0000001203988750846807DF0218843904926
:108400008875002223211046FAF798FD00222221C8
:108410001046FAF793FD2DE08948407CF02188430F
:108420007030874948740846807C00090001C01DEF
:10843000887408462030C078F02188437030804925
:108440002031C8707E48807D00090001C01D2039A0
:1084500088750846807DF02188437030784988759A
:10846000BA2223210020FAF769FDBA222221002036
:10847000FAF764FDF8F776F9002808D06E4800781E
:10848000012804D0F4F7ECF96C49884276D26D48A3
:10849000864209D96A4820304079F02188437030FB
:1084A00067492031487107E0654820304079F02164
:1084B000884363492031487163493046EFF740FEF5
:1084C0000A210190EFF73CFE0D465E48401C8642B3
:1084D00002D35E48445D01E05D48445DE007C00FA3
:1084E000002809D056482030C07800090001C01D7E
:1084F00053492031C87007E051482030C078000946
:1085000000014F492031C87002202040002809D0C6
:108510004B4820308078F021884370304849203122
:10852000887007E0464820308078F021884344492D
:108530002031887004202040002809D04048203095
:108540004078F021884370303D492031487007E081
:108550003B4820304078F021884339492031487029
:108560000820204000280AD03548203040790009F2
:108570000001C01D32492031487108E0A1E23048B5
:1085800020304079000900012D4920314871102028
:108590002040002809D02A4820300079F021884363
:1085A000703027492031087107E0254820300079D4
:1085B000F0218843224920310871202020400028E2
:1085C00009D01F482030007900090001C01D1C4956
:1085D0002031087107E01A482030007900090001B5
:1085E00017492031087140202040002809D0144844
:1085F0002030807800090001C01D114920318870A9
:1086000007E00F4820308078000900010C49203134
:1086100088707D21C9003046EFF792FD0A21019054
:10862000EFF78EFD0D460848864213D30748445D98
:1086300012E0000005050000F9000020B80B000062
:10864000202300209F86010010270000D4ED0100A8
:10865000E7ED0100F948445DE007C00F002807D0AE
:10866000F748C07FF02188437030F549C87705E0AE
:10867000F348C07FF0218843F149C87702202040A9
:10868000002807D0EE48C07F00090001C01DEC495A
:10869000C87705E0EA48C07F00090001E849C877CB
:1086A00004202040002807D0E548807F0009000111
:1086B000C01DE349887705E0E148807F000900019B
:1086C000DF49887708202040002809D0DC48203086
:1086D000407800090001C01DD9492031487007E0E9
:1086E000D7482030407800090001D5492031487032
:1086F00010202040002809D0D14820300078F021F7
:1087000088437030CE492031087007E0CC482030D3
:108710000078F0218843CA49203108702020204089
:10872000002809D0C6482030007800090001C01D8B
:10873000C3492031087007E0C148203000780009A3
:108740000001BF492031087040202040002807D098
:10875000BB48807FF02188437030B949887705E0B5
:10876000B748807FF0218843B54988776421304637
:10877000EFF7E6FC0A210190EFF7E2FC0D467D20C1
:10878000C000864202D3AF48445D01E0AB48445D7F
:10879000E007C00F002807D0A948007F00090001AA
:1087A000C01DA749087705E0A548007F0009000122
:1087B000A349087702202040002807D0A048C07EA7
:1087C000F021884370309E49C87605E09C48C07E01
:1087D000F02188439A49C87604202040002807D019
:1087E0009748807EF021884370309549887605E06F
:1087F0009348807EF0218843914988760820204064
:10880000002807D08E48407FF021884370308C4983
:10881000487705E08A48407FF021884388494877B7
:1088200010202040002807D08548407F0009000123
:10883000C01D8349487705E08148407F0009000159
:108840007F49487720202040002807D07C48007FBF
:10885000F021884370307A49087705E07848007F36
:10886000F02188437649087740202040002807D02F
:108870007348C07E00090001C01D7149C87605E03B
:108880006F48C07E000900016D49C8760A21304654
:10889000EFF756FC0A210190EFF752FC0D46642ECB
:1088A00002D36848445D01E06448445DE007C00FBE
:1088B000002807D06248007EF0218843703060496C
:1088C000087605E05E48007EF02188435C49087622
:1088D00002202040002807D05948007E00090001EE
:1088E000C01D5749087605E05548007E0009000183
:1088F0005349087604202040002807D05048C07D06
:1089000000090001C01D4E49C87505E04C48C07DF6
:10891000000900014A49C87508202040002807D0F6
:108920004748807E00090001C01D4549887605E062
:108930004348807E0009000141498876102020408C
:10894000002807D03E48407EF021884370303C49E3
:10895000487605E03A48407EF02188433849487619
:1089600020202040002807D03548407E0009000123
:10897000C01D3349487605E03148407E00090001BA
:108980002F49487640202040002807D02C48C07D41
:10899000F021884370302A49C87505E02848C07D19
:1089A000F02188432649C8750A213046EFF7C8FBF5
:1089B0000D462448445DE007C00F002807D020483A
:1089C000007DF021884370301D49087505E01C4882
:1089D000007DF02188431A490875022020400028B4
:1089E00007D01748007D00090001C01D1449087513
:1089F00005E01348007D00090001114908750420B5
:108A00002040002807D00E48C07C00090001C01D8E
:108A10000B49C87405E00A48C07C000900010849F8
:108A2000C8740820204000280ED00548807CF02122
:108A300088437030024988740CE00000E7ED0100C3
:108A400020230020D4ED0100FA48807CF0218843E7
:108A5000F849887410202040002807D0F548407D50
:108A6000F02188437030F349487505E0F148407DB6
:108A7000F0218843EF49487520202040002807D086
:108A8000EC48407D00090001C01DEA49487505E039
:108A9000E848407D00090001E64948754020204033
:108AA000002807D0E348C07CF02188437030E149BA
:108AB000C8746DE2DF48C07CF0218843DD49C8748A
:108AC000F7E7F7F74FFE01287CD1DA4820304079EC
:108AD000F0218843D749203148710846C078000901
:108AE0000001C87008468078F0218843D1492031C0
:108AF000887008464078F0218843CE49203148707C
:108B00000846407900090001487108460079F021C3
:108B10008843C849203108710846007900090001DE
:108B20000871084680780009000188707D21C9001D
:108B30000498EFF705FB0546BF48445DE007C00F0A
:108B4000002807D0BB48C07FF02188437030B94966
:108B5000C87705E0B748C07FF0218843B549C8779A
:108B600002202040002807D0B248C07F0009000141
:108B7000C01DB049C87705E0AE48C07F00090001BC
:108B8000AC49C87704202040002807D0A948807F3E
:108B900000090001C01DA749887705E0A548807F2E
:108BA00000090001A34988770820204000280AD046
:108BB000A0482030407800090001C01D9D492031A7
:108BC000487008E0ECE19B48203040780009000143
:108BD00098492031487010202040002809D095483D
:108BE00020300078F021884370309249203108709D
:108BF00007E0904820300078F02188438D492031EB
:108C0000087020202040002809D08A4820300078B1
:108C100000090001C01D87492031087007E0854820
:108C2000203000780009000182492031087040207E
:108C30002040002807D07F48807FF0218843703093
:108C40007C49887705E07B48807FF021884379491B
:108C5000887764210498EFF773FA0A210190EFF7FF
:108C60006FFA0D467D21C9000498884202D37348EB
:108C7000445D01E07048445DE007C00F002807D064
:108C80006C48007F00090001C01D6A49087705E0B3
:108C90006848007F000900016649087702202040EB
:108CA000002807D06348C07EF021884370306149B6
:108CB000C87605E05F48C07EF02188435D49C876EC
:108CC00004202040002807D05A48807EF0218843A5
:108CD00070305849887605E05648807EF0218843F8
:108CE0005449887608202040002807D05148407F0A
:108CF000F021884370304F49487705E04D48407F68
:108D0000F02188434B49487710202040002807D0A5
:108D10004848407F00090001C01D4649487705E0EA
:108D20004448407F00090001424948772020204004
:108D3000002807D03F48007FF021884370303D492C
:108D4000087705E03B48007FF021884339490877E0
:108D500040202040002807D03648C07E000900018E
:108D6000C01D3449C87605E03248C07E00090001C4
:108D70003049C8760A210498EFF7E2F90A210190F8
:108D8000EFF7DEF90D462D48445DE007C00F0028DF
:108D900007D02848007EF0218843703025490876A6
:108DA00005E02448007EF02188432249087602200D
:108DB0002040002807D01F48007E00090001C01D88
:108DC0001C49087605E01B48007E0009000119498E
:108DD000087604202040002807D01648C07D0009EE
:108DE0000001C01D1349C87505E01248C07D000987
:108DF00000011049C87508202040002807D00D4800
:108E0000807E00090001C01D0A49887605E00948F6
:108E1000807E000900010749887610202040002844
:108E20000ED00448407EF0218843703001494876D6
:108E30000CE0000020230020E7ED0100D4ED01004C
:108E4000FE48407EF0218843FC494876202020409F
:108E5000002807D0F948407E00090001C01DF749ED
:108E6000487605E0F548407E00090001F349487660
:108E700040202040002807D0F048C07DF0218843E2
:108E80007030EE49C87505E0EC48C07DF02188439C
:108E9000EA49C8750A210498EFF752F90D46E848E7
:108EA000445DE007C00F002807D0E448007DF021B2
:108EB00088437030E149087505E0E048007DF02105
:108EC0008843DE49087502202040002807D0DB488F
:108ED000007D00090001C01DD849087505E0D7488C
:108EE000007D00090001D5490875042020400028B4
:108EF00007D0D248C07C00090001C01DCF49C8740A
:108F000005E0CE48C07C00090001CC49C8740820A7
:108F10002040002807D0C948807CF0218843703069
:108F2000C649887405E0C548807CF0218843C34960
:108F3000887410202040002807D0C048407DF021D0
:108F400088437030BD49487505E0BC48407DF0213C
:108F50008843BA49487520202040002807D0B748E8
:108F6000407D00090001C01DB449487505E0B348C3
:108F7000407D00090001B14948754020204000288B
:108F800007D0AE48C07CF02188437030AB49C8742C
:108F90004CE2AA48C07CF0218843A849C87445E245
:108FA000F7F7E0FB02287DD1A44820304079F0217A
:108FB0008843A249203148710021A248F2F7A4F861
:108FC000552830D1A048FDF715F89C482030C078CE
:108FD0000009000199492031C87008468078F021C5
:108FE000884396492031887008464078F0218843AC
:108FF00092492031487008464079000900014871C3
:1090000008460079F02188438C49203108710846D0
:109010000079000900010871084680780009000104
:10902000C01D887002E289480078401C874908709A
:1090300082482030C07800090001C01D7F492031DE
:10904000C87008468078F021884370307B49203111
:10905000887008464078F02188437849203148706C
:109060000846407900090001487108460079F0215E
:109070008843703071492031087108460079000931
:109080000001C01D08710846807800090001C01D5C
:1090900088706F48007800280FD16E48006800285B
:1090A0000BD100E070E0FCF7A5FF002067490870D5
:1090B0006949086069490860B8E164480078642833
:1090C00028DA6748007862490978884204DB6048FA
:1090D0000078401E624908705D4802785D495E482C
:1090E0000068F6F777FA00280FD15D480078800015
:1090F00058490858002808D0594800788000085876
:109100005549086000205149087053480068534988
:10911000086034E04D480078642830DB504800781F
:10912000401C4F4908700846007849490978884230
:1091300002DB00204A490870494800788000454910
:1091400008584549086000204049087042480068B6
:1091500042490968884212D13D480078401E404982
:10916000097888420BDD3E480078401C3C49087075
:109170000846007880003749085837490860364863
:109180000068FCF737FF51E1F7F7ECFA032893D1B9
:109190002A4820304079F0218843284920314871FD
:1091A0000846C07800090001C01DC87008468078D4
:1091B000F021884321492031887008464078F02109
:1091C000884370301D4920314870084640790009B5
:1091D0000001C01D487108460079F02188431749F5
:1091E000203108710846007900090001C01D08718E
:1091F0000846807800090001C01D88700F48C07FB4
:10920000F02188430D49C8770846C07F0009000156
:10921000C8770846807F000900018877084620301B
:109220004078000900012031487008460078F0219C
:109230008843024920310870084613E020230020AB
:10924000D4ED0100200800200B0B0B0B6C0000205C
:109250007E000020B00B0020640000206800002089
:1092600060000020007800090001087008462038DE
:10927000807FF02188436E4988770846007F000987
:109280000001C01D08770846C07EF0218843703079
:109290006749C8760846807EF0218843703064496B
:1092A00088760846407FF0218843703060494877CF
:1092B0000846407F00090001C01D48770846007F2E
:1092C000F021884370305A4908770846C07E00096B
:1092D0000001C876F7F786FA002855D15448007E79
:1092E000F02188437030524908760846007E000914
:1092F000000108760846C07D00090001C8750846CF
:10930000807E0009000188760846407EF02188436F
:109310007030474948760846407E00090001C01D6C
:1093200048760846C07DF021884370304049C875B2
:109330000846007DF021884370303D490875084695
:10934000007D0009000108750846C07C0009000185
:10935000C8740846807CF0218843354988740846E3
:10936000407DF02188437030314948750846407D82
:1093700000090001C01D48750846C07CF0218843E3
:1093800070302B49C87451E02948007EF021884391
:109390007030274908760846007E00090001C01D8C
:1093A00008760846C07D00090001C01DC875084642
:1093B000807E0009000188760846407EF0218843BF
:1093C00070301B4948760846407E00090001C01DE8
:1093D00048760846C07DF02188431549C87508467F
:1093E000007DF0218843124908750846007D000978
:1093F000000108750846C07C00090001C8740846D1
:10940000807CF02188430A4988740846407DF02119
:109410008843074948750846407D000900014875A2
:109420000846C07CF02188430149C87405B0F0BDEE
:1094300020230020F7B582B00D461746002602987B
:1094400001287CD1632D0ADD0121FF200630FBF7C6
:1094500021FD0121FF200730FBF71CFD16E0092D3F
:109460000ADD0121FF200630FBF714FD0021FF205B
:109470000730FBF70FFD09E00021FF200630FBF766
:1094800009FD0021FF200730FBF704FDFA480078B2
:1094900001286ED0F3F7E4F9F849884269D3F7F769
:1094A00067F9032866D1002F30D1F7F7DFF90028DC
:1094B00016D0F348407BF0218843F14948730846B1
:1094C000C07B00090001C01DC873BA22082100201A
:1094D000F9F734FD002209211046F9F72FFD90E03D
:1094E000E748407BF0218843E54948730846C07B44
:1094F00000090001C873002208211046F9F71EFD7B
:10950000002209211046F9F719FD7AE0F7F7AEF9C4
:10951000002818D0DA48407BF02188437030D849C1
:1095200048730846C07B00090001C8730022082167
:109530001046F9F703FDBA220921002000E0ACE152
:10954000F9F7FCFC5DE0CE48407BF0218843CC4934
:1095500048730846C07B00090001C8730022082137
:109560001046F9F7EBFC002209211046F9F7E6FC5A
:1095700047E02FE0002F16D1C148407BF0218843FF
:10958000BF4948730846C07B00090001C01DC8736D
:10959000BA2208210020F9F7D1FC00220921104647
:1095A000F9F7CCFC2DE0B648407BF02188437030C1
:1095B000B34948730846C07B00090001C873002204
:1095C00008211046F9F7BAFCBA2209210020F9F760
:1095D000B5FC16E0AA48407BF02188437030A849CA
:1095E00048730846C07B00090001C01DC873BA2239
:1095F00008210020F9F7A2FCBA2209210020F9F77E
:109600009DFC64212846EEF79BFD0646012E09D1FC
:109610009B482038807B00090001C01D98492039F3
:10962000887307E096482038807B00090001944940
:10963000203988730A212846EEF782FD0A2101901D
:10964000EEF77EFD0E46642D02D38E48845D01E068
:109650008D48845DE007C00F002807D08848407A15
:10966000F021884370308649487205E08448407A8A
:10967000F02188438249487202202040002807D008
:109680007F48407A00090001C01D7D49487205E00D
:109690007B48407A00090001794948720420204043
:1096A000002809D076482038007CF02188437030AB
:1096B00073492039087407E071482038007CF02194
:1096C00088436F492039087408202040002809D0B9
:1096D0006B482038007C00090001C01D6849203912
:1096E000087407E066482038007C000900016449DE
:1096F0002039087410202040002809D06048203804
:10970000C07BF021884370305D492039C87307E081
:109710005B482038C07BF021884359492039C87301
:1097200020202040002809D055482038807BF02197
:109730008843703052492039887307E050482038F8
:10974000807BF02188434E49203988734020204097
:10975000002809D04A482038C07B00090001C01DFC
:1097600047492039C87307E045482038C07B0009C5
:10977000000143492039C8730A212846EEF7E0FC6E
:109780000E464048845DE007C00F002807D03C48E3
:10979000407B00090001C01D3949487305E0384885
:1097A000407B000900013649487302202040002810
:1097B00007D03348007BF02188437030304908736C
:1097C00005E02F48007BF02188432D4908730420D1
:1097D0002040002807D02A48007B00090001C01D56
:1097E0002749087305E02648007B00090001244949
:1097F000087308202040002807D02148C07AF021B3
:10980000884370301E49C87205E01D48C07AF021B7
:1098100088431B49C87210202040002807D01848F0
:10982000C07A00090001C01D1549C87205E014483E
:10983000C07A000900011249C87220202040002887
:1098400007D00F48807A00090001C01D0C498872BA
:1098500005E00B48807A0009000109498872402020
:109860002040002812D00648807AF02188437030CA
:10987000034988727FE00000F9000020B80B000067
:10988000AC220020D4ED0100E7ED01003B48807AD6
:10989000F0218843394988726DE000220821104682
:1098A000F9F74CFB002209211046F9F747FB334832
:1098B000407BF0218843314948730846C07B00094A
:1098C0000001C87308462038807B00090001203958
:1098D00088732A48407AF02188432849487208460C
:1098E000407A00090001487208462038007CF021C7
:1098F00088432249203908740846007C0009000189
:1099000008740846C07BF02188431C492039C8737D
:109910000846807BF021884318492039887308461F
:10992000C07B00090001C8731448407B0009000196
:10993000203148730846007BF02188430F490873A3
:109940000846007B0009000108730846C07AF02130
:1099500088430A49C8720846C07A00090001C872E3
:109960000846807AF0218843044988720846807A44
:1099700000090001887205B0F0BD0000AC22002093
:10998000F8B507460E460025002F7DD0FE48C07969
:1099900000090001C01DFC49C8710846807AF02109
:1099A00088437030F8498872F6F778FD01286CD04A
:1099B000F648007801287DD0F2F752FFF44988423A
:1099C00078D9F148C07AF02188437030EE49C872E6
:1099D0000846007A00090001C01D08720846C07BD5
:1099E000F0218843E849C8730846C07B000900019C
:1099F000C8730846807B0009000188730846407CD4
:109A00000009000148740846007CF0218843DE49C3
:109A100008740846007C0009000108740846807B31
:109A2000F0218843D84988730846007BF021884399
:109A3000D54908730846007B0009000108730846F1
:109A4000C07A00090001C8720846407CF0218843B2
:109A5000CD4948740846407BF0218843CA49487381
:109A60000846407B0009000148730846407A000917
:109A7000000148720846007AF0218843C249087202
:109A80000846C079F02101E0C4E113E08843BE49F3
:109A9000C8710846807C0009000188740846807AF5
:109AA0000009000188720846407AF0218843B649CF
:109AB0004872AFE164213046EEF758FB85B2B348F7
:109AC0000078012804D0F2F7CBFEB149884202D8D1
:109AD000B048445D01E0B048445DE007C00F002895
:109AE00007D0A948C07BF02188437030A649C873CD
:109AF00005E0A548C07BF0218843A349C873022034
:109B00002040002807D0A048C07B00090001C01DEC
:109B10009D49C87305E09C48C07B000900019A4933
:109B2000C87304202040002807D09748807B000994
:109B30000001C01D9449887305E09348807B0009AB
:109B400000019149887308202040002807D08E48E2
:109B5000407C00090001C01D8B49487405E08A481B
:109B6000407C0009000188494874102020400028EA
:109B700007D08548007CF021884370308249087402
:109B800005E08148007CF02188437F49087420204B
